:100000000C94EA020C9415030C9415030C9415033C
:100010000C94ED080C9415030C9415030C94150323
:100020000C9415030C94DA320C9415030C941503FC
:100030000C9415030C94FF620C9415030C94150397
:100040000C9415030C9415030C94646B0C94150319
:100050000C941F6D0C94B56D0C9415030C94150342
:100060000C9415030C9415030C949E690C941503C1
:100070000C94586D0C94026E0C9415030C9415039B
:100080000C9415030C9415030C9415032D33002DBB
:1000900032002D31002030002B31002B32002B3369
:1000A000002B340020430020432300204400204440
:1000B0002300204500204600204623002047002042
:1000C000472300204100204123002042004D53548B
:1000D000004D494400434C4B00322F3100312F3149
:1000E00000312F3200312F3400312F3800312F31C1
:1000F0003600312F34380053494E005452490053D2
:1001000041570053515500532F4800445732004483
:100110005733004457340044573500445736005491
:100120005731005457320054573300545734004568
:10013000585000485244005346540046555A005304
:10014000504B0053545000313025003235250035D6
:1001500030250037352500393025004348524F4DB2
:100160004154494320004D414A4F52202020202035
:10017000006D696E6F7220202020200050454E5483
:1001800041544F4E494300444F5249414E20202094
:100190002000504852594749414E2020004C5944B4
:1001A00049414E20202020004D49584F4C59444988
:1001B000414E004C4F435249414E20202000464FB3
:1001C00052574152442020004241434B5741524430
:1001D000200050494E472D504F4E470052414E444B
:1001E0004F4D2020200053594E0042504D00545294
:1001F00058004356525800434C4B004E4300505455
:1002000052004C454E0053434C0054524947004C59
:10021000464F005741560046525100414D50005341
:100220005450004E5445004F4354004C454E470037
:1002300055544D0050524F00525452470050554CA7
:10024000004241520043505900415554004D414E27
:10025000004F464600204F4E0052535400504F531B
:1002600000534E4700424400534400533100533280
:10027000004C54004D540048540043500043480083
:100280004F4800435200524400E601EA013D02F7A4
:100290000145025902FB01FB01FE01020206020AAE
:1002A000020F02130217021B024102230227022B34
:1002B000020602FB01FB01FB01410230023402385D
:1002C000024102300234022B024102020206020AFB
:1002D0000261025D02FE010202BE01C801D201DC20
:1002E000015B01660171017C01870192019D01A8FA
:1002F00001B30147014B014F0153015701F700FBC7
:1003000000FF00030107010B010F01130117011B7F
:10031000011F01230127012B012F01330137013B6D
:10032000013F014301D900DD00E100E500E900EDF6
:1003300000F200CD00D100D5008C008F0092009516
:100340000098009B009E00A100A400A700AB00AE97
:1003500000B200B500B800BC00BF00C300C600CAB0
:1003600000650268026B026E027102740277027A03
:10037000027D028002830286024D0249025102552B
:100380000220202020002E2E2E2E2E2E2E2E2E2E1F
:100390002E2E2E2E2E2E00444143732063616C6955
:1003A00062726174696F6E0020696E697469616C54
:1003B000697A6174696F6E200020202020204545F5
:1003C00050524F4D2020202020002B002D00546F34
:1003D00074616C204163632076616C756520005BFD
:1003E0005341564544215D004558540020202020AB
:1003F000202020202020202020202020002020201D
:10040000200020202020002020202000202020204C
:1004100000202020536F6E6720506C6179202020CF
:1004200000736E6720706F7320707472206C656E3D
:1004300020004F6E004F6666004F6E004F666600EC
:1004400020204C464F73202043562F47617465206F
:100450000073006261722075746D2070726F20727B
:10046000747267006261722075746D2070726F2003
:100470006C656E67006C666F2077617620667271BE
:1004800020616D702000435620547261636B2053CD
:1004900063616C653A20007300626172206E74655E
:1004A000206F6374206C656E670020202000312F60
:1004B0000046494C4C00626172206C656E2073638B
:1004C0006C20747269670045585400202050617494
:1004D0007465726E20506C617920200020202042CB
:1004E0006172202020205374657020200063707991
:1004F00020727374206E6320206E63202000737955
:100500006E2062706D2070756C20636C6B20002013
:100510005472636B20646972656374696F6E200046
:10052000205074726E20646972656374696F6E2006
:10053000002B002D00202053687566666C652076C0
:10054000616C7565200076312E3033380000002153
:1005500000240027002A0000002200250028002B8C
:1005600000000020002300260029000202020202EF
:100570000202020404040404040404030303030346
:10058000030303010101010101010101020408103B
:10059000204080010204081020408001020408105D
:1005A0002040800102040810204080000000010269
:1005B0000008090000000004030706000000000016
:1005C000000000000000000000000000112E36684E
:1005D0007D6F0A2E11241FBECFEFD0E4DEBFCDBF4A
:1005E00017E0A0E0B1E0E6E8FFEE00E00BBF02C0DC
:1005F00007900D92A831B107D9F71BBE17E3A8E108
:10060000B7E001C01D92AE3FB107E1F715E0C2EDC2
:10061000D5E004C02297FE010E947B77CC3CD10735
:10062000C9F70E9413700C94B6770C940000CF9316
:10063000DF93BC018230910510F462E070E0A0917C
:10064000FC37B091FD37ED01E0E0F0E040E050E034
:1006500021C0888199818617970769F48A819B81D7
:10066000309719F09383828304C09093FD37809371
:10067000FC37FE0134C06817790738F4411551057D
:1006800019F08417950708F4AC01FE018A819B815B
:100690009C01E9012097E9F641155105A9F1CA012C
:1006A000861B970B049708F4BA01E0E0F0E02AC03B
:1006B0008D919C91119784179507F9F4641775072C
:1006C00081F412968D919C911397309719F0938332
:1006D000828304C09093FD378093FC37FD013296EE
:1006E0004CC0CA01861B970BFD01E80FF91F6193EF
:1006F000719302978D939C9340C0FD0182819381F9
:100700009C01D9011097A1F68091FA379091FB379F
:10071000892B41F480913C0190913D019093FB37EE
:100720008093FA3740913E0150913F0141155105A8
:1007300041F44DB75EB780913A0190913B01481B5F
:10074000590B2091FA373091FB37CA01821B930B6A
:100750008617970780F0AB014E5F5F4F84179507B0
:1007600050F0420F531F5093FB374093FA37F90173
:100770006193719302C0E0E0F0E0CF01DF91CF918F
:100780000895CF93DF93009709F450C0EC012297AE
:100790001B821A82A091FC37B091FD37109709F1A6
:1007A00040E050E0AC17BD0708F1BB83AA83FE010F
:1007B00021913191E20FF31FAE17BF0779F48D91AC
:1007C0009C911197280F391F2E5F3F4F3983288343
:1007D00012968D919C9113979B838A8341155105A5
:1007E00071F4D093FD37C093FC3720C012968D91E1
:1007F0009C911397AD01009711F0DC01D3CFFA0162
:10080000D383C28321913191E20FF31FCE17DF070B
:1008100069F488819981280F391F2E5F3F4FFA01B3
:10082000318320838A819B8193838283DF91CF915F
:100830000895A0E0B0E0EFE1F4E00C948777EC01DC
:10084000A880B980CA80DB80A114B104C104D1049E
:1008500041F484E2A82E89EDB82E8BE5C82E87E0FE
:10086000D82EC601B5012DE133EF41E050E00E94E2
:100870005E7727EA31E440E050E00E94EA767B01AF
:100880008C01C601B5012DE133EF41E050E00E943B
:100890005E77CA01B9012CEE34EF4FEF5FEF0E9493
:1008A000EA766E0D7F1D801F911F97FF04C0615077
:1008B000704080409048688379838A839B839B0142
:1008C000AC015F77B901CA01CDB7DEB7EAE00C949D
:1008D000A3770E941904089580E491E00E9419040E
:1008E0000895609340017093410180934201909379
:1008F00043010895A0E0B0E0E0E8F4E00C948177D3
:100900006C01009729F4CB010E9417036C01C1C050
:100910008EEF882E8FEF982E8C0C9D1C8601060F73
:10092000171F0815190508F4B2C0F401A081B181A0
:10093000A617B707B8F0A530B10508F4AAC0CD01D5
:1009400004978617970708F4A4C01297A61BB70B45
:10095000F801A193B193D4016D937C93CF010E94D0
:10096000C10397C07B01EA1AFB0AEEEFFFEFEE0E20
:10097000FF1E36016A0E7B1EC091FC37D091FD37F9
:1009800044245524AA24BB244AC0C615D705E1F542
:10099000488159814E155F05B8F1CA0104978E153B
:1009A0009F05B0F41296A40FB51FF401B183A08384
:1009B0002A813B814114510431F0D20113963C93BA
:1009C0002E93129766C03093FD372093FC3761C099
:1009D0008A819B81F80193838283425050404E1953
:1009E0005F09518340834114510431F0D2011396C1
:1009F0001C930E93129704C01093FD370093FC379D
:100A0000F4017183608345C088819981A816B90675
:100A100008F45C012E018A819B819C01E9012097E9
:100A200009F0B3CF8091FA379091FB37861597057F
:100A3000E9F4A616B706D0F420913E0130913F01AB
:100A40002115310541F42DB73EB780913A019091BF
:100A50003B01281B390B02171307C8F41093FB370F
:100A60000093FA37D4016D937C9313C0CB010E949D
:100A70001703EC01009759F0F40140815181B60150
:100A80000E945605C6010E94C1036E0102C0CC241B
:100A9000DD24C601CDB7DEB7E0E10C949D77FB0104
:100AA000DC0105900D920020E1F70895FB01DC01C7
:100AB00002C001900D9241505040D8F70895FB01BB
:100AC000DC018D91019080190110D9F3990B0895E3
:100AD000FB01DC0101900D920020E1F70895FB017C
:100AE0009F01E8944230C4F04532B4F44A3029F40E
:100AF00097FB1EF4909581959F4F642F77270E9456
:100B00001577805D8A330CF0895D8193CB01009766
:100B1000A1F716F45DE251931082C9010C94A60569
:100B2000FB019F01423074F0453264F4642F772753
:100B30000E941577805D8A330CF0895D8193CB012B
:100B40000097A1F71082C9010C94A605DC01FC01F5
:100B5000672F71917723E1F7329704C07C916D93F1
:100B600070836291AE17BF07C8F30895FC01148229
:100B7000138290E0672B09F091E0908381819817B0
:100B800079F08281882319F4913009F4938392815A
:100B9000913021F48081882309F4948380818283B9
:100BA000808181830895AF92BF92CF92DF92EF92BE
:100BB000FF920F931F93482F9091190780E0209187
:100BC000180730E0282B392B442321F0413009F05D
:100BD00056C056C04091F3335091F433E1E3F7E04F
:100BE00060E070E081E0E82EF12C012D112D1382E0
:100BF000C901062E02C0969587950A94E2F7982FB0
:100C0000917090838181981761F18281882349F5E1
:100C1000913039F5938386818F5F8683813019F017
:100C20008230F9F40DC057016801062E04C0AA0CE9
:100C3000BB1CCC1CDD1C0A94D2F74A295B2911C0CD
:100C4000168257016801062E04C0AA0CBB1CCC1CDE
:100C5000DD1C0A94D2F7D601C501809590954823F2
:100C60005923808181836F5F7F4F37966031710593
:100C700009F0BDCF4093F3335093F43302C002C068
:100C8000A901CA011F910F91FF90EF90DF90CF90C3
:100C9000BF90AF9008952F923F924F925F927F92B4
:100CA0008F929F92AF92BF92CF92DF92EF92FF927C
:100CB0000F931F93CF93DF931C017090CA09472DA8
:100CC00050E0FA01E851F14D80808294A0EF8A2231
:100CD0002091D22E30E09090D30A01E317E060E03B
:100CE00070E07A01EE0CFF1CCA01E6E0880F991F44
:100CF000EA95E1F7E80EF91E87E299E0289FE00106
:100D0000299FD00D389FD00D112426EDA22E2EE262
:100D1000B22EA40EB51E6A01CC0EDD1E83EE9AE043
:100D2000C80ED91E882D860F482E5524F701E40DD4
:100D3000F51D3D96EE0FFF1FEC0FFD1FE452F54F22
:100D40008081482F4170282F26952170C101062EE1
:100D500002C0969587950A94E2F7382F3170F80112
:100D600030838181381709F476C0942F82818823DB
:100D700009F05EC0313009F05BC0F50130834423D7
:100D800009F44DC0222329F4F6018081882309F05B
:100D90004BC0F8011682F0E17F16F9F0D701A60FDB
:100DA000B71FFD013D96EE0FFF1FEC0FFD1FE45234
:100DB000F54F8081837080838181887F8460818307
:100DC000AA0FBB1FAC0FBD1FA950B54F8C918770E8
:100DD0008C93F501308390E02BC0FB01EE0FFF1FD9
:100DE000E60FF71FEC0FFD1FDF01AF5BBC4E8C91D0
:100DF0008E7F8C93EE5BFC4E8081877080839C910C
:100E000011968C911197887F846011968C9311971D
:100E1000917098619C9390E09924939409C0F60195
:100E20008081882319F491E021E002C091E020E064
:100E3000F701E40DF51D3D96EE0FFF1FEC0FFD1FB2
:100E4000E452F54F80818C7F220F892B822B808387
:100E5000F801808181836F5F7F4F095F1F4F603191
:100E6000710509F05FCF9092D30ADF91CF911F9166
:100E70000F91FF90EF90DF90CF90BF90AF909F9039
:100E80008F907F905F904F903F902F9008957F922A
:100E90008F929F92AF92BF92CF92DF92EF92FF928A
:100EA0000F931F93CF93DF934C01C090CA094C2D31
:100EB00050E02091D22E30E0FA01E851F14DD0807F
:100EC000D29460EFD622E091D30AC1E3D7E060E08C
:100ED00070E087E299E0289F8001299F100D389FDC
:100EE000100D1124772473947A01EE0CFF1CCA01B3
:100EF00026E0880F991F2A95E1F7E80EF91EB6ED56
:100F0000AB2EBEE2BB2EA40EB51EC401062E02C03F
:100F1000969587950A94E2F7482F41704883898116
:100F2000481709F469C08A81882309F064C04130F8
:100F300009F061C08D2D860F282F30E090E0F90177
:100F4000EE0FFF1FE20FF31FE00FF11FEF5BFC4EF0
:100F5000808180FF91E0F901EE0FFF1FE20FF31F88
:100F6000E00FF11FEF5BFC4E80818E7F892B808329
:100F7000992309F03FC080E1C816F1F0D701A60F10
:100F8000B71FFD013D96EE0FFF1FE00FF11FE4526A
:100F9000F54F8081837080838181887F8460818325
:100FA000AA0FBB1FA00FB11FA950B54F8C9187701E
:100FB0008C93F50170821EC0FB01EE0FFF1FE60F40
:100FC000F71FE00FF11FDF01AF5BBC4E8C918E7FEE
:100FD0008C93EE5BFC4E8081877080839C91119690
:100FE0008C911197887F846011968C9311979170E2
:100FF00098619C93E1E049836F5F7F4F2796603152
:10100000710509F082CFE093D30ADF91CF911F9150
:101010000F91FF90EF90DF90CF90BF90AF909F9097
:101020008F907F900895BF92CF92DF92EF92FF92C0
:101030000F931F93CF93DF93EC01B090C208C09041
:1010400046025091112FD0900C0A20910F2F309111
:10105000102FE1EAF7E060E070E0A1E0EA2EF12C69
:10106000012D112D462F1382CE01062E02C096951A
:1010700087950A94E2F7982F917090838181981751
:1010800009F452C08281882309F04EC0913009F0E2
:101090004BC09383BB2029F1552381F0C901062E53
:1010A00002C0969587950A94E2F780FD23C0CC2470
:1010B000C39450E0DD2420E030E036C0D801C70101
:1010C000062E04C0880F991FAA1FBB1F0A94D2F7CF
:1010D0009C0120953095CC24C39451E0DD24D39419
:1010E00023C0C901062E02C0969587950A94E2F79F
:1010F00080FF0EC0D801C70104C0880F991FAA1F26
:10110000BB1F4A95D2F780959095282339230CC0B0
:10111000D801C701062E04C0880F991FAA1FBB1F44
:101120000A94D2F7282B392B808181836F5F7F4F00
:1011300037966031710509F095CFC0924602509301
:10114000112FD0920C0A3093102F20930F2FDF9184
:10115000CF911F910F91FF90EF90DF90CF90BF90B4
:10116000089581E00E94D305AC019093F2338093FF
:10117000F13320E030E0CA01022E02C09695879537
:101180000A94E2F780FF02C0822F08952F5F3F4F3D
:101190002031310581F78FEF089581E00E94D3055A
:1011A000AC019093F0338093EF3360E020E030E0C7
:1011B000CA01022E02C0969587950A94E2F780FF35
:1011C00005C0613011F4822F089561E02F5F3F4F19
:1011D0002031310569F780E008951F920F920FB614
:1011E0000F920BB60F9211242F933F934F935F935F
:1011F0008F939F93AF93BF93EF93FF9380B18170D1
:101200008093B3339091B3338091B4339817B9F18D
:101210008091B333882379F581E08093B5331092C0
:101220006309EEE8F3E3819323E3EF39F207D9F79B
:101230002C9A2C9810925F09109269011092680103
:1012400080E090E021E0FC01EB58F64F1082FC01B9
:10125000EF50F64F1082FC01E253F64F2083FC0161
:10126000E956F64F1082FC01E855F64F20830196AF
:101270008131910541F78091B3338093B4338091EC
:101280004E09823009F0B8C080B190E095958795FD
:1012900081708093A9339091A9338091540298175B
:1012A00009F474C080915402882311F02C9A01C073
:1012B0002C988091A933882309F065C080919F33D1
:1012C0009091A033A091A133B091A2332091A53386
:1012D0003091A6334091A7335091A833821B930BD2
:1012E000A40BB50B80934C0290934D02A0934E0239
:1012F000B0934F0280914C0290914D02A0914E020A
:10130000B0914F02885E9340A040B04080F480913D
:101310004C0290914D02A0914E02B0914F028093E9
:10132000500290935102A0935202B093530221E0D5
:101330002093AA3380919F339091A033A091A13341
:10134000B091A2338093A5339093A633A093A73393
:10135000B093A8338091C4098823C1F42093AB33A0
:10136000209355028091500290915102A091520217
:10137000B091530280934C0290934D02A0934E0281
:10138000B0934F0203C081E08093AD338091A933C5
:101390008093540280914C0290914D02A0914E0294
:1013A000B0914F02885E9340A040B04060F088EE5C
:1013B00093E0A0E0B0E080934C0290934D02A093A4
:1013C0004E02B0934F0280914C0290914D02A09139
:1013D0004E02B0914F02893C9105A105B10560F420
:1013E00088EC90E0A0E0B0E080934C0290934D0236
:1013F000A0934E02B0934F02FF91EF91BF91AF9136
:101400009F918F915F914F913F912F910F900BBEC4
:101410000F900FBE0F901F901895E82F592F4091F5
:101420003433309135332091F533222381F021304C
:1014300051F48DB38093F7339DB38091F63380954B
:1014400089238DBB04C08FB7F8948093F7334CBDCC
:101450003DBD5D985EBD00000DB407FEFDCF8EB5AD
:10146000EEBD00000DB407FEFDCF8EB57EBD0000C1
:101470000DB407FEFDCF8EB56EBD00000DB407FEA6
:10148000FDCF8EB55D9A222339F08091F73321305C
:1014900011F48DBB01C08FBF50932207E093210749
:1014A0007093200760931F070895682F592F40916C
:1014B0003433309135332091F533222381F02130BC
:1014C00051F48DB38093F7339DB38091F6338095BB
:1014D00089238DBB04C08FB7F8948093F7334CBD3C
:1014E0003DBD5C985EBD00000DB407FEFDCF8EB51E
:1014F0006EBD00000DB407FEFDCF8EB55C9A2223B1
:1015000039F08091F733213011F48DBB01C08FBFCA
:1015100050931E0760931D07089540913433309116
:1015200035332091F533222381F0213051F48DB3EE
:101530008093F7339DB38091F633809589238DBBDB
:1015400004C08FB7F8948093F7334CBD3DBD5C98D1
:101550001EBC00000DB407FEFDCF8EB51EBC000002
:101560000DB407FEFDCF8EB55C9A222339F0809131
:10157000F733213011F48DBB08958FBF08959C017E
:101580003F70306160913433509135334091F53381
:10159000442381F0413051F48DB38093F7339DB3F0
:1015A0008091F633809589238DBB04C08FB7F89462
:1015B0008093F7336CBD5DBD12983EBD00000DB445
:1015C00007FEFDCF8EB52EBD00000DB407FEFDCF8A
:1015D0008EB5129A442339F08091F733413011F4DB
:1015E0008DBB08958FBF08959C013F70306160915D
:1015F0003433509135334091F533442381F04130F9
:1016000051F48DB38093F7339DB38091F633809579
:1016100089238DBB04C08FB7F8948093F7336CBDDA
:101620005DBD13983EBD00000DB407FEFDCF8EB525
:101630002EBD00000DB407FEFDCF8EB5139A4423D6
:1016400039F08091F733413011F48DBB08958FBF8D
:1016500008959C013F703069609134335091353367
:101660004091F533442381F0413051F48DB38093A0
:10167000F7339DB38091F633809589238DBB04C0E9
:101680008FB7F8948093F7336CBD5DBD13983EBD62
:1016900000000DB407FEFDCF8EB52EBD00000DB4C9
:1016A00007FEFDCF8EB5139A442339F08091F733AE
:1016B000413011F48DBB08958FBF089540913433AC
:1016C000309135332091F533222381F0213051F4CC
:1016D0008DB38093F7339DB38091F6338095892342
:1016E0008DBB04C08FB7F8948093F7334CBD3DBDDC
:1016F0005E9A1EBC00000DB407FEFDCF8EB51EBC69
:1017000000000DB407FEFDCF8EB580938C331EBC58
:1017100000000DB407FEFDCF8EB51EBC00000DB459
:1017200007FEFDCF8EB51EBC00000DB407FEFDCF39
:101730008EB580938A3380938B335E98222339F061
:101740008091F733213011F48DBB08958FBF089538
:101750009C0143B148704093363393B19470909399
:101760003733442311F5809138338823F1F09923DE
:1017700019F0260F371F19C08091C908882381F0FE
:1017800080914333813041F0813010F0823069F430
:101790002A30310554F007C02031310534F003C040
:1017A0002115310511F0261B370B40933833C90141
:1017B0000895482F53B1527050933C3393B19170B8
:1017C00090933D335523D9F480913E338823B9F06B
:1017D000992369F08FEF90E0841B9109262F30E068
:1017E0008217930714F44FEF0AC0460F08C046173C
:1017F00020F4442321F0462F02C04111461B509390
:101800003E33842F90E00895CF92DF92EF92FF92C3
:101810000F931F93CF93DF93EC01F42EE22E680118
:1018200018811093DE33812F0E94D90B8883F8161C
:1018300008F0F88288818E1508F0E8828881811787
:1018400039F08093DE3381E0F60180838093460295
:10185000DF91CF911F910F91FF90EF90DF90CF908C
:1018600008950F931F93DF93CF930F92CDB7DEB7F9
:1018700089838091D22E90E027E239E0829FF001A7
:10188000839FF00D929FF00D1124E45CFC4E2081AB
:10189000203311F0203609F428E12150CE010196C1
:1018A00061E040E003ED1AE00E94040C698160935E
:1018B000040A8091F408882331F18091D22E90E0BF
:1018C00040E050E027E239E0829FD001839FB00DD5
:1018D000929FB00D1124962F9F71990FFA01EE0F70
:1018E000FF1FE40FF51FEA0FFB1FEF5BFC4E80812B
:1018F000817C892B80834F5F5F4F4034510571F7A6
:1019000081E08093D30A862F0F90CF91DF911F91B2
:101910000F9108951F93FC0113B1127010933C3383
:1019200093B1917090933D33112361F580913E33D3
:10193000882341F19923D1F0CF01A0E0B0E02FEF4F
:101940003FEF40E050E0281B390B4A0B5B0B862F22
:1019500090E0A0E0B0E0281739074A075B071CF4C5
:10196000EFEFFFEF0FC0E60FF11D0CC070E0E617C0
:10197000F70720F4309731F0FB0104C0309711F0E5
:10198000E61BF70B10933E33CF011F9108959C0186
:1019900043B1427040933C3393B1917090933D3387
:1019A000442309F580913E338823E9F070E09923C0
:1019B00069F08FEF9FE7821B930B861797071CF444
:1019C0002FEF3FE710C0260F371F0DC02617370730
:1019D0002CF42115310539F09B0105C02115310585
:1019E00011F0261B370B40933E33C9010895AF9287
:1019F000BF92CF92DF92EF92FF920F931F93CF93FC
:101A0000DF93EC017A016901580108811981109373
:101A1000DD330093DC33C8010E94C70C99838883AF
:101A2000E816F90614F0F982E882888199818C150C
:101A30009D0514F0D982C882888199818017910709
:101A400049F09093DD338093DC3381E0F5018083AE
:101A500080934602DF91CF911F910F91FF90EF90FD
:101A6000DF90CF90BF90AF9008959F92AF92BF92BA
:101A7000CF92DF92EF92FF920F931F937B018C0125
:101A800059016A0193B082E0982290923C3393B15D
:101A9000917090933D339920D9F580913E338823FE
:101AA000B9F1992329F0C801B7010E94D5742EC05D
:101AB0008091C9088823D1F080914333813059F057
:101AC000813010F0823021F5C801B70120E030E00C
:101AD00040E251E406C0C801B70120E030E040E830
:101AE00051E40E94837688239CF00AC0C801B701A4
:101AF00020E030E040E050E00E943975882341F05A
:101B0000C801B701A60195010E94D4747B018C0124
:101B100090923E33B701C8011F910F91FF90EF9053
:101B2000DF90CF90BF90AF909F90089523B1227027
:101B300020933C3393B1917090933D331092DB33FB
:101B40001092DA33222379F480913E33882359F0BE
:101B5000992319F081E090E002C08FEF9FEF9093FE
:101B6000DB338093DA3320933E338091DA339091E4
:101B7000DB330895EF92FF920F931F93CF93DF9380
:101B8000582F2091D22E803109F04DC030E0A0E0D6
:101B9000B0E087E299E0289F7001299FF00C389F00
:101BA000F00C1124062F10E0C42FD0E0742F729592
:101BB000770F770F707C469546954770562F529554
:101BC000550F550F507C669566956770FD01EE0FB9
:101BD000FF1FEA0FFB1FEE0DFF1DEF5BFC4E208188
:101BE000922F92959695969593703181832F877059
:101BF000880F880F892B90E08017910734F42F739A
:101C0000252B2083387F362B08C08C179D0734F096
:101C10002F73272B2083387F342B31831196A034E8
:101C2000B105A1F689C030E0A0E0B0E087E299E01C
:101C3000289FE001299FD00D389FD00D1124062F39
:101C400010E0242F30E0F42EF294FF0CFF0C80EC17
:101C5000F822469546954770762F7295770F770F45
:101C6000707C669566956770852F90E0FC0168949E
:101C700015F8EE0FFF1F1694E1F7880F991FE80F74
:101C8000F91FEA0FFB1F3D96EE0FFF1FEC0FFD1F24
:101C9000E452F54F90819295969596959370818137
:101CA0008770880F880F892B90E080179107F4F4D4
:101CB000852F90E0FC01689415F8EE0FFF1F169435
:101CC000E1F7880F991FE80FF91FEA0FFB1F3D96F8
:101CD000EE0FFF1FEC0FFD1FE452F54F80818F7355
:101CE000872B80838181887F862B20C08217930772
:101CF000F4F0852F90E0FC01689415F8EE0FFF1FBB
:101D00001694E1F7880F991FE80FF91FEA0FFB1FE0
:101D10003D96EE0FFF1FEC0FFD1FE452F54F808143
:101D20008F738F2980838181887F842B8183119693
:101D3000A034B10509F098CFDF91CF911F910F9199
:101D4000FF90EF9008952F923F924F925F926F9283
:101D50007F928F929F92AF92BF92CF92DF92EF923B
:101D6000FF920F931F93DF93CF93CDB7DEB76097AA
:101D70000FB6F894DEBF0FBECDBF8091090988234E
:101D800051F0809124028F5F80932402883018F0F4
:101D900087E08093240280910209882349F0809192
:101DA0002402815080932402883010F01092240283
:101DB000DE011196E7EDF6E080E101900D92815091
:101DC000E1F78091D22E482F50E087E299E0489FBA
:101DD000F001499FF00D589FF00D1124E55CFC4E79
:101DE000E081E33018F4E13048F405C0E33049F015
:101DF000E93048F403C0ACE0AA2E05C0F7E0AF2EEE
:101E000002C0E5E0AE2E8091C409882309F444C0E5
:101E10008091C909813009F03FC08091D20A88239E
:101E2000D9F18091960990E0FC01EE0FFF1FE80FB9
:101E3000F91F87E299E0489F9001499F300D589F14
:101E4000300D1124E20FF31FED5BFC4E9091D9335E
:101E50009F708081807F892B80838091960990E09C
:101E6000FC01EE0FFF1FE80FF91FE20FF31FEF5BFE
:101E7000FC4E8081817C806380838091960990E014
:101E8000FC01EE0FFF1FE80FF91FE20FF31FEF5BDE
:101E9000FC4E808181608083B090D93301E118E0ED
:101EA000EE24FF242E010894411C511C8A2C9924F5
:101EB00047E2642E49E0742E3324339437E0232E16
:101EC000F801138280912709909128090E2C02C0F5
:101ED000969587950A94E2F7982F91709083818167
:101EE000981709F4CBC08281882309F0C4C09130CF
:101EF00009F0C1C09383F201EE0DFF1DE0818E2F2A
:101F000090E06A2D70E00E9415779B018091240279
:101F1000860F80932502883010F020922502289D9C
:101F2000C001299D900D389D900D11242E2F281B46
:101F30008091D22E90E0869DF001879DF00D969DB8
:101F4000F00D1124E55CFC4E8081833018F4813063
:101F500058F405C0833069F0893080F405C0E22F61
:101F6000F0E0E854FE4F09C0E22FF0E0E455FE4FE8
:101F700004C0E22FF0E0ED54FE4FB08090E0FC0191
:101F8000EE0FFF1FE80FF91FEE0FFF1FEE0FFF1FF1
:101F9000EB0DF11DE854FE4FE081F0E0EE0FFF1F66
:101FA000EE56FE4F80912502D82EDD0CCC24808188
:101FB00091818C0D9D1D0E94BF0A5F9A3092D20ABA
:101FC0008091C409882309F456C08091C9098130E1
:101FD00009F051C02091D22E30E08091960990E016
:101FE000FC01EE0FFF1FE80FF91FA901469D9001AC
:101FF000479D300D569D300D1124E20FF31FED5B10
:10200000FC4E9B2D9F708081807F892B80838091E7
:10201000960990E0FC01EE0FFF1FE80FF91FE20F99
:10202000F31FED5BFC4E9091250297709295907F87
:1020300080818F78892B80838091960990E0FC01C4
:10204000EE0FFF1FE80FF91FE20FF31FEF5BFC4ECF
:102050008081817C886180838091960990E0FC0179
:10206000EE0FFF1FE80FF91FE20FF31FEF5BFC4EAF
:10207000808181608083F801808181830894E11CE4
:10208000F11C095F1F4FF0E1EF16F10409F018CFC2
:10209000B092D9338091270990912809892B21F595
:1020A0008091D20A882301F15F981092D20A809120
:1020B000960990E02091D22E30E0FC01EE0FFF1F38
:1020C000E80FF91F87E299E0AC01249FC001259F2A
:1020D000900D349F900D1124E80FF91FEF5BFC4E1B
:1020E0008081817C8861808360960FB6F894DEBF22
:1020F0000FBECDBFCF91DF911F910F91FF90EF9059
:10210000DF90CF90BF90AF909F908F907F906F9017
:102110005F904F903F902F900895EF92FF920F9312
:102120001F9304E013E37801E80EF11C609153095A
:102130007091540980E090E00E94D1752091323373
:10214000020F111DD8015496EC91F0E0EE0FFF1F25
:10215000EE0FFF1FEA5DFD4F2081318142815381E7
:102160000E9487769B01AC0160E070E080E792E41A
:102170000E943D7521E338E04CEA5CEB0E943D751E
:1021800020E030E040E853E40E94D5740E94A57539
:10219000F70162831F910F91FF90EF9008953F9296
:1021A0004F925F926F927F928F929F92AF92BF9267
:1021B000CF92DF92EF92FF920F931F93CF93DF9313
:1021C0006090C20860923F099090C90890923E09C1
:1021D00070901D09709240098090BB08809241095F
:1021E00080919F08809342092091D708209343094A
:1021F00080910109809344099091080990934509C1
:10220000A82FB0E0AA0FBB1FAA0FBB1F492F50E099
:10221000F3E0440F551FFA95E1F7622F70E0E5E017
:10222000660F771FEA95E1F790913709990F9A2B7E
:1022300080913B09982B942B80913C098295807F5B
:10224000892B862B80932F09E0905909F0905A0929
:1022500021E0E216F10419F4B090440108C0E11441
:10226000F10419F4BB24B39402C0B090F308B09207
:102270003B09C7010397029720F08CE0E816F104B0
:1022800019F40091440106C000E022E0E216F104D6
:1022900009F401E00093370984E0E816F10421F025
:1022A0002CE0E216F10419F4A090440105C08091DD
:1022B000A608811181E0A82EA092380980910333ED
:1022C000882321F081E08093350906C08091DE08E3
:1022D000809335098091E508809336092091AD08F7
:1022E0002093390981E090E00090A30802C0880F94
:1022F000991F0A94E2F78093470980919C08809384
:102300003A098091C909882341F081E08093480906
:1023100010914809E6EDFEE216C08091D52E882383
:1023200061F480915809882341F48091D30A88236D
:1023300021F480913333882319F080914401E6CF52
:1023400010924809E5CF8081882311F01091440153
:1023500031968EE2E63EF807B1F71093480985E022
:10236000E816F10421F481E080933C0902C0109248
:102370003C09C0900F2FD090102FD0924D09C092E1
:102380004C0988E0E816F10419F48091440102C078
:102390008091B40880933D09E091C40930E0EE23B8
:1023A00009F431E030933409EE2311F081E002C0EA
:1023B00080914401809346094A2B5B2B462B572B77
:1023C00080913C0990E074E0880F991F7A95E1F7BD
:1023D000482B592B882D90E066E0880F991F6A954D
:1023E000E1F7482B592B822F90E09695982F88275C
:1023F00097958795482B592B972D80E0482B592B83
:10240000962D990F990F80E0482B592B992D990FF4
:10241000990F990F80E0482B592B20914609922F54
:102420009295907F80E0482B592B912F9295990F90
:10243000990F907C80E0482B592B932F9295990F00
:10244000907E80E0482B592B8B2D90E0482B592B08
:10245000802F90E0880F991F482B592B9A2D990FA8
:1024600080E0482B592B50933109409330096090FC
:10247000CA09C62DD0E021E030E0C901062C02C017
:10248000880F991F0A94E2F790934A0980934909AB
:1024900044E0E416F10409F426C265E0E616F1040E
:1024A00064F472E0E716F10411F143E0E416F1047C
:1024B0000CF0E7C0F7FE3EC253C267E0E616F10437
:1024C00009F4DFC078E0E716F10434F485E0E8169B
:1024D000F10409F045C23AC229E0E216F10409F418
:1024E000D0C04CE0E416F10409F03AC2FCC180917E
:1024F000F308882341F00090CB0902C0220F331F5C
:102500000A94E2F71EC2EE2309F46CC090910B2FDF
:10251000992309F44BC080910C2F482F50E04F7045
:10252000507060E070E020E030E0E92FF0E011E072
:10253000E12EF12C012D112D10C0C901840F951F22
:102540005701680104C0AA0CBB1CCC1CDD1C8A9579
:10255000D2F76A297B292F5F3F4FE217F3076CF709
:1025600080914401FE01EB5BFE4FE081CC59D64FD8
:10257000288140E050E0882311F441E050E0809150
:10258000CC098F7002C0440F551F8A95E2F7409521
:102590005095642375238E2F90E02F7002C0880F12
:1025A000991F2A95E2F7682779275AC0409144017C
:1025B000FE01EB5BFE4F8081CC59D64F288190E025
:1025C0002F7002C0880F991F2A95E2F750E02091E2
:1025D000CC092F7002C0440F551F2A95E2F78427BB
:1025E0009527BAC190910B2F992309F43EC0809191
:1025F0000C2F482F50E04F70507060E070E020E0EA
:1026000030E0E92FF0E0B1E0EB2EF12C012D112D9F
:1026100010C0C901840F951F5701680104C0AA0C9E
:10262000BB1CCC1CDD1C8A95D2F76A297B292F5F45
:102630003F4FE217F3076CF78091440120E030E050
:10264000882311F421E030E08091CC098F7002C022
:10265000220F331F8A95E2F720953095622373236A
:1026600070932A09609329097BC18091440190E00D
:102670002091CC092F7002C0880F991F2A95E2F78C
:102680006BC1992009F068C1FE01E851F14D7080DD
:10269000372C3294A0EF3A222091D22E30E040E045
:1026A00050E000E010E060E070E04E01880C991C02
:1026B000CE01E6E0880F991FEA95E1F7880E991E92
:1026C00087E299E0289F2001299F500C389F500CE9
:1026D000112421E0A22EB12CC12CD12C832D840FEA
:1026E000A82FB0E020E1621669F4FD01EE0FFF1F94
:1026F000EA0FFB1FE40DF51DEF5BFC4E808180FFB0
:102700003DC010C0A80DB91D1D96AA0FBB1FA40D7A
:10271000B51DA452B54F8C91982F917081FF0FC0B9
:102720009923E1F0D601C501042E04C0880F991F3A
:10273000AA1FBB1F0A94D2F7682B792B1FC09923BD
:1027400069F0D601C501042E04C0880F991FAA1F85
:10275000BB1F0A94D2F7082B192B10C0D601C50154
:10276000042E04C0880F991FAA1FBB1F0A94D2F71A
:102770008095909568237923082319234F5F5F4F35
:102780004034510509F0AACF00932D0910932E096A
:1027900060932B0970932C09FE01E750F14D3081B5
:1027A0007316B1F4FE01EB5BFE4F8081FE01EC5924
:1027B000F64F208190E02F7002C0880F991F2A9554
:1027C000E2F78627972790932A098093290904C066
:1027D00070932A096093290980914B09883C08F17C
:1027E0007316B9F4FE01EB5BFE4F8081CC59D64FD6
:1027F000288190E02F7002C0880F991F2A95E2F778
:1028000080279127862B972B90932A09809329095B
:1028100006C0062B172B10932A0900932909109242
:102820004B0947E0E416F10429F069E0E616F104EB
:1028300009F096C07720A1F480916209803108F0F8
:102840008FC02091440130E002C0220F331F8A95CF
:10285000E2F78091290990912A09822793277CC069
:1028600071E0771679F420916209203208F078C07F
:10287000203108F475C08091440190E030E020518F
:10288000304025C082E0781679F420916209203327
:1028900008F066C0203208F463C08091440190E0E3
:1028A00030E02052304013C013E0A12E7A1409F01A
:1028B00057C020916209203408F052C0203308F438
:1028C0004FC08091440190E030E02053304002C07E
:1028D000880F991F2A95E2F72091290930912A093A
:1028E000282739272EC080914E098823A9F081E03E
:1028F0000E94D3052091C1093091C209409133094A
:1029000050E069014C9D90014D9D300D5C9D300D56
:102910001124282B392B15C00091BD091091BE0937
:1029200081E00E94D305082B192B10932A090093EC
:10293000290916C00090132F02C0220F331F0A94DA
:10294000E2F730932A09209329090AC08091BB0934
:102950009091BC098C299D2990932A09809329097B
:1029600060913009709131098091290990912A096B
:1029700040912F090E940D0ADF91CF911F910F9175
:10298000FF90EF90DF90CF90BF90AF909F908F908F
:102990007F906F905F904F903F900895DF92EF92FD
:1029A000FF920F931F93CF93DF932091D22E80310C
:1029B00009F480C0422F50E0282F30E084E890E0F6
:1029C000289FD001299FB00D389FB00D112487E2B8
:1029D00099E0BA01689FA001699F500D789F500D42
:1029E0001124FD01E40FF51FE452F54FE656FF4FA9
:1029F0000191A65DB24EA656BF4F0D9380818C9378
:102A00001296329680818C9382918E93D901A65D25
:102A1000B24EFA01E452F54FE20FF31F8781179689
:102A20008C9310E0B901F6E0660F771FFA95E1F795
:102A3000220F331F620F731FEA01DB01A10FB11DCB
:102A40001D96FD01EE0FFF1F1D97AF01465D524E13
:102A5000EC0FFD1FE452F54F8081282F229526951B
:102A60002695237091819770990F990F922B292F9A
:102A70002295220F220F207C8F73822BFA018083F4
:102A80009695969597708181887F892B8183AA0F6F
:102A9000BB1FFD01EB5BF24EAC0FBD1FA950B54F44
:102AA0009C91987F80818770892B80831F5F01179D
:102AB00020F678C030E087E299E0A901489F9001B4
:102AC000499F300D589F300D1124F901E452F54F04
:102AD000EF59F74FD080D0928B25829180938A2531
:102AE0003296819180938C25808180938D253497B7
:102AF00080818093892500E0E901802F90E0DC014E
:102B0000AA0FBB1FA80FB91F9D0121573A4DBD0148
:102B10006C0F7D1F81E4E82E83E1F82EE60EF71E90
:102B2000F7011081912F9170F90180818E7F892B9F
:102B30008083AD014F565A4DFB01ED5BFC4E808109
:102B4000FA018083912F9E73F9018081817C892B0A
:102B50008083A057BA4D6E5B7C4EFB019081987FBD
:102B60008C918770892B8C931295169516951370FE
:102B7000F70191819770990F990F912B492F4295E9
:102B8000440F440F407CF90180818F73842B808334
:102B9000969596958181887F892B81830F5FD016CA
:102BA00008F0ABCFDF91CF911F910F91FF90EF9085
:102BB000DF900895AF92BF92CF92DF92EF92FF9293
:102BC0000F931F93CF93DF932091D22E803109F47E
:102BD000A1C0422F50E0A82EBB24262F30E084E86D
:102BE00090E0289FD001299FB00D389FB00D11248F
:102BF000A65DB24EA656BF4FFD90A89EF001A99EBD
:102C0000F00DB89EF00D112487E299E0BA01689F9B
:102C1000A001699F500D789F500D1124E40FF51FFE
:102C2000E452F54FE656FF4FF1928C918083329635
:102C300012968C9180838E918293FA01E452F54F23
:102C4000EA0DFB1DD901A65DB24E17968C918783C4
:102C5000EE248501000F111FC501F6E0880F991FB2
:102C6000FA95E1F7080F191F6A01B901E6E0660F4E
:102C7000771FEA95E1F7220F331F620F731F8E2D26
:102C800090E09801280F391FF9013D96EE0FFF1FC4
:102C9000EC0DFD1DE452F54FDB01A80FB91FAA0F83
:102CA000BB1FCD018C5B924EEC014881542F529595
:102CB00056955695537099819770990F990F952B4A
:102CC000892F8295880F880F807C4F73482B408313
:102CD0009695969597708181887F892B8183220FA5
:102CE000331F2C0D3D1D2950354FAB5BB24E9C91CF
:102CF000987FF90180818770892B8083E394FE148B
:102D000008F0BDCF46ED5EE2A40EB51E81E0E50100
:102D100088837BC030E0D0908B2587E299E0F90171
:102D2000E89F9001E99F300DF89F300D1124F901C3
:102D3000E452F54FEF59F74FD08280918A25829364
:102D4000329680918C25819380918D258083349754
:102D500080918925808300E0E901802F90E0DC01EB
:102D6000AA0FBB1FA80FB91FBD016C0F7D1F9B01D0
:102D70002F5B3C4E1FE8E12E15E2F12EEA0EFB1E02
:102D8000F7011081912F9170F90180818E7F892B3D
:102D90008083AB014D5B5C4EFD01EF56FA4D8081A7
:102DA000FA018083912F9E73F9018081817C892BA8
:102DB00080836E5B7C4EA057BA4D9C91987FFB013F
:102DC00080818770892B80831295169516951370D4
:102DD000F70191819770990F990F912B492F429587
:102DE000440F440F407CF90180818F73842B8083D2
:102DF000969596958181887F892B81830F5FD01668
:102E000008F0ABCF81E08093D30A81E08093460243
:102E1000DF91CF911F910F91FF90EF90DF90CF90B6
:102E2000BF90AF900895CF93DF932091D22E30E0E2
:102E3000C82FD0E084E890E0C89FF001C99FF00D52
:102E4000D89FF00D112487E299E0A901489F9001D5
:102E5000499F300D589F300D1124E20FF31FE452AB
:102E6000F54FE656FF4F8FE0819388E180833296DD
:102E700081E08083129240E050E0BE01660F771F30
:102E8000CE01E6E0880F991FEA95E1F7680F791FF8
:102E9000DB01A40FB51FFD013D96EE0FFF1FE20FF2
:102EA000F31FE452F54F82E080838181887F846044
:102EB0008183AA0FBB1FA20FB31FA950B54F8C91DE
:102EC00087708C934F5F5F4F4034510509F7CA52AA
:102ED000D14D81E0888380934602DF91CF910895A0
:102EE000CF93DF938091D22E90E027E239E0A901C1
:102EF000849F9001859F300D949F300D1124F9011E
:102F0000E452F54FEF59F74F8FE0808388E18293C9
:102F1000329681E0819310823497108240E050E035
:102F2000B901FA01EE0FFF1FE40FF51FE60FF71FBF
:102F3000DF01AF5BBC4E8C918E7F8C93CF018D5B9C
:102F40009C4E20E3EC0128838C91817C88618C93DA
:102F5000EE5BFC4E8081877080838C918F738C93A5
:102F600011968C911197887F846011968C934F5F96
:102F70005F4F40345105A9F681E08093D30A8093D6
:102F80004602DF91CF9108951F9310E0812F0E9498
:102F9000CE141F5F1131D1F78091043380931B331E
:102FA0008091063380931D338091083390910933CB
:102FB000A0910A33B0910B3380931F339093203349
:102FC000A0932133B09322338091163380932D3315
:102FD0008091183380932F338091053380931C3375
:102FE0008091073380931E3380910C3390910D3381
:102FF000A0910E33B0910F338093233390932433F9
:10300000A0932533B09326338091173380932E33CA
:1030100080911933809330331F9108951F9310E0EE
:10302000812F612F0E94DA151F5F1131C9F780913E
:103030001B338093043380911D338093063380913A
:103040001F3390912033A0912133B091223380938C
:10305000083390930933A0930A33B0930B338091D4
:103060002D338093163380912F33809318338091C2
:103070001C338093053380911E33809307338091F6
:10308000233390912433A0912533B091263380933C
:103090000C3390930D33A0930E33B0930F33809184
:1030A0002E338093173380913033809319331F91DF
:1030B00008951F9310E0812F0E9413171F5F103196
:1030C000D1F70E9470171F910895CF92DF92EF926F
:1030D000FF920F931F93CF93DF93082FE42E20913D
:1030E000D22E803161F430E0F62E87E299E0289FFD
:1030F0006001299FD00C389FD00C11248AC130E088
:10310000162F87E299E0289FE001299FD00D389F74
:10311000D00D11240AC1612F70E0412F4F7050E093
:10312000802F90E0DC0126E0AA0FBB1F2A95E1F773
:10313000880F991FA80FB91FA60FB71F1D96AA0FBA
:10314000BB1FAC0FBD1FA452B54F802F90E0FC01F8
:1031500036E0EE0FFF1F3A95E1F7880F991FE80F51
:10316000F91FE40FF51F3D96EE0FFF1FEC0FFD1F3B
:10317000E452F54F908191708C918E7F892B8C93C6
:10318000802F90E0DC0126E0AA0FBB1F2A95E1F713
:10319000880F991FA80FB91FA60FB71F1D96AA0F5A
:1031A000BB1FAC0FBD1FA452B54F802F90E0FC0198
:1031B00036E0EE0FFF1F3A95E1F7880F991FE80FF1
:1031C000F91FE40FF51F3D96EE0FFF1FEC0FFD1FDB
:1031D000E452F54F908192708C918D7F892B8C9366
:1031E000802F90E0DC0126E0AA0FBB1F2A95E1F7B3
:1031F000880F991FA80FB91FA60FB71F1D96AA0FFA
:10320000BB1FAC0FBD1FA452B54F802F90E0FC0137
:1032100036E0EE0FFF1F3A95E1F7880F991FE80F90
:10322000F91FE40FF51F3D96EE0FFF1FEC0FFD1F7A
:10323000E452F54F90819C738C91837C892B8C9305
:10324000802F90E0DC0126E0AA0FBB1F2A95E1F752
:10325000880F991FA80FB91FA60FB71F1D96AA0F99
:10326000BB1FAC0FBD1FA452B54F802F90E0FC01D7
:1032700036E0EE0FFF1F3A95E1F7880F991FE80F30
:10328000F91FE40FF51F3D96EE0FFF1FEC0FFD1F1A
:10329000E452F54F80818295869586958370918161
:1032A0009770990F990F982B292F2295220F220F93
:1032B000207C8C918F73822B8C939695969511968A
:1032C0008C911197887F892B11968C93802F90E099
:1032D000DC01F6E0AA0FBB1FFA95E1F7880F991FF2
:1032E000A80FB91FA60FB71FAA0FBB1FAC0FBD1F9A
:1032F000A950B54F802F90E0FC0136E0EE0FFF1F84
:103300003A95E1F7880F991FE80FF91FE40FF51FB1
:10331000EE0FFF1FEC0FFD1FE950F54F9081987FD6
:103320008C918770892B8C931F5FE11608F0F3CE88
:10333000E02FF0E0EA52F14D81E0808370C02F2D44
:1033400030E08F2D8F7090E0D901AA0FBB1FA20F24
:10335000B31FAC0DBD1DBD016F5B7C4EFC01EE0FBC
:10336000FF1FE80FF91FEC0DFD1D8F010F5B1C4EB9
:10337000E80198819170EB0188818E7F892B888389
:10338000AD014D5B5C4E9F012D5B3C4EE901988188
:103390009F70EA018881807F892B8883E901988169
:1033A00090778F78892BEA018883E901988190785A
:1033B0008F77892BEA018883E80198819E73EB015E
:1033C0008881817C892B8883AE5BBC4EEE5BFC4E92
:1033D0009081987F8C918770892B8C93F8018081E4
:1033E000829586958695837091819770990F990F34
:1033F000982B292F2295220F220F207C88818F73F2
:10340000822B8883969596958981887F892B8983DD
:10341000F394EF1408F093CF81E08093D30A81E016
:1034200080934602DF91CF911F910F91FF90EF9013
:10343000DF90CF9008952F923F924F925F926F92BC
:103440007F928F929F92AF92BF92CF92DF92EF9234
:10345000FF920F931F93DF93CF9300D000D000D043
:10346000CDB7DEB72091D22E803109F0F8C0A22E60
:10347000BB2487E299E0A89E9001A99E300DB89EDA
:10348000300D1124F901E35CFC4E9080D901AF5B53
:10349000BC4E9C91882483948922F901ED5BFC4EFB
:1034A00080817FE0772E7822182F12951770C82E12
:1034B000CC1CCC24CC1CF92EF6948FE1F822F90117
:1034C000EE5BFC4ED080D694D694D6949295969589
:1034D0009695937011960C910770000F000F092BB1
:1034E000EE24E394190171C02E2D30E0C90101973B
:1034F000AC01440F551F480F591F420D531DBA010F
:103500006F5B7C4ED901AA0FBB1FA20FB31FA20D88
:10351000B31DFD01EF5BFC4EFA83E983908191704E
:10352000FB0180818E7F892B80839A012D5B3C4E2D
:1035300083E4482E83E1582E4A0E5B1EF2019081EF
:103540009F70F9018081807F892B8083F2019081B7
:1035500090778F78892BF9018083F20190819078A0
:103560008F77892BF9018083E981FA8180818295A7
:1035700086958695837091819770990F990F982BF6
:10358000292F2295220F220F207CFB0180818F732F
:10359000822B8083969596958181887F892B818364
:1035A0004E5B5C4EAE5BBC4E9C91987FDA018C9179
:1035B0008770892B8C93E981FA8190819E73DB015E
:1035C0008C91817C892B8C93E3949E1408F08CCF92
:1035D000892D90E0FC01EE0FFF1FE80FF91F87E235
:1035E00099E09C01A29EC001A39E900DB29E900DF9
:1035F0001124E80FF91F9F012F5B3C4ED9018C91DC
:103600008E7F88298C93CF018D5B9C4E177012950D
:10361000107FC794CC24C79417291C29DC011C9364
:10362000902F9295990F990F907CD9018C918F735F
:10363000892B8C93EE5BFC4EDD0CDD0CDD0C0695CE
:1036400006950D290083BFE1FB22FF0CF901808163
:10365000817C8F29808381E08093D30AF5C0422E3C
:103660005524E82EFF2484E890E0E89ED001E99EEE
:10367000B00DF89EB00D112487E299E0489E9001AC
:10368000499E300D589E300D1124A20FB31FFD012D
:10369000EA58F44F3080FD01EA50F54F8081222432
:1036A00023942822582F56955170082F0695069579
:1036B0000F70829586958695837011811770110F12
:1036C000110F182BA950B54FCC90C694C694C69430
:1036D000DD24D3943701660C771C4701F6E0880C93
:1036E000991CFA95E1F75301A80CB91C3E832D8370
:1036F00069C0AD2DB0E01197B5016A0F7B1F9D0128
:103700002F5F3F4F3C832B839B01235F3F4F220F53
:10371000331F8D819E81280F391F2452354FAB8175
:10372000BC81AA0DBB1DBC83AB83FD013D96EE0F92
:10373000FF1FE80FF91FE452F54F90819170D901F6
:103740008C918E7F892B8C93908192708D7F892BA9
:103750008C9390819C73837C892B8C9340814295C0
:1037600046954695437091819770990F990F942BC8
:10377000492F4295440F440F407C8F73842B8C93C8
:103780009695969511968C911197887F892B119615
:103790008C93660F771FED81FE816E0F7F1F69503E
:1037A000754F2B813C81220F331F2E0F3F1F295055
:1037B000354FD9019C91987FFB0180818770892BBF
:1037C0008083D3943D1408F094CFD301A80DB91D84
:1037D000A30DB11DFD013D96EE0FFF1F87E299E09D
:1037E000489E9001499E300D589E300D1124E20FE5
:1037F000F31FE452F54F5170550F52700F70000FC8
:10380000000F5229812F8295880F880F807C502BC2
:10381000582B5083169516958181887F812B818343
:10382000AA0FBB1FA20FB31FA950B54FCC0CCC0CD5
:10383000CC0C8C9187708C298C9326ED3EE2E20EA5
:10384000F31E81E0D7018C938091590990915A0918
:103850008930910511F0079719F481E080934602B1
:1038600026960FB6F894DEBF0FBECDBFCF91DF9185
:103870001F910F91FF90EF90DF90CF90BF90AF908E
:103880009F908F907F906F905F904F903F902F9080
:1038900008952F923F924F925F926F927F928F92F4
:1038A0009F92AF92BF92CF92DF92EF92FF920F93CF
:1038B0001F93DF93CF9300D000D000D0CDB7DEB7F9
:1038C0004091D22E803109F009C1442E552487E25F
:1038D00099E0489EA001499E500D589E500D11241C
:1038E000FA01E35CFC4E208130E0F901EE0FFF1F8E
:1038F000E20FF31FE40FF51FBF016F5B7C4EDB018E
:103900009C91662463946922DF01AD5BBC4E8C916F
:10391000B82FBF70BA83782E771C7724771CE82ED7
:10392000E294AFE0EA2217E0E122B92EB6948FE1EB
:10393000B822EE5BFC4EA080A694A694A694929525
:10394000969596959370DB011196FC90F122FF0CF1
:10395000FF0CF92A1C821B826901160108942108B8
:1039600031084A0174C0C601EB81FC818E1B9F0B9C
:103970009C01220F331F280F391F280D391DB90153
:103980006F5B7C4EDA01AA0FBB1FA40FB51FA80DF9
:10399000B91D8D010F5B1C4EF80190819170FB01E8
:1039A00080818E7F892B8083A9014D5B5C4ECD0188
:1039B0008D5B9C4E9E838D83FC0190819F70FA01EC
:1039C0008081807F892B8083ED81FE81908190773B
:1039D0008F78892BFA018083ED81FE819081907828
:1039E0008F77892BFA018083F801808182958695F3
:1039F0008695837091819770990F990F982B492F15
:103A00004295440F440F407CFB0180818F73842BCF
:103A10008083969596958181887F892B81832E5B03
:103A20003C4EAE5BBC4E9C91987FD9018C918770C7
:103A3000892B8C93F80190819E73DB018C91817CA2
:103A4000892B8C93EB81FC813196FC83EB83A10164
:103A50002B813C81421B530B2C153D0509F083CF74
:103A600087E299E0489EA001499E500D589E500D56
:103A70001124DA01AF5BBC4E8C918E7F86298C932A
:103A8000CA018D5B9C4E37E0E322E29420EFE222F4
:103A9000779477247794EA81EE2AE728FC01E08284
:103AA0009F2D9295990F990F907C8C918F73892BF4
:103AB0008C934E5B5C4EAA0CAA0CAA0CF694F6945E
:103AC000FA28FA01F082FFE1BF22BB0C8C91817CC5
:103AD0008B298C9381E08093D30A02C1242E332456
:103AE000282F30E03C832B8384E890E0289FF0016E
:103AF000299FF00D389FF00D112487E299E0289E50
:103B0000B001299E700D389E700D1124E60FF71F2D
:103B1000EA58F44F208130E04B815C81440F551FFF
:103B20008B819C8106E0880F991F0A95E1F7480F69
:103B3000591FDA01A20FB31F1DE0E12EF12CEA0E8E
:103B4000FB1EEE0CFF1CE60EF71E8CED9AE0E80E55
:103B5000F91EF7018081F82FF170F983082F06957F
:103B60000170B82EB694B6941FE0B1228295869566
:103B700086958370F70111811770110F110F182BA3
:103B8000AA0FBB1FA60FB71FA950B54FAC90A694A4
:103B9000A694A694EE24FF24490124010894410828
:103BA00051083A016B015AC0A4014E195F09460D34
:103BB000571DDA011D96AA0FBB1FAC0DBD1DA452E7
:103BC000B54FB301680F791FFB013D96EE0FFF1F44
:103BD000EC0DFD1DE452F54F908191708C918E7F1C
:103BE000892B8C93908192708D7F892B8C939081FF
:103BF0009C73837C892B8C93208122952695269516
:103C0000237091819770990F990F922B292F2295EC
:103C1000220F220F207C8F73822B8C939695969582
:103C200011968C911197887F892B11968C93440F54
:103C3000551F4C0D5D1D4950554F660F771F6C0D7C
:103C40007D1D6950754FDB019C91987FFA01808141
:103C50008770892B80830894E11CF11CC2018E19A6
:103C60009F09E814F90409F09FCF84E890E02B81C4
:103C70003C81289FF001299FF00D389FF00D112401
:103C800087E299E0DC012A9EC0012B9E900D3A9EAE
:103C9000900D1124E80FF91F9F012A50354F017034
:103CA000000F0270BFE0BB22BB0CBB0C8981082B4C
:103CB000812F8295880F880F807C0B29082BD901D2
:103CC0000C93E950F54FAA0CAA0CAA0C1695169560
:103CD0001A291083EB81FC81EA52F14D81E0808347
:103CE0008091590990915A098930910511F00797EF
:103CF00019F481E08093460226960FB6F894DEBF51
:103D00000FBECDBFCF91DF911F910F91FF90EF902C
:103D1000DF90CF90BF90AF909F908F907F906F90EB
:103D20005F904F903F902F900895CF93DF93782F1F
:103D30006F5F2091D22E8031B9F530E087E299E0B3
:103D4000289FA001299F500D389F500D112429C094
:103D5000862F90E0FC01EE0FFF1FE80FF91FE40F24
:103D6000F51FDF01AF5BBC4E8C918E7F8C93CF0132
:103D70008D5B9C4E20E3EC0128838C91817C8861D3
:103D80008C93EE5BFC4E8081877080838C918F7367
:103D90008C9311968C911197887F846011968C93E7
:103DA0006F5F6034A8F28CC030E087E299E0289F12
:103DB000A001299F500D389F500D11247EC0262F41
:103DC00030E0872F90E0FC01B6E0EE0FFF1FBA95C0
:103DD000E1F7880F991FE80FF91FE20FF31F3D96D7
:103DE000EE0FFF1FE40FF51FE452F54F80818E7F29
:103DF0008083872F90E0FC01B6E0EE0FFF1FBA959D
:103E0000E1F7880F991FE80FF91FE20FF31F3D96A6
:103E1000EE0FFF1FE40FF51FE452F54F8081826023
:103E20008083872F90E0FC01B6E0EE0FFF1FBA956C
:103E3000E1F7880F991FE80FF91FE20FF31F3D9676
:103E4000EE0FFF1FE40FF51FE452F54F8081837CD6
:103E50008083872F90E0FC01B6E0EE0FFF1FBA953C
:103E6000E1F7880F991FE80FF91FE20FF31F3D9646
:103E7000EE0FFF1FE40FF51FE452F54F80818F73A3
:103E800080838181887F84608183872F90E0FC011B
:103E9000B6E0EE0FFF1FBA95E1F7880F991FE80F04
:103EA000F91FE20FF31FEE0FFF1FE40FF51FE9509C
:103EB000F54F8081877080836F5F603408F47FCF17
:103EC000DF91CF910895DF92EF92FF920F931F93AE
:103ED000CF93DF938091D22E90E027E239E0829F4A
:103EE000F001839FF00D929FF00D1124E452F54FE5
:103EF00010821182C0E0D0E034E8E32EF12C07E21A
:103F000019E0DD24D3944C2F8091D22E282F30E05D
:103F1000CE9DF001CF9DF00DDE9DF00D1124209F70
:103F2000C001219F900D309F900D1124E80FF91FC3
:103F3000EA58F44FE081DC01A452B54F8C918E1702
:103F400018F4EC93C093E72ECE9DF001CF9DF00DB9
:103F5000DE9DF00D1124209FC001219F900D309F08
:103F6000900D1124E80FF91FE958F44FE081DC01AE
:103F7000A452B54F11968C9111978E1710F411968B
:103F8000EC93FE01E253F64FD082CE9DF001CF9D1F
:103F9000F00DDE9DF00D1124209FC001219F900D9A
:103FA000309F900D1124E80FF91FEA58F44F842F29
:103FB00060810E94951E2196C031D10509F0A3CFE2
:103FC0008091D22E282F30E087E299E0289FF001DF
:103FD000299FF00D389FF00D1124E452F54FEF5951
:103FE000F74F9081E156F8408081891720F4908343
:103FF00080E18093E72E87E299E0289FF001299FD6
:10400000F00D389FF00D1124E452F54FE05AF74FB0
:104010009081E056F8408181891708F4918381E00E
:104020008093DE0987E299E0289FF001299FF00D37
:10403000389FF00D1124E35CFC4E80E160810E940A
:10404000951EDF91CF911F910F91FF90EF90DF9020
:1040500008958091D108882349F12091142F30913F
:10406000152F2F5F3F4F3093152F2093142F8091E2
:10407000182F9091192F8217930724F43093192F3A
:104080002093182F8091182F9091192F885E9340BC
:1040900034F087EE93E09093192F8093182F285EC9
:1040A000334024F01092152F1092142F0895809110
:1040B0004E09882319F0833050F523C060915309CD
:1040C0007091540980E090E00E94D17520E030E0CA
:1040D00040EC52E40E94877620E030E040E752E472
:1040E0000E943D759B01AC0160E074E284EF99E4AD
:1040F0000E943D750E94A5757093890060938800A9
:10410000089584EF91E0909389008093880008954A
:10411000E1E8F0E0108280818093800080818A60F5
:1041200080830E945720EFE6F0E0808182608083E8
:1041300008959F92AF92BF92CF92DF92EF92FF923B
:104140000F931F93DF93CF9300D000D0CDB7DEB78E
:104150008091590990915A0982309105D1F00C97BC
:10416000C1F08091433390E061E070E00E94A80BC1
:10417000982F843008F093E0909343338091EB3391
:10418000981739F09093EB3381E080934702809346
:10419000460280914933882309F4B6C00091CA09C8
:1041A0004091D22E0031A1F4842F90E027E239E033
:1041B000AC01429FC001439F900D529F900D11246E
:1041C000825C9C4E61E041E027E003ED1AE01FC0F5
:1041D00010E084E890E0BC01069FC001079F900DAD
:1041E000169F900D112450E027E239E0D9014A9F33
:1041F00090014B9F300D5A9F300D1124820F931F59
:104200000A52114D8758944F61E041E027E00E9427
:10421000040C8091C208882339F480915909909147
:104220005A09029709F070C05091CA094091D22EE4
:104230005031A1F4242F30E087E299E0289FF0016B
:10424000299FF00D389FF00D1124E452F54FEE59DF
:10425000F74F8081E256F84083831FC0242F30E05F
:1042600087E299E0289FD001299FB00D389FB00DBB
:104270001124252F30E084E890E0289FF001299F49
:10428000F00D389FF00D1124EA0FFB1FE758F44F93
:104290008081A452B54F13968C9320E030E004E85F
:1042A00010E067E279E0FF24F3948091D22E90E051
:1042B000209FF001219FF00D309FF00D1124AC01E3
:1042C000469FC001479F900D569F900D1124E80F07
:1042D000F91FE758F44FDC01A452B54FAD014D5F13
:1042E0005F4F13968C9113978083F901EA52F14D39
:1042F000F0822F5F3F4F20313105B9F6FD01EE59B5
:10430000F74FDA018C91808380914833882309F438
:10431000B8C00091CA094091D22E0031A1F4842F77
:1043200090E027E239E0FC01E29FC001E39F900D9D
:10433000F29F900D1124815C9C4E61E040E023E0EF
:1043400003ED1AE01FC010E084E890E09C01029F9A
:10435000C001039F900D129F900D112450E027E2A1
:1043600039E0B901469F9001479F300D569F300DAF
:104370001124820F931F0A52114D8858944F61E007
:1043800040E023E00E94040C8091C208882339F4A5
:104390008091590990915A09029709F072C02091B1
:1043A000CA094091D22E203169F450E087E299E0A9
:1043B000489FF001499FF00D589FF00D1124E15CDA
:1043C000FC4E19C050E030E084E890E0289FF001F6
:1043D000299FF00D389FF00D112487E299E0DC0150
:1043E0004A9FC0014B9F900D5A9F900D1124E80FDA
:1043F000F91FE858F44F208187E299E0489FF001C7
:10440000499FF00D589FF00D1124E452F54F22837F
:1044100020E030E004E810E067E279E0FF24F39464
:104420008091D22E90E0209FF001219FF00D309FCF
:10443000F00D1124AC01469FC001479F900D569F7F
:10444000900D1124E80FF91FE858F44FDC01A45235
:10445000B54FAD014E5F5F4F12968C9112978083DE
:10446000F901EA52F14DF0822F5F3F4F20313105C3
:10447000B9F6FD01ED59F74FDA018C918083F09286
:10448000D30A8091590990915A098630910509F40F
:104490005FC48730910584F482309105F9F0833050
:1044A00091052CF4019711F00C947A2D61C30597B6
:1044B00014F00C947A2DCAC08830910509F4D0C349
:1044C000883091050CF45AC58930910509F413C759
:1044D0000C9711F00C947A2D0C94642D8091D708D0
:1044E000882309F469C08091D22E90E077E2E72E0C
:1044F00079E0F72E8E9DF0018F9DF00D9E9DF00DC1
:104500001124E452F54FD080CF0161E040E02FE369
:1045100005ED1EE20E94040C8091D22E90E08E9D4B
:10452000F0018F9DF00D9E9DF00D1124E452F54F8A
:1045300080818D1591F120E030E064E870E047E281
:1045400059E011E08091D22E90E0269FF001279F44
:10455000F00D369FF00D1124DC01A49FC001A59F32
:10456000900DB49F900D1124E80FF91FEA58F44FF5
:10457000DC01A452B54F8C918083F901EA52F14DD0
:1045800010832F5F3F4F20313105E1F6FD01EF59D8
:10459000F74F8C9180831093D30A8091CA09082F1A
:1045A00010E00851114DF801F0808F2D90E061E08E
:1045B00070E00E94A80B89C0809153099091540922
:1045C00061E00E948A0C90935409809353098F31C3
:1045D000910530F48EE190E0909354098093530953
:1045E00080915309909154098A3F910530F08AEFE8
:1045F00090E090935409809353092091530930918E
:1046000054098091E8339091E9332817390749F02C
:104610003093E9332093E8330E94572081E0809360
:10462000460280914E09882311F00C947A2D8091D6
:104630001633882319F080E00E948D108091173383
:10464000882311F40C947A2D81E0DFC380914333E9
:104650008130F1F1813040F0823009F4CCC08330F8
:1046600011F00C947A2D5FC2809110098823D9F043
:104670008091C9088823B9F490E080910A2F88239B
:1046800009F491E090930A2F992351F0E091CA091F
:10469000F0E0DF01A750B14D8C91E851F14D8083DE
:1046A00081E08093460280910A2F882311F00C94B8
:1046B0007A2D8091CA09082F10E00851114DF80198
:1046C000F0808F2D61E00E94D90BD8018C93FAC63F
:1046D0000091CA094091D22E0031A1F4842F90E0BC
:1046E00027E239E0FC01E29FC001E39F900DF29FB9
:1046F000900D1124835C9C4E61E040E02FE303EDBC
:104700001AE01FC010E084E890E09C01029FC00105
:10471000039F900D129F900D112450E027E239E085
:10472000B901469F9001479F300D569F300D1124CF
:10473000820F931F0A52114D8A58944F61E040E056
:104740002FE30E94040C8091D22E90E027E239E002
:10475000829FF001839FF00D929FF00D1124E4528F
:10476000F54F108220E030E064E870E047E259E065
:104770008091D22E90E0269FF001279FF00D369F6A
:10478000F00D1124DC01A49FC001A59F900DB49FE2
:10479000900D1124E80FF91FEA58F44FE081DC0175
:1047A000A452B54F8C918E1718F4EC932093E72EFA
:1047B0002F5F3F4F20313105D9F68091D22E90E006
:1047C00027E239E0829FF001839FF00D929FF00D68
:1047D0001124E452F54FEF59F74F9081E156F8401C
:1047E0008081891710F00C947A2D908380E180935A
:1047F000E72E0C947A2D2091CA094091D22E2031B7
:1048000071F4242F30E087E299E0289FF001299F7E
:10481000F00D389FF00D1124E45CFC4E19C030E01F
:1048200050E084E890E0289FF001299FF00D389F28
:10483000F00D112487E299E09C01429FC001439F43
:10484000900D529F900D1124E80FF91FE958F44F75
:1048500010811831A9F0193128F41C30A9F0103159
:10486000B1F410C0103341F0103619F0103279F461
:1048700005C01092A3080BC081E007C082E005C00C
:1048800083E003C084E001C085E08093A3088091A9
:10489000A30861E00E94D90B982F863008F095E0BC
:1048A0009093A3088091E733981711F40C947A2D14
:1048B0009093E73381E080934602E091CA09E031AA
:1048C00019F48093D30A04C0F0E0EA52F14D8083DA
:1048D0008091A3088230A9F0833028F4882351F016
:1048E000813011F509C08430A1F0843060F085304A
:1048F000D9F415C010E601C010E3EE246FE1F62EE6
:1049000013C010E2FACF18E154E0E52E4BE1F42E8B
:104910000BC010E138E0E32E27E1F22E05C01CE0C9
:104920009AE0E92E85E1F82E8091CA096E2D4F2D6F
:104930000E94BA0D8091CA098031E1F5103321F04F
:10494000103611F0812F01C088E150E0A7E2B9E0F4
:10495000682F70E0482F41504F71440F17C0852FCA
:1049600090E0FC01EE0FFF1FE80FF91FE20FF31FAD
:10497000EF5BFC4E2081822F86958F7190E0861729
:1049800097071CF0217C242B20835F5F8091D22E1F
:1049900090E08A9F90018B9F300D9A9F300D1124DB
:1049A000F901E35CFC4E80818517C8F61092D00AAD
:1049B0001092CF0A2091CA094091D22E203171F471
:1049C000242F30E087E299E0289FF001299FF00D25
:1049D000389FF00D1124E45CFC4E19C030E050E02B
:1049E00084E890E0289FF001299FF00D389FF00D9A
:1049F000112487E299E0BC01469FC001479F900DBA
:104A0000569F900D1124E80FF91FE958F44F1083B9
:104A10008091F308882311F40C947A2D5091CA09DF
:104A20004091D22E5031A1F4242F30E087E299E05A
:104A3000289FF001299FF00D389FF00D1124E452BA
:104A4000F54FE05AF74F8081E056F84081831FC050
:104A5000242F30E087E299E0289FD001299FB00DF4
:104A6000389FB00D1124252F30E084E890E0289F76
:104A7000F001299FF00D389FF00D1124EA0FFB1F64
:104A8000E958F44F8081A452B54F11968C9300E001
:104A900010E024E8A22EB12C97E2C92E99E0D92E7D
:104AA000992493948091D22E90E00A9DD0010B9D81
:104AB000B00D1A9DB00D11248C9DF0018D9DF00D4F
:104AC0009C9DF00D1124AE0FBF1FA958B44FE452A6
:104AD000F54F81818C93802F6E2D4F2D0E94BA0D42
:104AE000F801EA52F14D90820F5F1F4F003111051E
:104AF000C9F680E16E2D4F2D0E94BA0D8091D22E05
:104B000090E027E239E0829FF001839FF00D929FB1
:104B1000F00D1124E452F54F8181E05AF74F808364
:104B20009092D30AE7C7809110098823D9F0809129
:104B3000D22E90E04091CA0927E239E0829FF0012D
:104B4000839FF00D929FF00D1124E452F54FE40F76
:104B5000F11D90E08781882309F491E0978381E03B
:104B6000809346028AEC99E061E040E020E126C0B3
:104B7000E091142FF091152FEE5EF04D918580910C
:104B8000CC09981741F081E0809341338091590915
:104B90008093423302C0109241338091433381307D
:104BA00091F0813030F0823051F1833009F0A2C7AA
:104BB00045C083E19FE261E040E02FE000E010E0CB
:104BC0000E94040C97C780910F09882349F0209117
:104BD000182F3091192F84E19FE26AE070E008C03D
:104BE0002091182F3091192F84E19FE261E070E04D
:104BF00040E050E000E010E00E94F70C7BC780919D
:104C0000142F9091152F855E904D61E040E02FE7C5
:104C100000E010E00E94040C80910F09882309F441
:104C200069C7E091142FF091152FEE5EF04D81854C
:104C30008093CD0981E08093D32E5CC780910F09CA
:104C4000882329F088E19FE26AE070E004C088E1EF
:104C50009FE261E070E041E050E027EE33E0CACF30
:104C600080914533813021F0823009F043C75FC025
:104C7000809143338130F9F0813038F0823009F48B
:104C800048C0833009F036C74AC080914E0961E0C0
:104C90000E94D90B982F833008F092E090934E0930
:104CA0008091E633981709F425C79093E63381E0A5
:104CB00080934F092BC0809155099091560961E06E
:104CC0000E948A0C9C018E31910518F42EE130E08F
:104CD00005C08B3F910510F02AEF30E03093560964
:104CE000209355098091E53390E02817390709F49E
:104CF00001C72093E5330E94572080915509909178
:104D00005609909354098093530981E08093580980
:104D1000EFC68CE599E061E042E02AE005C082E55B
:104D200099E061E040E023E008E519E049CF809197
:104D30004333882321F0813009F0DCC603C08DE5C0
:104D400099E002C08EE599E061E040E021E0ECCF1F
:104D500080914333813071F0813030F0823099F0AE
:104D6000833009F0C7C654C082E393E361E040E0BA
:104D700021E024CF8091323390E08C5F9C4C61E045
:104D800040E024E030C080911009882389F08091B0
:104D90003233E82FF0E0EC5FFC4C90E0828988230E
:104DA00009F491E0928B81E0809333338093460243
:104DB00080913233282F30E0F901EC5FFC4C82897E
:104DC0008823A1F48091C208F9013296882329F042
:104DD000CF018C5F9C4C6AE004C0CF018C5F9C4C7F
:104DE00061E040E02EEF03E313E3EACE813009F007
:104DF00081C6C901885E9C4C61E040E025E003E388
:104E000013E30E94040C809132330E948D1072C60D
:104E10008091C20800913233882389F010E0000F9E
:104E2000111F000F111F085F1C4CD8016D917D915F
:104E30008D919C912DEC3CEC4CEC5DE310C010E0AE
:104E4000000F111F000F111F085F1C4CD8016D913E
:104E50007D918D919C912AE037ED43E25CE30E94C5
:104E6000350DF8016083718382839383809132339F
:104E7000C82EDD24F601EE0FFF1FEE0FFF1FE85FC7
:104E8000FC4CE080F18002811381C801B70120E071
:104E900030E040E050E00E94397588235CF40F2E2A
:104EA000F0E0EF2EF0E0FF2EF0E00F2FF0E01F2FEC
:104EB000F02D14C0C801B70120E030E040E85FE306
:104EC0000E948376181654F40F2EF0E0EF2EF0E0D7
:104ED000FF2EF0E80F2FFFE31F2FF02DCC0CDD1C71
:104EE000CC0CDD1C28E033E3C20ED31ED601ED92BC
:104EF000FD920D931C931397E0913233F0E0EE0F87
:104F0000FF1FEE0FFF1FE20FF31FE080F180028111
:104F10001381C801B7012091E1333091E233409110
:104F2000E3335091E4330E943975882369F0E092AD
:104F3000E133F092E2330093E3331093E43381E002
:104F4000809333338093460280911009882309F4BB
:104F5000D1C5E0913233F0E0EE0FFF1FEE0FFF1FDF
:104F6000E85FFC4C80E090E0A0E8BFE380839183A1
:104F7000A283B38381E080933333BAC52091D22ECC
:104F800030E08091620990E0DC01AA0FBB1FA80FFE
:104F9000B91F87E2E82E89E0F82EF901EE9D900115
:104FA000EF9D300DFE9D300D1124A20FB31FFD01AA
:104FB000ED5BFC4E8081082F0F708295877089838E
:104FC000255C3C4EF9011081AF5BBC4E8C918695FF
:104FD0008F71909143339130A1F1913038F092303C
:104FE00009F401C1933009F085C566C18091D50AE5
:104FF000882309F454C2813009F07CC5812F61E017
:105000000E94D90B482F893008F048E08091DF33A7
:10501000481739F04093DF3381E08093D30A8093BF
:1050200046028091D22E90E027E239E0829FF00183
:10503000839FF00D929FF00D1124E55CFC4E4083A0
:1050400059C50E94960D402F480FA02FB0E0642F45
:1050500070E0CD01861B970B8130910551F5212F12
:1050600030E0F901EE0FFF1FE20FF31FEE0FFF1FFD
:10507000EE0FFF1FAE0FBF1FA854BE4F9C91E60F4F
:10508000F71FE854FE4F8081981709F44150F90149
:10509000EE0FFF1FE20FF31FEE0FFF1FEE0FFF1FBC
:1050A000E40FF11DE854FE4F8081981771F54150CF
:1050B0002CC08F5F9F4F49F5212F30E0F901EE0F93
:1050C000FF1FE20FF31FEE0FFF1FEE0FFF1FAE0FCC
:1050D000BF1FA854BE4F9C91E60FF71FE854FE4F28
:1050E0008081981709F44F5FF901EE0FFF1FE20F5F
:1050F000F31FEE0FFF1FEE0FFF1FE40FF11DE8542B
:10510000FE4F8081981709F44F5F4F3F41F489812A
:10511000815089838F3F09F419824BE00AC04C30DB
:1051200040F089818F5F8983873010F087E0898321
:1051300040E04C3008F04BE08091E033481739F004
:105140004093E03381E08093D30A809346024093FA
:10515000050A8091F408882321F120E030E067E21D
:1051600079E08091D22E90E0F901EE0FFF1FE20F5F
:10517000F31FDC01A69FC001A79F900DB69F900D65
:105180001124E80FF91FED5BFC4E9091050A9F700A
:105190008081807F892B80832F5F3F4F20343105B2
:1051A00001F78091620990E02091D22E30E0FC015D
:1051B000EE0FFF1FE80FF91F87E299E0BC01269F61
:1051C000C001279F900D369F900D1124E80FF91F05
:1051D000ED5BFC4E4F70808180789981977092953D
:1051E000907F842B6EC48091F4088823B1F10E94D3
:1051F000960D8093060A8823C9F140E050E067E2EB
:1052000079E08091D22E90E0FA01EE0FFF1FE40FBB
:10521000F51FDC01A69FC001A79F900DB69F900DC2
:105220001124E80FF91FED5BFC4E2081822F82953F
:105230008F709091060A890F87708295807F2F78F2
:10524000282B20834F5F5F4F40345105D1F681E01A
:105250008093D30A8093460209C0CE01019661E093
:1052600040E027E003ED1AE00E94040C8091100951
:10527000882311F083E089838091620990E0209176
:10528000D22E30E0FC01EE0FFF1FE80FF91F87E27E
:1052900099E0AC01249FC001259F900D349F900D93
:1052A0001124E80FF91FED5BFC4E998197709295E0
:1052B000907F80818F7805C40E94310C2091620913
:1052C00030E04091D22E50E0F901EE0FFF1FE20FC7
:1052D000F31F4E9D90014F9D300D5E9D300D1124AA
:1052E000E20FF31FEF5BFC4E8F71880F9081917C72
:1052F000982B9083FFC31C82B091CA094091D22E93
:1053000060916209B031A9F5862F90E0242F30E03A
:105310008C01000F111F080F191F87E299E0B901D6
:10532000689F9001699F300D789F300D1124020F06
:10533000131FD801AF5BBC4E4C91942F929596955C
:105340009695937011968C918770880F880F892B92
:105350008983245C3C4EF901A0810E5B1C4EF80150
:1053600080818695869586958A83842F86958F7110
:105370006DC070E08B2F90E0FC01A6E0EE0FFF1FE8
:10538000AA95E1F7880F991FE80FF91FE60FF71F9D
:105390003D96242F30E0EE0FFF1F87E299E0289F13
:1053A000A001299F500D389F500D1124E40FF51FC7
:1053B000E452F54F908192959695969593708181E0
:1053C0008770880F880F892B89832B2F30E084E822
:1053D00090E0289FF001299FF00D389FF00D1124D7
:1053E000E40FF51FE958F44FA081F90196E0EE0FA4
:1053F000FF1F9A95E1F7220F331FE20FF31FE60F0D
:10540000F71F3D96EE0FFF1FE40FF51FE452F54F17
:105410008081869586958F708A838B2F90E0FC0122
:1054200016E0EE0FFF1F1A95E1F7880F991FE80F9E
:10543000F91FE60FF71FEE0FFF1FE40FF51FE950EE
:10544000F54F80818695869586958B839091433321
:10545000913009F44CC0913038F0923009F478C1A1
:10546000933009F047C362C2809110098823B9F0D4
:1054700090E080910A2F882309F491E090930A2FFD
:10548000992351F0E091CA09F0E0DF01A750B14D36
:105490008C91E851F14D808381E0809346028091A8
:1054A0000A2F882309F026C38091CA09082F10E02B
:1054B0000851114DD801FC908F2D61E00E94D90B4D
:1054C000F80180838091CA09E82FF0E0E851F14D9E
:1054D0008081843008F083E08083E091CA09F0E0A5
:1054E000E851F14D8081F81609F001C303C3A831DA
:1054F00099F0A93128F4AC30D9F0A03119F512C0D7
:10550000A03321F0A03611F0A032E1F4CE010196D3
:1055100061E040E02FE111C0CE01019661E044E07E
:105520002BE10BC0CE01019661E048E027E105C008
:10553000CE01019661E04AE025E18E010C5F1F4F2C
:105540000E94040C80911009882331F080E1898346
:1055500081E08C83809346028C81882309F46BC0A0
:105560007091CA094091D22E6091620959817031BF
:1055700059F5862F90E0242F30E0FC01EE0FFF1F3D
:10558000E80FF91F87E299E0BC01269FC001279F21
:10559000900D369F900D1124E80FF91FEF5BFC4E24
:1055A000952F9295990F990F907C80818F73892BFD
:1055B00080835695569557708181887F852B81838E
:1055C00081E08093D30A37C0872F90E0FC0136E05A
:1055D000EE0FFF1F3A95E1F7880F991FE80FF91FAB
:1055E000E60FF11D3D96242F30E0EE0FFF1F87E2FE
:1055F00099E0DC012A9FC0012B9F900D3A9F900DEE
:105600001124E80FF91FE452F54F952F9295990F49
:10561000990F907C80818F73892B80835695569546
:1056200057708181887F852B8183E72FF0E0EA52D4
:10563000F14D81E080838091F408882309F45AC2F7
:105640008091D22E90E027E239E0829FF001839F83
:10565000F00D929FF00D1124E452F54F898185835E
:105660008091CA09803199F520E030E047E259E0A5
:105670008091D22E90E0F901EE0FFF1FE20FF31F91
:10568000849FD001859FB00D949FB00D1124EA0F27
:10569000FB1FEF5BFC4EA452B54F15969C911597DE
:1056A0009295990F990F907C80818F73892B8083BD
:1056B00015969C919695969597708181887F892BF8
:1056C00081832F5F3F4F2034310591F6F0C040E0D9
:1056D00050E007E219E02091D22E30E06091CA0933
:1056E000862F90E0FC01B6E0EE0FFF1FBA95E1F7C0
:1056F000880F991FE80FF91FE40FF51F3D96EE0F75
:10570000FF1F209FD001219FB00D309FB00D1124AD
:10571000EA0FFB1FE452F54FA452B54F15969C912A
:1057200015979295990F990F907C80818F73892B93
:10573000808315969C919695969597708181887F28
:10574000892B81834F5F5F4F4034510521F6E8C0BC
:10575000CE01029661E040E02FE08E010C5F1F4F0A
:105760000E94040C80911009882329F01A8281E09C
:105770008C83809346028C81882309F459C07091F0
:10578000CA094091D22E609162095A81703111F597
:10579000862F90E0242F30E0FC01EE0FFF1FE80F72
:1057A000F91F87E299E0BC01269FC001279F900D59
:1057B000369F900D1124E80FF91FEE5BFC4E550F3C
:1057C000550F550F80818770852B808381E08093F2
:1057D000D30A2EC0872F90E0FC0136E0EE0FFF1FAA
:1057E0003A95E1F7880F991FE80FF91FE60FF11DB1
:1057F0003D96242F30E0EE0FFF1F87E299E0DC0199
:105800002A9FC0012B9F900D3A9F900D1124E80F05
:10581000F91FE452F54F5F70550F550F8081837C5F
:10582000852B8083E72FF0E0EA52F14D81E0808301
:105830008091F408882309F45DC18091D22E90E014
:1058400027E239E0829FF001839FF00D929FF00DD7
:105850001124E452F54F8A8184838091CA098031F2
:1058600051F520E030E047E259E08091D22E90E0FF
:10587000D901AA0FBB1FA20FB31F849FF001859F00
:10588000F00D949FF00D1124AE0FBF1FAE5BBC4E08
:10589000E452F54F9481990F990F990F8C9187706D
:1058A000892B8C932F5F3F4F20343105F1F681E037
:1058B0008093D30A1FC140E050E007E219E0209135
:1058C000D22E30E06091CA09862F90E0FC01A6E05C
:1058D000EE0FFF1FAA95E1F7880F991FE80FF91F38
:1058E000E40FF51F3D96EE0FFF1F209FD001219F73
:1058F000B00D309FB00D1124EA0FFB1FE452F54F9D
:10590000A452B54F14969C919F70990F990F808166
:10591000837C892B80834F5F5F4F4034510579F63C
:10592000E62FF0E0EA52F14D81E0CCC00091CA09C7
:10593000003161F50E94310C482F809110098823B5
:1059400031F081E08093D30A809346024CE080914D
:10595000620990E02091D22E30E0FC01EE0FFF1F93
:10596000E80FF91F87E299E0BC01269FC001279F3D
:10597000900D369F900D1124E80FF91FEF5BFC4E40
:105980004F71440F8081817C842B9CC0E6E7F1E05D
:105990002CE08081A81721F0215031972223C9F7EC
:1059A000215010E00A52114DCE01039661E040E013
:1059B0000E94040C80911009882351F01B82E09111
:1059C000CA09F0E0EA52F14D81E0808380934602FB
:1059D0008091F408882309F44AC08091D22E90E087
:1059E00027E239E0829FF001839FF00D929FF00D36
:1059F0001124E452F54F8B81868340E050E007E2AA
:105A000019E02091D22E30E06091CA09862F90E0F3
:105A1000FC01B6E0EE0FFF1FBA95E1F7880F991F62
:105A2000E80FF91FE40FF51FEE0FFF1F209FD001B5
:105A3000219FB00D309FB00D1124EA0FFB1FE950DC
:105A4000F54FA452B54F16969C91990F990F990F47
:105A500080818770892B80834F5F5F4F4034510571
:105A600081F6E62FF0E0EA52F14D81E0808320914B
:105A700062098091CA0990E0FC0166E0EE0FFF1F09
:105A80006A95E1F7880F991FE80FF91FE20FF11DE2
:105A90008091D22E90E0EE0FFF1F27E239E0DC016B
:105AA000A29FC001A39F900DB29F900D1124E80FFB
:105AB000F91FE950F54F9B81990F990F990F80813C
:105AC0008770892B808316C08091B63390E061E0A7
:105AD00070E00E94A80B982F873008F096E0909312
:105AE000B6338091EA33981729F09093EA3381E036
:105AF000809346020F900F900F900F90CF91DF91FF
:105B00001F910F91FF90EF90DF90CF90BF90AF90DB
:105B10009F900895CF92EF920F938130910509F0F5
:105B20004CC06F5F7F4F09F071C080E580933433C4
:105B3000109235338AE493E360E071E00E94887349
:105B400081E593E360E071E00E94887388E593E368
:105B500060E071E00E9488738FE593E360E071E09C
:105B60000E94887386E693E360E071E00E94887388
:105B70008DE693E360E071E00E94887384E793E32D
:105B800060E071E00E9488738BE793E360E071E06E
:105B90000E94887382E893E360E071E00E9488735A
:105BA00089EB93E362E143E124E105E1F6E1EF2EC5
:105BB000E7E1CE2E0E94B96729C0892B39F56F5FC6
:105BC0007F4F21F582E893E30E94C8748BE793E34B
:105BD0000E94C87484E793E30E94C8748DE693E33F
:105BE0000E94C87486E693E30E94C8748FE593E32D
:105BF0000E94C87488E593E30E94C87481E593E32A
:105C00000E94C8748AE493E30E94C8740F91EF90D5
:105C1000CF90089580E090E06FEF7FEF0E948A2D93
:105C2000089581E090E06FEF7FEF0E948A2D089544
:105C30000E94AC6B20912D0730912E0740912F07C9
:105C400050913007621B730B840B950B6630710506
:105C50008105910508F470C00E94AC6B60932D071C
:105C600070932E0780932F07909330074091343321
:105C7000309135332091F533222381F0213051F4D6
:105C80008DB38093F7339DB38091F633809589234C
:105C90008DBB04C08FB7F8948093F7334CBD3DBDE6
:105CA0005E9A1EBC00000DB407FEFDCF8EB580933A
:105CB00023071EBC00000DB407FEFDCF8EB58093F8
:105CC00025071EBC00000DB407FEFDCF8EB58093E6
:105CD00027071EBC00000DB407FEFDCF8EB58093D4
:105CE00029071EBC00000DB407FEFDCF8EB58093C2
:105CF0002B075E98222339F08091F733213011F47D
:105D00008DBB01C08FBF93B1907290933933E3E2A2
:105D1000F7E0A8E1B7E020818181281709F42C93EE
:105D20003296119687E0ED32F807A9F780913A3361
:105D3000981711F490933B334091343330913533BD
:105D40002091F533222381F0213051F48DB38093DB
:105D5000F7339DB38091F633809589238DBB04C0C2
:105D60008FB7F8948093F7334CBD3DBD5E9A1EBC4F
:105D700000000DB407FEFDCF8EB5809324071EBC36
:105D800000000DB407FEFDCF8EB5809326071EBC24
:105D900000000DB407FEFDCF8EB5809328071EBC12
:105DA00000000DB407FEFDCF8EB580932A071EBC00
:105DB00000000DB407FEFDCF8EB580932C075E98D2
:105DC000222339F08091F733213011F48DBB01C0CB
:105DD0008FBF83B1807280933A330895DF92EF9240
:105DE000FF920F931F93CF93DF930E94182EE090A2
:105DF0001A07D0901C0700911B0710E0B8016470CF
:105E0000707080EC98E00E94B605B8016870707000
:105E100087EC98E00E94B605B801617070708BE164
:105E200099E00E94B605FF24B7016270707084E1AA
:105E300099E00E94B6050270107084EA98E0B801FB
:105E40000E94B605B701647070708FEF98E00E94F1
:105E5000B605B7016870707086E099E00E94B605DB
:105E6000B701607870708BEA98E00E94B605CD2D7E
:105E7000D0E0BE016170707081E898E00E94B605C4
:105E8000BE016270707088E898E00E94B605B701A4
:105E90006072707085ED98E00E94B605B70160747D
:105EA000707089EB98E00E94B605B7016071707060
:105EB0008AEE98E00E94B60521E0E222FF2481EFFD
:105EC00098E0B7010E94B605BE01607270708FE85D
:105ED00098E00E94B605BE01607170708DE099E097
:105EE0000E94B6057091190760E08091180790E054
:105EF000682B792B88EF98E00E94B6051092D208A3
:105F00001092D108D695C795D695C795CE018170C8
:105F1000682F8093CE088091CF08681711F1809187
:105F2000D008882371F4613061F46093D1080E9435
:105F3000AC6B60932209709323098093240990939A
:105F400025099091D008913041F48091CE088823A2
:105F500021F49093D2081092D3088091CE088093B8
:105F6000D0088091CE088093CF088091D0088823F4
:105F7000B1F00E94AC6B209122093091230940912D
:105F8000240950912509621B730B840B950B695EE4
:105F900073408040904018F081E08093D308E4E3A0
:105FA000F7E010821182379687E0E43AF807C9F7E4
:105FB000DF91CF911F910F91FF90EF90DF900895A7
:105FC0001F93CF93DF9310E0C0E0D0E082EA96E326
:105FD000BE0140E00E94586B219682EA96E3BE0122
:105FE00043E60E94586B219682EA96E3BE0144E69E
:105FF0000E94586B219682EA96E3BE0141E00E941E
:10600000586B219682EA96E3BE0143E00E94586BEA
:106010002196CA30D105D1F61F5F1038A9F6DF915D
:10602000CF911F9108952F923F924F925F926F925E
:106030007F928F929F92AF92BF92CF92DF92EF9218
:10604000FF920F931F93CF93DF93C4E0D3E394E0C9
:10605000A92EB12CAC0EBD1EEE24FF24C82EDD24CB
:1060600016010894211C311C02E0402E512C4C0CCE
:106070005D1C13E0612E712C6C0C7D1CB4E08B2E2A
:10608000912C8C0C9D1CB7016C0D7D1D82EA96E352
:1060900048810E94586BB1016E0D7F1D82EA96E324
:1060A0004A810E94586B82010E0D1F1DF5016191FE
:1060B0007191819191915F0120E030E048EC52E4D0
:1060C0000E9487760E94A5759B01AC0182EA96E347
:1060D000B801422F0E94586BB3016E0D7F1D82EAFA
:1060E00096E34A890E94586BB4016E0D7F1D82EAC7
:1060F00096E34C890E94586B219685E090E0E80E6B
:10610000F91E93E3C630D90709F0BDCFDF91CF91D7
:106110001F910F91FF90EF90DF90CF90BF90AF90C5
:106120009F908F907F906F905F904F903F902F90B7
:10613000089582EA96E360EA7FE040E00E94586BAF
:10614000089582EA96E360EA7FE040918D330E94F1
:10615000586B08954F925F926F927F928F929F92A9
:10616000AF92BF92CF92DF92EF92FF920F931F9365
:10617000CF93DF93C4E0D3E354E0C52ED12CCC0EF3
:10618000DD1E00E010E0E82EFF2427010894411CEA
:10619000511C42E0642E712C6E0C7F1C33E0832E68
:1061A000912C8E0C9F1C24E0A22EB12CAE0CBF1C97
:1061B000B8016E0D7F1D82EA96E30E94516B853017
:1061C00008F084E08883B201600F711F82EA96E3D1
:1061D0000E94516B8F3F09F48EEF8A83B301600FE9
:1061E000711F82EA96E30E94516B853608F084E6BF
:1061F000682F70E0882777FD8095982F0E94D375CF
:1062000020E030E048EC52E40E943D75F6016083E6
:10621000718382839383B401600F711F82EA96E3D6
:106220000E94516B811181E08A8BB501600F711F53
:1062300082EA96E30E94516B843008F083E08C8BF5
:106240001C861E86188A0B5F1F4F219684E090E003
:10625000C80ED91E0A30110509F0AACFDF91CF91DF
:106260001F910F91FF90EF90DF90CF90BF90AF9074
:106270009F908F907F906F905F904F9008951092B5
:10628000323310921A3380E00E94AA30089582EAD5
:1062900096E360EA7FE00E94516B80938D3308950E
:1062A000AF92BF92CF92DF92EF92FF920F931F9324
:1062B000909110339F5F90931033809111338F5FD3
:1062C0008093113380911A33882349F080E098E05D
:1062D0000E94F40A80E098E00E94290B2DC1892FCA
:1062E00090E04091063320E031E0241B3109821711
:1062F00093070CF48AC010921033909104339430B9
:10630000D9F580911233882309F074C060E070E001
:1063100080E090E020E031E040E050E00E94157223
:10632000E0900833F090093300910A3310910B3359
:106330000E94D375A80197010E9487765B016C01CA
:10634000C801B70120E030E040E053EC0E948776BE
:1063500020E030E040E053E40E94D5749B01AC01A2
:10636000C601B5010E94D5740E94A57514E0660FA0
:10637000771F1A95E1F73AC0A0900833B09009331F
:10638000C0900A33D0900B3380911233F92FE0E0A4
:10639000E80FF11DEB52FD4F608170E0882777FD1B
:1063A0008095982F0E94D375A60195010E9487764B
:1063B0007B018C01C601B50120E030E040E053ECE8
:1063C0000E94877620E030E040E053E40E94D574DC
:1063D0009B01AC01C801B7010E94D57420E030E0F8
:1063E00040E851E40E9487760E94A5757093D233ED
:1063F0006093D1338091D1339091D2330E94F40ACB
:10640000809112338F5F809312338091113390E02B
:106410004091073320E031E0241B310982179307B4
:106420000CF48AC010921133909105339430D9F551
:1064300080911333882309F074C060E070E080E03D
:1064400090E020E031E040E050E00E941572E090E2
:106450000C33F0900D3300910E3310910F330E94E6
:10646000D375A80197010E9487765B016C01C80172
:10647000B70120E030E040E053EC0E94877620E056
:1064800030E040E053E40E94D5749B01AC01C601AA
:10649000B5010E94D5740E94A575B4E0660F771F00
:1064A000BA95E1F73AC0A0900C33B0900D33C0908C
:1064B0000E33D0900F3380911333F92FE0E0E80FC3
:1064C000F11DEB52FD4F608170E0882777FD8095CC
:1064D000982F0E94D375A60195010E9487767B01B3
:1064E0008C01C601B50120E030E040E053EC0E9491
:1064F000877620E030E040E053E40E94D5749B01B1
:10650000AC01C801B7010E94D57420E030E040E83A
:1065100051E40E9487760E94A5757093D0336093F2
:10652000CF338091CF339091D0330E94290B80914B
:1065300013338F5F8093133380916009882361F157
:106540009091610980914E09813069F4E0915C0974
:10655000F0E0EE0FFF1FEE5AFE4F0190F081E02DAC
:10656000F695E7950AC0E0915C09F0E0EE0FFF1F99
:10657000EE5AFE4F0190F081E02D9F5F90936109EC
:106580009150892F90E08E179F0730F00E948D0A5E
:10659000109261091092600980914B098F5F80937E
:1065A0004B091F910F91FF90EF90DF90CF90BF901C
:1065B000AF9008951F920F920FB60F920BB60F92E5
:1065C00011242F933F934F935F936F937F938F93F8
:1065D0009F93AF93BF93EF93FF930E945031FF912E
:1065E000EF91BF91AF919F918F917F916F915F914B
:1065F0004F913F912F910F900BBE0F900FBE0F90B8
:106600001F901895FF920F931F93F82E09EB13E339
:10661000C8016F2D41E00E94CE66C80161E873E0B9
:106620000E944C70C8016F2D41E00E94CE661F9100
:106630000F91FF9008950F931F9309EB13E3C80187
:1066400064E040E00E94CE66C8016FED73E00E94F6
:106650004C7081E0809340331F910F91089589EB36
:1066600093E36CEE73E00E944C7008950F931F93B8
:1066700009EB13E3C80160E040E00E94CE66C80168
:1066800067E973E00E944C70C80160E041E00E943D
:10669000CE660E942F33C80160E041E00E94CE66C2
:1066A000C80166E873E00E944C701F910F91089535
:1066B0000F931F9309EB13E3C80160E040E00E94D1
:1066C000CE66C80169EB73E00E944C70C80160E0BF
:1066D00041E00E94CE660E942F33C80160E041E095
:1066E0000E94CE66C80168EA73E00E944C701F9158
:1066F0000F9108950F931F93CF93DF93C0E0D0E0E5
:10670000082F10E006C089EB93E361EA0E946F70E6
:106710002196C017D107BCF3DF91CF911F910F9144
:10672000089588E00E940233E0913233F0E0EC5F9C
:10673000FC4C8489823019F1833038F4882309F4C1
:1067400040C0813009F047C031C0843031F084301E
:1067500020F1853009F03FC009C089EB93E360E088
:106760000E949C6689EB93E361E011C089EB93E39F
:1067700060E00E949C6689EB93E361E01FC089EBB7
:1067800093E360E00E949C6689EB93E363E00E94E0
:106790009C6689EB93E362E011C089EB93E360E0D0
:1067A0000E949C6689EB93E363E008C089EB93E366
:1067B00060E00E949C6689EB93E366E00E949C6621
:1067C000089589EB93E360E00E949C6689EB93E374
:1067D00067E00E949C6608951F93882319F08FEF4D
:1067E0008093D3332091CA094091D22E203171F485
:1067F000242F30E087E299E0289FF001299FF00DD7
:10680000389FF00D1124E45CFC4E19C030E050E0DC
:1068100084E890E0289FF001299FF00D389FF00D4B
:10682000112487E299E09C01429FC001439F900D93
:10683000529F900D1124E80FF91FE958F44F108171
:106840008091D333181709F452C088E00E940233B4
:10685000183109F1193130F41C3059F0103109F0B8
:1068600044C010C0103371F11036A9F11032E9F5AF
:106870001BC089EB93E360E00E949C6689EB93E385
:1068800064E031C089EB93E360E00E949C6689EB91
:1068900093E361E011C089EB93E360E00E949C66A2
:1068A00089EB93E361E01FC089EB93E360E00E9412
:1068B0009C6689EB93E363E00E949C6689EB93E31B
:1068C00062E011C089EB93E360E00E949C6689EB73
:1068D00093E363E008C089EB93E360E00E949C6669
:1068E00089EB93E366E00E949C661093D3331F917B
:1068F0000895CF92DF92EF92FF920F931F93CF9361
:10690000DF93EC018B017A0169016AE473E30E9471
:10691000A272882321F589EB93E360E041E00E94B5
:10692000CE6689EB93E36CE074E00E944C708C813E
:106930009D81029720F489EB93E361E003C089EB2A
:1069400093E360E041E00E94CE6689EB93E3BE01F1
:106950000E9477718AE493E3BE010E949B74C80190
:1069600061E573E30E94A2728823E1F489EB93E36B
:1069700064E041E00E94CE6689EB93E367E074E057
:106980000E944C7089EB93E364E041E00E94CE6684
:1069900089EB93E3B8010E94777181E593E3B80135
:1069A0000E949B74C70168E573E30E94A27288236A
:1069B00061F5C70160E070E00E944C72882329F500
:1069C00089EB93E368E041E00E94CE6689EB93E3B4
:1069D00062E074E00E944C70F70184819581029717
:1069E00020F489EB93E369E003C089EB93E368E06B
:1069F00041E00E94CE6689EB93E3B7010E94777174
:106A000088E593E3B7010E949B74C6016FE573E3C9
:106A10000E94A272882329F589EB93E36CE041E0A0
:106A20000E94CE6689EB93E36DEF73E00E944C7099
:106A3000F60184819581029720F489EB93E36DE060
:106A400003C089EB93E36CE041E00E94CE6689EBE2
:106A500093E3B6010E9477718FE593E3B6010E943C
:106A60009B74DF91CF911F910F91FF90EF90DF907A
:106A7000CF9008959F92AF92BF92CF92DF92EF9204
:106A8000FF920F931F93DF93CF93CDB7DEB7C05420
:106A9000D2400FB6F894DEBF0FBECDBF8091413318
:106AA0008823A1F089EB93E36091443341E00E9495
:106AB000CE66809144018823F1F489EB93E363E08F
:106AC00071E00E9474711092D6331EC08091D6334B
:106AD0008823D1F48091423390E02091590930917C
:106AE0005A098217930781F489EB93E36091443349
:106AF00041E00E94CE6689EB93E362E873E30E9473
:106B0000777181E08093D6338091423390E0209179
:106B1000590930915A098217930711F010924133A5
:106B200080914602882311F40C94924410924602FC
:106B300080914933882309F471C089EB93E360E0C5
:106B400040E00E94CE6689EB93E365E375E00E9426
:106B50004C7089EB93E360E041E00E94CE660E94B6
:106B60002F3389EB93E362E041E00E94CE6689EB2C
:106B700093E363E375E00E944C7089EB93E365E077
:106B800041E00E94CE6687E00E947A3389EB93E36E
:106B90006EE041E00E94CE6689EB93E361E375E02D
:106BA0000E944C702091CA094091D22E203171F47C
:106BB000242F30E087E299E0289FF001299FF00D13
:106BC000389FF00D1124E25CFC4E19C030E050E01B
:106BD00084E890E0289FF001299FF00D389FF00D88
:106BE000112487E299E09C01429FC001439F900DD0
:106BF000529F900D1124E80FF91FE758F44F608160
:106C00006C5F89EB93E341E00E94CE6689EB93E3EE
:106C10006BED0E946F708BE090E078C080914833FC
:106C2000882309F479C089EB93E360E040E00E9497
:106C3000CE668091590990915A09029729F489EBFF
:106C400093E360E275E004C089EB93E36FE075E0E5
:106C50000E944C7089EB93E360E041E00E94CE66B5
:106C60000E942F3389EB93E363E041E00E94CE66FC
:106C70002091CA094091D22EDE01A25DBD4F203184
:106C8000B9F4242F30E087E299E0289FF001299F92
:106C9000F00D389FF00D1124E15CFC4E8081E82F4F
:106CA000F0E0EE0FFF1FE752FD4F6591749122C097
:106CB00030E050E084E890E0289FF001299FF00D3B
:106CC000389FF00D112487E299E09C01429FC0019A
:106CD000439F900D529F900D1124E80FF91FE85823
:106CE000F44F8081E82FF0E0EE0FFF1FE752FD4FD9
:106CF00065917491CD010E944F0589EB93E3BE012C
:106D0000625D7D4F0E9474718AE090E09093C809A3
:106D10008093C7090C9492448091590990915A0923
:106D20008530910511F40C94BF428630910594F49E
:106D30008230910509F4B1C1833091050CF0BCC2D9
:106D4000009711F40C942944019711F00C9492448B
:106D50000C94024388309105B1F0893091054CF4D0
:106D60008630910509F49EC7079711F00C94924460
:106D700055C58930910511F40C94943F0C9711F08E
:106D80000C949244BDC48091C7099091C80908979A
:106D9000A9F08FE593E368E071E00E94BC73BC0149
:106DA00088E593E30E949B74BC0181E593E30E9414
:106DB0009B74BC018AE493E30E949B7480914533E9
:106DC000813029F0823011F00C949244BAC0809145
:106DD000C7099091C809089761F4809177018130C3
:106DE00041F480914702882321F480914033882325
:106DF000D1F188E090E09093C8098093C709809111
:106E0000453380937701109247021092403389EB0B
:106E100093E360E040E00E94CE6689EB93E36EEF7F
:106E200074E00E944C7080914333E82FF0E0EE0F45
:106E3000FF1FE757FD4F659174918E010F5F1F4F44
:106E4000C8010E944F05E0914333F0E0E85BFD4F3D
:106E500089EB93E3608140E00E94CE6689EB93E387
:106E6000B8010E94747180914E09E82FF0E0EE0F96
:106E7000FF1FED5CFC4F659174917E010894E11C4D
:106E8000F11CC7010E944F0586E693E3B7010E94FB
:106E9000BC738E010B5F1F4F6091550970915609AD
:106EA000C8014AE00E94D5738DE693E3B8010E94C1
:106EB0009B74C8010E94C8748E01045F1F4FC801F3
:106EC00060915C094AE00E94377484E793E3B8015B
:106ED0000E949B74C8010E94C87480915209E82FD7
:106EE000F0E0EE0FFF1FEB5DFC4F65917491C70161
:106EF0000E944F058BE793E3B7010E94BC7373E1D7
:106F0000A72EB12CAC0EBD1EC50166E673E30E9430
:106F1000B2746AE1C62ED12CCC0EDD1EC6016DE620
:106F200073E30E94B27451E2E52EF12CEC0EFD1ECB
:106F3000C70164E773E30E94B2748E01085D1F4FBE
:106F400093C080917701823041F480914702882379
:106F500021F480914033882399F182E08093770176
:106F6000109247021092403389EB93E360E040E0D7
:106F70000E94CE6689EB93E36DEE74E00E944C7044
:106F800080914333E82FF0E0EE0FFF1FEF56FD4FE7
:106F9000659174918E010F5F1F4FC8010E944F05CC
:106FA000E0914333F0E0E85BFD4F89EB93E36081D0
:106FB00040E00E94CE6689EB93E3B8010E947471B1
:106FC00080915D09E82FF0E0EE0FFF1FE758FC4FBE
:106FD000659174918E010F5F1F4FC8010E944F058C
:106FE00086E693E3B8010E94BC7380915E09E82FA6
:106FF000F0E0EE0FFF1FE358FC4F65917491C8015C
:107000000E944F058DE693E3B8010E94BC7384E7AC
:1070100093E36AE071E00E94BC738BE793E36AE05C
:1070200071E00E94BC739FE2A92EB12CAC0EBD1E74
:10703000C50166E673E30E94B27486E3C82ED12CC4
:10704000CC0EDD1EC6016DE673E30E94B2740DE343
:10705000E02EF12CEC0EFD1EC70164E773E30E94E5
:10706000B2748E010C5B1F4FC8016BE773E30E9483
:10707000B274C501B601A70198010E947934C80114
:107080000E94C874C7010E94C874C6010E94C874D7
:10709000C5010E94C8740C94924489EB93E360E0AC
:1070A00040E00E94CE6680914633882309F445C0B3
:1070B00089EB93E36CED74E00E944C7089EB93E3F1
:1070C00060E041E00E94CE660E942F3389EB93E39B
:1070D00064E041E00E94CE66E091CA09F0E0E85128
:1070E000F14D608170E06F5F7F4F89EB93E34AE081
:1070F00050E00E94617189EB93E36BE041E00E94F4
:10710000CE668091D22E90E027E239E0829FF00196
:10711000839FF00D929FF00D1124E452F54F608192
:1071200070E06F5F7F4F89EB93E34AE050E00E948D
:10713000617181E08093473377C08091C709909156
:10714000C809029749F480914733882329F4809134
:107150004033882309F468C082E090E09093C80926
:107160008093C709109247331092403389EB93E321
:107170006BEC74E00E944C7089EB93E360E041E0BB
:107180000E94CE660E942F3389EB93E362E041E0D8
:107190000E94CE666091CB096F5B89EB93E30E94FE
:1071A0006F706091CC0970E06F5F7F4F8091CB0969
:1071B00090E014E0880F991F1A95E1F7681B790B8E
:1071C00089EB93E34AE050E00E9461718091CC0921
:1071D0008093D83389EB93E369E041E00E94CE6667
:1071E00089EB93E365E00E949C6689EB93E361E0A1
:1071F00071E00E94747180914E09882359F4609166
:1072000053097091540989EB93E34AE050E00E94DE
:10721000FE7006C089EB93E367EC74E00E944C704B
:10722000809153098093D7339091CC098091D833C2
:10723000981719F182E00E9402336091CB096F5BCD
:1072400089EB93E30E946F706091CC0970E06F5FEF
:107250007F4F8091CB0990E0B4E0880F991FBA95D9
:10726000E1F7681B790B89EB93E34AE050E00E9459
:1072700061718091CC098093D8338091D73390E0AD
:1072800020915309309154098217930711F40C94FB
:1072900092448BE00E94023360915309709154092B
:1072A00089EB93E34AE050E00E94FE70809153091D
:1072B0008093D7330C9492448091C7099091C80968
:1072C0000397C1F08FE593E368E071E00E94BC731F
:1072D000BC0188E593E30E949B74BC0181E593E3C4
:1072E0000E949B74BC018AE493E30E949B7481E03A
:1072F0000E94EC338091C7099091C809039741F42B
:1073000080914702882321F480914033882381F1C2
:1073100089EB93E360E040E00E94CE6689EB93E363
:1073200066EB74E00E944C7080914333E82FF0E0EC
:10733000EE0FFF1FE753FD4F659174918E010F5FB4
:107340001F4FC8010E944F05E0914333F0E0E85B16
:10735000FD4F89EB93E3608140E00E94CE6689EBAC
:1073600093E3B8010E947471109247021092403367
:107370008E01055B1F4FE091CA09F0E0E750F14D27
:10738000608170E06F5F7F4FC8014AE00E94067421
:10739000CE018E5A9F4FB8010E94BD7480910A2F72
:1073A000882311F460E201C06EE7E2E5CE2ED12C15
:1073B000CC0EDD1EC6010E9440738C0179E5E72EDC
:1073C000F12CEC0EFD1EE091CA09F0E0E851F14D00
:1073D000608170E06F5F7F4FC7014AE00E940674D2
:1073E000C801B7010E945173BC018E01005A1F4FA2
:1073F000C8010E94B27486E693E3B8010E949B74B0
:10740000C8010E94C874C7010E94C874C6010E94C6
:10741000CE74CE01855B9F4F0E94C8742091CA092B
:107420004091D22E203171F4242F30E087E299E090
:10743000289FF001299FF00D389FF00D1124E35C87
:10744000FC4E19C030E050E084E890E0289FF00145
:10745000299FF00D389FF00D112487E299E09C01DF
:10746000429FC001439F900D529F900D1124E80F41
:10747000F91FEA58F44F8081682F70E06F5F7F4FEB
:107480008E0109591F4FC8014AE00E9406748DE61B
:1074900093E3B8010E949B74C8010E94C87484E7FA
:1074A00093E360E070E00E94BC734091CA094031F0
:1074B00039F48E0102591F4FC8016CE071E092C08F
:1074C00080918D33882309F481C0E42FF0E0EE0F22
:1074D000FF1FEF59FC4F65917491CE0101960E94F8
:1074E0004F054091CA094C3090F58091D22E90E022
:1074F00027E239E0829FF001839FF00D929FF00D0B
:107500001124E452F54FE40FF11D8781882311F413
:1075100060E201C06BE25CE7C52ED12CCC0EDD1E13
:10752000C6010E94827445E7E42EF12CEC0EFD1E8C
:10753000C701BE016F5F7F4F0E948873C601B7010C
:107540000E945173BC018E010D571F4F8AC04F30EE
:1075500041F480915E09882321F08E0106571F4F68
:107560003EC08091D22E90E027E239E0829FF00168
:10757000839FF00D929FF00D1124E452F54FE40F1C
:10758000F11D8781882311F460E201C06BE238E9C4
:10759000C32ED12CCC0EDD1EC6010E94827421E9BF
:1075A000E22EF12CEC0EFD1E6091CA0970E06F5FB7
:1075B0007F4FC7014AE00E940674C601B7010E94CE
:1075C0005173BC018E0101561F4F4BC04F30A9F4BF
:1075D00080915E09882389F08E010A551F4FC801EA
:1075E0006FE071E00E9488738BE793E3B8010E941B
:1075F0009B74C8010E94C87445C08091D22E90E04F
:1076000027E239E0829FF001839FF00D929FF00DF9
:107610001124E452F54FE40FF11D8781882311F402
:1076200060E201C06BE294EBC92ED12CCC0EDD1EC2
:10763000C6010E9482748DEAE82EF12CEC0EFD1E2C
:107640006091CA0970E06F5F7F4FC7014AE00E94F6
:107650000674C601B7010E945173BC018E01055426
:107660001F4FC8010E94B2748BE793E3B8010E94D8
:107670009B74C8010E94C874C7010E94C874C601E7
:107680000E94CE7402ECA02EB12CAC0EBD1EC50122
:1076900066E673E30E94B27419ECC12ED12CCC0EB5
:1076A000DD1EC6016DE673E30E94B274B0EDEB2EF1
:1076B000F12CEC0EFD1EC70164E773E30E94B27467
:1076C0008E0109521F4FC8016BE773E30E94B27429
:1076D000C501B601A70198010E947934C8010E9432
:1076E000C874C7010E94C874C6010E94C874C5014D
:1076F0000E94C87480E00E94EC3383E090E006CBE7
:107700008091C7099091C8090C9721F4809140336A
:107710008823B1F189EB93E360E040E00E94CE66FC
:107720000E942F3389EB93E362E040E00E94CE6633
:1077300089EB93E361EB74E00E944C7089EB93E377
:1077400060E041E00E94CE660E942F3389EB93E314
:1077500062E041E00E94CE6689EB93E36EEA74E05A
:107760000E944C70E091B633F0E0EA5AFD4F89EB8D
:1077700093E360814AE050E00E940F711092403321
:107780008E0102521F4FE091B633F0E0EA5AFD4FEE
:10779000C80160814AE00E9437748AE493E3B8012B
:1077A0000E94A272F82EC8010E94C874FF2099F5A9
:1077B00089EB93E364E041E00E94CE6689EB93E3BA
:1077C0006AEA74E00E944C7089EB93E364E041E064
:1077D0000E94CE66E091B633F0E0EA5AFD4F89EBA5
:1077E00093E360814AE050E00E940F718E010B51DB
:1077F0001F4FE091B633F0E0EA5AFD4FC8016081B7
:107800004AE00E9437748AE493E3B8010E949B74B3
:10781000C8010E94C8748CE090E078CA8091D50AB3
:10782000882321F0813009F039C2E6C18091C7096F
:107830009091C809079721F4809177018823A9F0D6
:107840008FE593E368E071E00E94BC73BC0188E5BA
:1078500093E30E949B74BC0181E593E30E949B74B7
:10786000BC018AE493E30E949B748091C7099091C4
:10787000C809079771F49091D50A809177019817FC
:1078800041F480914702882321F48091403388237A
:10789000A1F189EB93E360E040E00E94CE6689EBC2
:1078A00093E369E974E00E944C7080914333E82FC0
:1078B000F0E0EE0FFF1FE755FD4F659174918E01CB
:1078C0000F5F1F4FC8010E944F05E0914333F0E066
:1078D000E85BFD4F89EB93E3608140E00E94CE6658
:1078E00089EB93E3B8010E9474718091D50A80936B
:1078F000770110924702109240338E0104511F4FBE
:10790000E091CA09F0E0E750F14D608170E06F5FEF
:107910007F4FC8014AE00E940674CE018D509F4FF0
:10792000B8010E94BD7480910A2F882311F460E28F
:1079300001C06EE773EFC72ED12CCC0EDD1EC60141
:107940000E9440738C016AEFE62EF12CEC0EFD1EB6
:10795000E091CA09F0E0E851F14D608170E06F5F9D
:107960007F4FC7014AE00E940674C801B7010E9418
:107970005173BC018E010F5F1E4FC8010E94B2748B
:1079800086E693E3B8010E949B74C8010E94C87404
:10799000C7010E94C874C6010E94CE74CE018451F2
:1079A0009F4F0E94C8742091D22E30E080916209CE
:1079B00090E0FC01EE0FFF1FE80FF91F47E2C42E15
:1079C00049E0D42E2C9DD0012D9DB00D3C9DB00DD5
:1079D0001124EA0FFB1FED5BFC4E20812F70A55C8C
:1079E000BC4E8C9190E0FC01EE0FFF1FE80FF91FD9
:1079F000EE0FFF1FEE0FFF1FE20FF11DE854FE4FC9
:107A00008081E82FF0E0EE0FFF1FE95BFC4F6591EE
:107A100074917E010894E11CF11CC7010E944F057E
:107A20008E01085F1E4FC801B7010E9488738DE662
:107A300093E3B8010E949B74C8010E94C8748091AE
:107A4000620990E02091D22E30E0FC01EE0FFF1F82
:107A5000E80FF91F2C9DC0012D9D900D3C9D900DB0
:107A60001124E80FF91FED5BFC4E80818295877031
:107A7000E82FF0E0EE0FFF1FE75CFC4F659174917B
:107A8000C7010E944F058E01015F1E4FC801B7015B
:107A90000E94887384E793E3B8010E949B74C80135
:107AA0000E94C8742091D22E30E08091620990E04B
:107AB000FC01EE0FFF1FE80FF91F2C9DD0012D9D3B
:107AC000B00D3C9DB00D1124EA0FFB1FEF5BFC4E87
:107AD000608166956F71262F2F5FA45CBC4EAC91C0
:107AE000A03619F4220F220F03C0A03309F4220F8D
:107AF000CE018A5E9E4F2A1729F464E171E00E944C
:107B0000887306C070E06F5F7F4F4AE00E94067482
:107B10008E010A5E1E4F8BE793E3B8010E949B74AF
:107B2000C8010E94C874ADE1AA2EA1E0BA2EAC0E25
:107B3000BD1EC50166E673E30E94B274F4E2CF2E67
:107B4000F1E0DF2ECC0EDD1EC6016DE673E30E9470
:107B5000B274EBE2EE2EE1E0FE2EEC0EFD1EC7014C
:107B600064E773E30E94B2748E010E5C1E4FC8017D
:107B70006BE773E30E94B274C501B601A7019801D7
:107B80000E947934C8010E94C874C7010E94C87459
:107B9000C6010E94C874C5010E94C87489EB93E3B2
:107BA0006FE041E00E94CE668091620990E02091F2
:107BB000D22E30E0FC01EE0FFF1FE80FF91F87E225
:107BC00099E0AC01249FC001259F900D349F900D3A
:107BD0001124E80FF91FED5BFC4E808187FF07C081
:107BE00089EB93E367E974E00E944C7057C089EB1E
:107BF00093E36AE071E050C08091C7099091C80991
:107C0000079741F480917701813021F480914033CE
:107C1000882391F089EB93E360E040E00E94CE6618
:107C200089EB93E366E874E00E944C708091D50A7A
:107C300080937701109240331092433389EB93E3A2
:107C400060E041E00E94CE660E942F3389EB93E30F
:107C500062E041E00E94CE668091D22E90E027E261
:107C600039E0829FF001839FF00D929FF00D112467
:107C7000E55CFC4E8081E82FF0E0EE0FFF1FEF5136
:107C8000FD4F659174918E01095C1D4FC8010E94E2
:107C90004F0589EB93E3B8010E94747187E090E08F
:107CA0000C9486368091C7099091C8090697A9F06F
:107CB0008FE593E368E071E00E94BC73BC0188E546
:107CC00093E30E949B74BC0181E593E30E949B7443
:107CD000BC018AE493E30E949B74E0913233F0E0AC
:107CE000EC5FFC4C92898091D533981771F088E550
:107CF00093E368E071E00E94BC73E0913233F0E0FE
:107D0000EC5FFC4C82898093D5338091C7099091B8
:107D1000C809069741F480914702882321F4809195
:107D200040338823B1F189EB93E360E040E00E94A7
:107D3000CE6689EB93E365E774E00E944C70809116
:107D40004333E82FF0E0EE0FFF1FEF55FD4F659135
:107D500074918E010F5F1F4FC8010E944F05E09183
:107D60004333F0E0E85BFD4F89EB93E3608140E053
:107D70000E94CE6689EB93E3B8010E94747186E09D
:107D800090E09093C8098093C7091092470210921F
:107D90004033E0913233F0E0EC5FFC4C8081E82F1F
:107DA000F0E0EE0FFF1FE350FD4F659174917E01EF
:107DB0000894E11CF11CC7010E944F058E01075C6D
:107DC0001E4F6091323370E06F5F7F4FC8014AE011
:107DD0000E94067486E693E3B8010E949B74C80172
:107DE0000E94C8748E01005C1E4FC801B7010E943A
:107DF00088738DE693E3B8010E949B74C8010E94CA
:107E0000C87480913233E82FF0E0EC5FFC4C82893B
:107E10009E01295B3E4F882331F0C90160E070E08C
:107E20000E94887308C0628170E06F5F7F4FC90154
:107E30004AE00E9406748E01095B1E4F84E793E3BB
:107E4000B8010E949B74C8010E94C8748E01025B35
:107E50001E4FE0913233F0E0EE0FFF1FEE0FFF1FD9
:107E6000E85FFC4C608171818281938120E030E089
:107E700048EC52E40E9487760E94A5759B01AC01F4
:107E8000C801622F4AE00E9437748BE793E3B80180
:107E90000E949B74C8010E94C87425E5A22E21E0AF
:107EA000B22EAC0EBD1EC50166E673E30E94B2742D
:107EB0009CE5C92E91E0D92ECC0EDD1EC6016DE6E3
:107EC00073E30E94B27483E6E82E81E0F82EEC0E94
:107ED000FD1EC70164E773E30E94B2748E01065968
:107EE0001E4FC8016BE773E30E94B274C501B6016F
:107EF000A70198010E947934C8010E94C874C70183
:107F00000E94C874C6010E94C874C5010E94C8744A
:107F1000E0913233F0E0EC5FFC4C8289882309F475
:107F200001C50E949133FEC48091C7099091C80990
:107F30000997A9F08FE593E368E071E00E94BC73B4
:107F4000BC0188E593E30E949B74BC0181E593E347
:107F50000E949B74BC018AE493E30E949B7489EBAA
:107F600093E360E040E00E94CE668091CA092091D0
:107F7000C7093091C809803109F044C02930310562
:107F800069F480914702882349F48091D433803189
:107F900029F480914033882309F475C089EB93E379
:107FA00064E674E00E944C7080914333E82FF0E067
:107FB000EE0FFF1FEF53FD4F659174918E010F5F20
:107FC0001F4FC8010E944F05E0914333F0E0E85B8A
:107FD000FD4F89EB93E3608140E00E94CE6689EB20
:107FE00093E3B8010E94747189E090E09093C8090E
:107FF0008093C709109240331092470280E180932A
:10800000D43341C02930310561F48091470288237F
:1080100041F48091D433803121F080914033882322
:1080200091F189EB93E363E574E00E944C708091D9
:108030004333E82FF0E0EE0FFF1FE754FD4F65914B
:1080400074918E010F5F1F4FC8010E944F05E09190
:108050004333F0E0E85BFD4F89EB93E3608140E060
:108060000E94CE6689EB93E3B8010E94747189E0A7
:1080700090E09093C8098093C70910924033109202
:1080800047021092D4332091D22E30E0A091CA0939
:1080900080916209482F50E08A2F90E0FC01B6E001
:1080A000EE0FFF1FBA95E1F7880F991FE80FF91F30
:1080B000E40FF51FEE0FFF1F87E299E0289FB00144
:1080C000299F700D389F700D1124E60FF71FE9509E
:1080D000F54F9080969496949694A03111F5FA01FC
:1080E000EE0FFF1FE40FF51FE60FF71FDF01AF5B79
:1080F000BC4E9C91929596959695937011968C9105
:108100008770880F880F892BA82EBB2480EF9FEFE4
:10811000A80EB91EEE5BFC4EC080C694C694C694F1
:108120003FC08A2F90E0FC0126E0EE0FFF1F2A954A
:10813000E1F7880F991FE80FF91FE40FF51F3D962F
:10814000EE0FFF1FE60FF71FE452F54F9081929557
:1081500096959695937081818770880F880F892BEB
:10816000A82EBB2420EF3FEFA20EB31E8A2F90E073
:10817000FC01B6E0EE0FFF1FBA95E1F7880F991FDB
:10818000E80FF91FE40FF51F3D96EE0FFF1FE60FF6
:10819000F71FE452F54FC080C694C6943FE0C32257
:1081A0004AE04C1590F4EC2DF0E0EE0FFF1FE35287
:1081B000FD4F659174918E010F5F1F4FC8010E94A2
:1081C0004F0584E793E3B80106C0CC2039F484E777
:1081D00093E368E171E00E94BC733DC058E0C516AE
:1081E00029F484E793E36CE171E0F5CF89E0C816E8
:1081F00029F484E793E360E271E0EDCF9AE0C916D9
:1082000029F484E793E364E271E0E5CF38E7E32EF5
:1082100031E0F32EEC0EFD1EC70168E271E00E9412
:10822000A2738E010F581E4F6C2D70E06F5F7F4F51
:10823000C8014AE00E940674C701B8010E94517348
:10824000BC0184E793E30E949B74C8010E94C87438
:10825000C7010E94CE748E0101581E4FE091CA09D9
:10826000F0E0E750F14D608170E06F5F7F4FC80133
:108270004AE00E940674CE018A579E4FB8010E94C0
:10828000BD7480910A2F882311F460E201C06EE76B
:1082900026E8C22E21E0D22ECC0EDD1EC6010E94A1
:1082A00040738C019DE8E92E91E0F92EEC0EFD1E45
:1082B000E091CA09F0E0E851F14D608170E06F5F34
:1082C0007F4FC7014AE00E940674C801B7010E94AF
:1082D0005173BC018E010C561E4FC8010E94B2742E
:1082E00086E693E3B8010E949B74C8010E94C8749B
:1082F000C7010E94C874C6010E94CE74CE01815885
:108300009E4F0E94C874B7FC23C082EAE82E81E029
:10831000F82EEC0EFD1EC7016BE271E00E94A27305
:108320008E0105561E4FC801B5014AE00E94067431
:10833000C701B8010E945173BC018DE693E30E940E
:108340009B74C8010E94C874C7010E94CE7410C0FB
:108350008E0107551E4FC801B5014AE00E94067400
:108360008DE693E3B8010E949B74C8010E94C87413
:108370002091D22E30E08091620990E0FC01EE0F56
:10838000FF1FE80FF91F87E299E0289FD001299F7E
:10839000B00D389FB00D1124EA0FFB1FEF5BFC4EB0
:1083A000608166956F71262F2F5FA45CBC4EAC91E7
:1083B000A03619F4220F220F03C0A03309F4220FB4
:1083C0008091CA098031E1F4CE0180559E4F2A1771
:1083D00029F464E171E00E94887306C070E06F5F69
:1083E0007F4F4AE00E9406748E0100551E4F8BE7B6
:1083F00093E3B8010E949B74C8010E94C87451C0E5
:1084000015ECA12E11E0B12EAC0EBD1E992041F449
:10841000C50168E171E00E948873EE24FF2428C042
:10842000BEEBEB2EB1E0FB2EEC0EFD1EC7016DE2A4
:1084300071E00E94A2738E0109541E4FE92DF0E0F5
:10844000E659FE4F608180E891E070E00E94297754
:10845000C8014AE00E940674C701B8010E94517326
:10846000BC01C5010E94B274EE24E394FF24F3948E
:108470008E010B531E4F8BE793E3B8010E949B7450
:10848000C8010E94C874FF2029F0CE0189549E4F74
:108490000E94C874EE2029F0CE0182549E4F0E94A3
:1084A000CE74ACECAA2EA1E0BA2EAC0EBD1EC50156
:1084B00066E673E30E94B274F3EDCF2EF1E0DF2E97
:1084C000CC0EDD1EC6016DE673E30E94B274EAEDC8
:1084D000EE2EE1E0FE2EEC0EFD1EC70164E773E315
:1084E0000E94B2748E010F511E4FC8016BE773E3F7
:1084F0000E94B274C501B601A70198010E947934A7
:10850000C8010E94C874C7010E94C874C6010E94B5
:10851000C874C5010E94C8748091CA09803109F0ED
:1085200001C289EB93E36FE041E00E94CE66809147
:10853000620990E02091D22E30E0FC01EE0FFF1F87
:10854000E80FF91F87E299E0AC01249FC001259F45
:10855000900D349F900D1124E80FF91FED5BFC4E38
:10856000808187FF05C089EB93E361E574E047C034
:1085700089EB93E36AE071E00E947471D3C1909338
:10858000C8098093C70989EB93E360E040E00E944B
:10859000CE6689EB93E360E474E00E944C7089EB53
:1085A00093E360E041E00E94CE660E942F3389EBA6
:1085B00093E362E041E00E94CE6680911A33882303
:1085C00029F089EB93E36CE374E004C089EB93E357
:1085D00069E374E00E944C7089EB93E36AE041E048
:1085E0000E94CE6680910C0A882329F089EB93E3E0
:1085F00065E374E004C089EB93E362E374E00E94F6
:108600004C7090C18091C7099091C8090197A9F059
:108610008FE593E368E071E00E94BC73BC0188E5DC
:1086200093E30E949B74BC0181E593E30E949B74D9
:10863000BC018AE493E30E949B748091C7099091E6
:10864000C809019741F480914702882321F4809161
:108650004033882381F189EB93E360E040E00E949E
:10866000CE6689EB93E361E274E00E944C708091E6
:108670004333E82FF0E0EE0FFF1FEF52FD4F6591FF
:1086800074918E010F5F1F4FC8010E944F05E0914A
:108690004333F0E0E85BFD4F89EB93E3608140E01A
:1086A0000E94CE6689EB93E3B8010E947471109228
:1086B0004702109240338E0108511E4F6091132FD4
:1086C00070E06F5F7F4FC8014AE00E94067486E643
:1086D00093E3B8010E949B74C8010E94C8748E0184
:1086E00001511E4F6091142F7091152FC8014AE05F
:1086F0000E9406748DE693E3B8010E949B74C80142
:108700000E94C87456EFC52E51E0D52ECC0EDD1E4A
:10871000E091142FF091152FEE5EF04D618562957A
:108720006F706F5BC6010E94697444E0E42E42E002
:10873000F42EEC0EFD1EC701B6010E94BD74E0913F
:10874000142FF091152FEE5EF04D21858E01035010
:108750001E4F622F70E06F5F7F4F822F82958F7068
:1087600090E034E0880F991F3A95E1F7681B790B88
:10877000C8014AE00E940674C701B8010E94517303
:10878000BC0184E793E30E949B74C8010E94C874F3
:10879000C7010E94CE74C6010E94C87482E893E3A8
:1087A00064E773E30E949B7488E0809344338E01F6
:1087B000055F1D4F6091182F7091192FC8014AE075
:1087C0000E9406748BE793E3B8010E949B74C80172
:1087D0000E94C87422E1A22E22E0B22EAC0EBD1E71
:1087E000C50166E673E30E94B27499E1C92E92E076
:1087F000D92ECC0EDD1EC6016DE673E30E94B27465
:1088000080E2E82E82E0F82EEC0EFD1EC70164E740
:1088100073E30E94B2748E01095D1D4FC8016BE7BE
:1088200073E30E94B274C501B601A70198010E94CA
:108830007934C8010E94C874C7010E94C874C60177
:108840000E94C874C5010E94C87481E090E00C9435
:1088500086368091C7099091C809892B49F4809187
:108860004702882329F480914033882309F456C0B5
:1088700089EB93E360E040E00E94CE6689EB93E3EE
:1088800061E174E00E944C7089EB93E360E041E0A9
:108890000E94CE660E942F3389EB93E360E041E0B3
:1088A0000E94CE6689EB93E36FE271E00E947471DF
:1088B0006091142F7091152F89EB93E34AE050E0FB
:1088C0000E94617189EB93E368E041E00E94CE660B
:1088D00089EB93E364E371E00E9474716091CB09CA
:1088E0006F5B89EB93E30E946F706091CC0970E03D
:1088F0006F5F7F4F8091CB0990E004E0880F991F54
:108900000A95E1F7681B790B89EB93E34AE050E0A5
:108910000E94617110924702109240331092C80970
:108920001092C709C05CDD4F0FB6F894DEBF0FBED2
:10893000CDBFCF91DF911F910F91FF90EF90DF900E
:10894000CF90BF90AF909F900895CF92DF92EF921B
:10895000FF920F931F937B018C0132E0C32E35E30E
:10896000D32E9C0144275527205BC601622F0E940D
:10897000F2675527412F302F2F2DC601622F0E94FD
:108980007E68C6016E2D0E947E681F910F91FF9038
:10899000EF90DF90CF9008950F931F9360E070ECFD
:1089A00084E090E00E94A54402E015E3C8016091D4
:1089B0004E090E947E68C801609155090E947E6838
:1089C000C801609151090E947E68C80160915009F8
:1089D0000E947E68C801609152090E947E68C801A9
:1089E00060915C090E947E68C80160915D090E94E7
:1089F0007E68C80160915E090E947E68C8010E947D
:108A0000C1686AE070E080E090E00E94BA6B1F915C
:108A10000F9108951F93CF93DF9380914F0988237F
:108A200071F110914E09113099F0113018F0123097
:108A300021F513C0809155099091560990935409DE
:108A4000809353090E94882081E08093550215C0CD
:108A50000E9488201093550210C080E293E0A0E0AD
:108A6000B0E080934C0290934D02A0934E02B093DD
:108A70004F020E9488201092550210924F09809157
:108A80005809882351F08091D108882331F00E9441
:108A9000CC44109258090E941B338091590990913F
:108AA0005A09089711F01092580980914E098230A6
:108AB00009F097C1C6E1D3E310E08881882309F467
:108AC00027C180914C0290914D02A0914E02B0912D
:108AD0004F02885B9B40A040B04008F01FC18091CE
:108AE0004C0290914D02A0914E02B0914F02825AD9
:108AF0009840A040B04008F411C160914C027091C0
:108B00004D0280914E0290914F020E94D1759B01BF
:108B1000AC010E94D57429EC3EE84DE059E3E5C074
:108B200080914C0290914D02A0914E02B0914F0263
:108B300089519740A040B04008F4FEC060914C02BB
:108B400070914D0280914E0290914F020E94D1751A
:108B50009B01AC010E94D57428EA37EA4FE059E343
:108B6000C4C080914C0290914D02A0914E02B091F0
:108B70004F02895E9540A040B04008F4EBC0609180
:108B80004C0270914D0280914E0290914F020E94D2
:108B9000D1759B01AC010E94D57427E830EC41E10E
:108BA00059E3A3C080914C0290914D02A0914E02D6
:108BB000B0914F0281519540A040B04008F4D8C018
:108BC00060914C0270914D0280914E0290914F0243
:108BD0000E94D1759B01AC010E94D57425E432EF4F
:108BE00045E159E382C080914C0290914D02A091E1
:108BF0004E02B0914F0289569440A040B04008F414
:108C0000C5C060914C0270914D0280914E029091CE
:108C10004F020E94D1759B01AC010E94D5742CE5D6
:108C200031E948E159E361C080914C0290914D02D5
:108C3000A0914E02B0914F02895A9340A040B0409B
:108C400008F4B2C060914C0270914D0280914E02C6
:108C500090914F020E94D1759B01AC010E94D57486
:108C600022EE3CE34CE159E340C080914C029091EC
:108C70004D02A0914E02B0914F0289549340A04002
:108C8000B04008F49FC060914C0270914D028091F9
:108C90004E0290914F020E94D1759B01AC010E943F
:108CA000D57420EA3EE640E259E31FC080914C02B1
:108CB00090914D02A0914E02B0914F02855F91407C
:108CC000A040B04010F160914C0270914D02809133
:108CD0004E0290914F020E94D1759B01AC010E94FF
:108CE000D5742EEE33E943E259E30E9487769B0167
:108CF000AC0160E070E080E792E40E943D750E9464
:108D0000A5757093540960935309812F0E948D10AB
:108D10001F5F2196123009F0D0CE63C080914C02C3
:108D200090914D02A0914E02B0914F02825A98400C
:108D3000A040B04008F4F4CE80914C0290914D02D6
:108D4000A0914E02B0914F0289519740A040B0408F
:108D500008F407CF80914C0290914D02A0914E02F1
:108D6000B0914F02895E9540A040B04008F41ACF00
:108D700080914C0290914D02A0914E02B0914F0211
:108D800081519540A040B04008F42DCF80914C0215
:108D900090914D02A0914E02B0914F02895694409D
:108DA000A040B04008F440CF80914C0290914D0219
:108DB000A0914E02B0914F02895A9340A040B0401A
:108DC00008F453CF80914C0290914D02A0914E0235
:108DD000B0914F0289549340A040B04008F095CF25
:108DE00065CFDF91CF911F9108953F924F925F928F
:108DF0006F927F928F929F92AF92BF92CF92DF92AB
:108E0000EF92FF920F931F93DF93CF9300D000D088
:108E100000D0CDB7DEB7062FC82EDD24EE24FF2408
:108E2000603109F42FC1262F30E040E050E0298363
:108E30003A834B835C83C701B60123E130E040E015
:108E400050E00E94EA7629813A814B815C81620F71
:108E5000731F841F951FA7E0660F771F881F991F38
:108E6000AA95D1F70E94A5443324402E552484E8C6
:108E700090E0489E4001499E900C589E900C112411
:108E80005201AA0CBB1CC201E6E0880F991FEA95AB
:108E9000E1F7A80EB91E4CC0D501A30DB11DFD010F
:108EA0003D96EE0FFF1FE40FF51FE452F54F2081B2
:108EB000022F0695017010E0000F111F822F86957A
:108EC00086958F7090E0880F991F880F991F082B47
:108ED000192B822F817090E0082B192B2295269553
:108EE0002695237081818770880F880F822B90E0F0
:108EF00026E0880F991F2A95E1F7082B192BAA0F56
:108F0000BB1FA40FB51FA950B54F8C91887F8E83CE
:108F10001D824D815E81042B152B82E095E3602F2D
:108F20000E947E6882E095E3612F0E947E68339400
:108F30008091D22E90E017E2612E19E0712E869D6D
:108F4000A001879D500D969D500D1124F401E40F52
:108F5000F51FEA58F44F8081831508F09DCF82E019
:108F600095E30E94C1686AE070E080E090E00E94B2
:108F7000BA6BC701B60120E839E040E050E00E943A
:108F8000EA767B018C0180E098E0A0E0B0E0E80E9A
:108F9000F91E0A1F1B1F69817A818B819C8126E043
:108FA00030E040E050E00E94EA76E60EF71E081F2F
:108FB000191FC801B7010E94A54482E095E360E053
:108FC0000E947E688091D22E90E0869DF001879D60
:108FD000F00D969DF00D1124E80DF91DEA58F44F9F
:108FE00082E095E360810E947E688091D22E90E0BD
:108FF000869DF001879DF00D969DF00D1124E80DE2
:10900000F91DE958F44F82E095E360810E947E6883
:109010008091D22E90E0869DF001879DF00D969D67
:10902000F00D1124E80DF91DE758F44F82E095E3A7
:1090300060810E947E688091D22E90E0869DF00132
:10904000879DF00D969DF00D1124E80DF91DE8584F
:10905000F44F82E095E360810E947E688091D22E79
:1090600090E0869DF001879DF00D969DF00D1124F6
:10907000E452F54FE40DF51D82E095E367810E940F
:109080007E68F5C0C701B60120E839E040E050E055
:109090000E94EA766B017C016058774F8F4F9F4F9B
:1090A0000E94A5448091D22E90E007E219E0809FB3
:1090B000F001819FF00D909FF00D1124E35CFC4EB8
:1090C00082E095E360810E947E688091D22E90E0DC
:1090D000809FF001819FF00D909FF00D1124E45CC2
:1090E000FC4E82E095E360810E947E688091D22EE2
:1090F00090E0809FF001819FF00D909FF00D112472
:10910000E25CFC4E82E095E360810E947E68809183
:10911000D22E90E0809FF001819FF00D909FF00D86
:109120001124E15CFC4E82E095E360810E947E6840
:109130008091D22E90E0809FF001819FF00D909F52
:10914000F00D1124E55CFC4E82E095E360810E9405
:109150007E6800E0B7E2AB2EB9E0BB2E11C0802FD5
:1091600090E0FC01EE0FFF1FE80FF91FE20FF31F65
:10917000ED5BFC4E608182E095E30E947E680F5FAC
:109180008091D22E90E08A9D90018B9D300D9A9D0A
:10919000300D1124F901E35CFC4E80810817F8F2D0
:1091A00082E095E30E94C1686AE070E080E090E0B0
:1091B0000E94BA6BC701B6016050774F8F4F9F4F27
:1091C0000E94A544FF24E7E2CE2EE9E0DE2E3EC059
:1091D0008F2D90E0FC01EE0FFF1FE80FF91FE20F4B
:1091E000F31FDF01AF5BBC4E2C91022F06950F7170
:1091F00010E0000F111F422F42954695469543708F
:1092000011968C918770880F880F842B90E056E020
:10921000880F991F5A95E1F7082B192B217030E020
:10922000022B132BEE5BFC4E808148EF942E98228C
:1092300088240829192982E095E3602F0E947E681E
:1092400082E095E3612F0E947E68F3948091D22E94
:1092500090E08C9D90018D9D300D9C9D300D1124D2
:10926000F901E35CFC4E80818F1508F0B1CF82E0FC
:1092700095E30E94C1686AE070E080E090E00E949F
:10928000BA6B26960FB6F894DEBF0FBECDBFCF9156
:10929000DF911F910F91FF90EF90DF90CF90BF90E3
:1092A000AF909F908F907F906F905F904F903F9086
:1092B00008952F923F924F925F927F928F929F924A
:1092C000AF92BF92CF92DF92EF92FF920F931F93D4
:1092D000DF93CF9300D000D0CDB7DEB77724C8C0DE
:1092E000003109F43FC0C701B6010E94A54410E057
:1092F00082E095E362E00E947E6882E095E364E0AC
:109300000E947E681F5F103499F782E095E30E9407
:10931000C1686AE070E080E090E00E94BA6BC5012D
:10932000B4010E94A54482E095E361E00E947E685A
:1093300082E095E36FE00E947E6882E095E368E159
:109340000E947E6882E095E361E00E947E6882E090
:1093500095E360E00E947E6882E095E360E00E9411
:109360007E6844C069817A818B819C810E94A5447A
:1093700082E095E36FE00E947E6882E095E368E119
:109380000E947E6882E095E361E00E947E6882E050
:1093900095E360E00E947E6882E095E360E00E94D1
:1093A0007E6810E082E095E360E30E947E681F5FC4
:1093B0001034C1F782E095E30E94C1686AE070E072
:1093C00080E090E00E94BA6BC201B1010E94A54406
:1093D00010E082E095E368E10E947E6882E095E318
:1093E00064E00E947E681F5F103499F782E095E385
:1093F0000E94C1686AE070E080E090E00E94BA6B71
:109400000F5F86E090E0A0E0B0E0880E991EAA1EF3
:10941000BB1E80E890E0A0E0B0E0C80ED91EEA1EB6
:10942000FB1E013109F05CCF272D26952695269548
:1094300081E090E0A0E0B0E004C0880F991FAA1F6F
:10944000BB1F2A95D2F79C01AD018091EC3390911E
:10945000ED33822B932B9093ED338093EC3360E0CC
:1094600070E040E00E940D0A739490E8791651F183
:10947000672D70E080E090E020E839E040E050E0C7
:109480000E94EA766B017C01812C18E0912EA12CC0
:10949000B12C860E971EA81EB91EDC01CB01805888
:1094A000974FAF4FBF4F89839A83AB83BC83212CE7
:1094B000B9E03B2E412C512C2C0C3D1C4E1C5F1C4A
:1094C00000E00ECF60E070EC84E090E00E94A544E4
:1094D00082E095E360E00E947E6882E095E368E7C1
:1094E0000E947E6882E095E361E00E947E6882E0EF
:1094F00095E361E00E947E6882E095E361E00E946E
:109500007E6882E095E30E94C1686AE070E080E0D6
:1095100090E00E94BA6B82E095E367E570E00E94FC
:10952000FC6782E095E36FEF0E947E6882E095E33E
:109530006DEF0E947E6882E095E360E00E947E68A5
:1095400082E095E361E00E947E6882E095E363E05B
:109550000E947E6882E095E30E94C1686AE070E044
:1095600080E090E00E94BA6B0F900F900F900F90E8
:10957000CF91DF911F910F91FF90EF90DF90CF90EF
:10958000BF90AF909F908F907F905F904F903F9053
:109590002F90089560E070EC84E090E00E94A54474
:1095A00082E095E30E94C16882E095E364E540E8CB
:1095B0000E94D66882E095E30E940F68833008F02D
:1095C00082E080934E0982E095E30E940F6890E06C
:1095D0008E31910518F48EE190E005C08B3F910526
:1095E00010F08AEF90E0909356098093550982E03D
:1095F00095E30E940F68882311F481E003C0813154
:1096000008F080E18093510982E095E30E940F68A1
:10961000882311F481E003C0813108F080E1809358
:10962000500982E095E30E940F68843008F083E0DF
:109630008093520982E095E30E940F68823010F413
:1096400082E003C08B3008F08AE080935C0982E0FE
:1096500095E30E940F68811181E080935D0982E0AB
:1096600095E30E940F68811181E080935E0908955F
:109670001F930E94CA4A10926309109269011092C6
:1096800068011092453383E090E090935A098093EB
:10969000590980E00E94656C0E94337280916800D5
:1096A000816080936800D89A80916B00836080937A
:1096B0006B0010920C0A8091550990915609909375
:1096C00054098093530910914E09113059F011300B
:1096D00018F0123081F40BC00E94882081E0809342
:1096E000550209C00E9488201093550204C00E94B0
:1096F00088201092550210924F0980915F098823AB
:1097000011F02C9A01C02C988091D22E90E027E283
:1097100039E0829FF001839FF00D929FF00D11249C
:10972000DF01AD5BBC4E2C91322F3F70E55CFC4EEF
:10973000808190E0FC01EE0FFF1FE80FF91FEE0F94
:10974000FF1FEE0FFF1FE30FF11DE854FE4FE081F6
:10975000F0E0EE0FFF1FEE56FE4F2695269526955C
:10976000922F9E7080E020813181820F931F0E9492
:10977000BF0A1F9108952F923F924F925F926F926E
:109780007F928F929F92AF92BF92CF92DF92EF9291
:10979000FF920F931F93DF93CF93CDB7DEB76E97F2
:1097A0000FB6F894DEBF0FBECDBF062F90E0A0E04D
:1097B000B0E0BC01CD0120E839E040E050E00E947B
:1097C000EA765B016C01412C78E0572E612C712CFC
:1097D0004A0C5B1C6C1C7D1CA60195012058374F60
:1097E0004F4F5F4F2B873C874D875E87CA01AA2763
:1097F000BB27382F305B3E83D601C5018050974F81
:10980000AF4FBF4F8A839B83AC83BD83CD01AA2713
:10981000BB27E82FE05BE98310E087E299E09C0139
:10982000029FC001039F900D129F900D112436E7F7
:10983000832E3BE0932E880E991EAC014D51554F5F
:1098400058874F831A8619861C018452954FDC0174
:10985000AF59B74FBC8BAB8BFC01E05AF74FFE8B77
:10986000ED8B9C012E59374F388F2F8BAC014D5902
:10987000574F5A8F498FDC01A15AB74FBC8FAB8F1E
:10988000E985FA85709709F4D9C0C301B2010E9435
:10989000A54482E095E30E94C168930144275527BF
:1098A000205B82E095E3622F46E00E94D66882E06A
:1098B00095E30E940F6882E095E30E940F68D4014F
:1098C0008C9382E095E30E940F68F401818382E02B
:1098D00095E30E940F68D40113968C9382E095E380
:1098E0000E940F68F401828382E095E30E940F6872
:1098F000AF81B8858C93F401E080FF240894E11CCB
:10990000F11CEE0CFF1C0027F7FC0095102FC60180
:10991000B5010E94A54482E095E30E94C1689601CA
:1099200044275527205B82E095E3622F4E2D0E944D
:10993000D668EE2429853A85220F331F89859A85BA
:1099400016E0880F991F1A95E1F7280F391F3E8FEF
:109950002D8F6EC082E095E30E940F688C0182E03B
:1099600095E30E940F68888B1F86A80150708F8531
:109970009889482B592B6E2D70E0ED8DFE8DE60FEA
:10998000F71F3D96EE0FFF1FE20DF31DE452F54F5A
:10999000242F217030813C7FCA018270907096958F
:1099A00087958170880F322B382BCA018C73907089
:1099B00096958795969587958F70282F220F220F61
:1099C000337C322B3083882311F4337C3083AD8D8C
:1099D000BE8DA60FB71FFD013D96EE0FFF1FE20DD6
:1099E000F31DE452F54FCA01807C977076E096959E
:1099F00087957A95E1F7382F3295330F330F307C06
:109A000020812F73232B2083869586958770218153
:109A1000287F282B2183AA0FBB1FA20DB31DA9509D
:109A2000B54F952F987F8C918770892B8C93E394F9
:109A3000D4018C918E1508F08DCFD0C06B857C85BC
:109A40008D859E850E94A54482E095E30E94C168B1
:109A500082E095E36E8140E80E94D66882E095E35B
:109A60000E940F68EB89FC89808382E095E30E9465
:109A70000F68AD89BE898C9382E095E30E940F68E0
:109A8000EF89F88D808382E095E30E940F68A98DAD
:109A9000BA8D8C9382E095E30E940F68EB8DFC8D6C
:109AA0008083893008F088E0AB8DBC8D8C9300E01A
:109AB00022C082E095E30E940F68202F30E0F90178
:109AC000EE0FFF1FE20FF31FE20DF31DED5BFC4EE7
:109AD000282F30E02077307094E0359527959A95BF
:109AE000E1F727702295207F982F90788F70282B90
:109AF000292B20830F5FEB89FC89E080E016C8F6F4
:109B00006A817B818C819D810E94A54482E095E3DE
:109B10000E94C1682E2D30E02F5F3F4F220F331F70
:109B2000442737FD4095542F82E095E36981422F09
:109B30000E94D668EE244CC082E095E30E940F6834
:109B40008C0182E095E30E940F688A8B198A10705D
:109B500029893A89022B132B8E2D90E0AC01440FFA
:109B6000551F480F591F420D531DFA01EF5BFC4E64
:109B7000702F7170C8018E739070969587958F7154
:109B8000880F9801207C377066E0369527956A9596
:109B9000E1F7622F6295660F660F607C872B862B3C
:109BA000808326952695812F869586958695FA0140
:109BB000EE5BFC4E982F990F990F990F2770292B68
:109BC0002083815E8F71803110F027702083E394B1
:109BD000AB89BC898C918E1508F0AECFE985FA85EA
:109BE0003196FA87E98724E830E0820E931E86E0FA
:109BF00090E0A0E0B0E0480E591E6A1E7B1EAF81C7
:109C0000B8851196B887AF8320E830E040E050E097
:109C1000A20EB31EC41ED51E719709F031CE6E96EA
:109C20000FB6F894DEBF0FBECDBFCF91DF911F916D
:109C30000F91FF90EF90DF90CF90BF90AF909F90EB
:109C40008F907F906F905F904F903F902F900895EE
:109C5000AF92BF92CF92DF92EF92FF920F931F933A
:109C60008F3708F08FE700D000D0682F70E080E0D9
:109C700090E02AEF3FE040E050E0EDB7FEB72183EF
:109C800032834383548320E030E040E050E0EFE74C
:109C9000EE2EF12C012D112DAA24BB2465010E946A
:109CA000AA717F70706940913433309135332091BF
:109CB000F5330F900F900F900F90222381F02130F9
:109CC00051F48DB38093F7339DB38091F633809533
:109CD00089238DBB04C08FB7F8948093F7334CBDB4
:109CE0003DBD12987EBD00000DB407FEFDCF8EB5C0
:109CF0006EBD00000DB407FEFDCF8EB5129A222373
:109D000039F08091F733213011F48DBB01C08FBF42
:109D10001F910F91FF90EF90DF90CF90BF90AF9089
:109D20000895EF92FF920F931F93CF93DF938C01CF
:109D3000C8E0D0E057E2E52E59E0F52EC8010C2E20
:109D400002C0969587950A94E2F780FF39C0599A28
:109D5000FE01EC59F64F2081FE01EE0FFF1FCE01F0
:109D600036E0880F991F3A95E1F7E80FF91FE20FE7
:109D7000F11D3D968091D22E90E0EE0FFF1F9C01C9
:109D80002E9DC0012F9D900D3E9D900D1124E80F3A
:109D9000F91FE452F54F808181FD02C084E101C0CA
:109DA0008FE70E94284E82B18F71FE01EA5CFD4F61
:109DB0009081892B82B988E290E00E94136C5998B7
:109DC0002196CC30D10509F0B9CF88E290E00E940D
:109DD000136C599AC0E0D0E097E2E92E99E0F92E91
:109DE000C8010C2E02C0969587950A94E2F780FF71
:109DF00039C0149AFE01EC59F64F2081FE01EE0F96
:109E0000FF1FCE01B6E0880F991FBA95E1F7E80F62
:109E1000F91FE20FF11D3D968091D22E90E0EE0FDA
:109E2000FF1F9C012E9DC0012F9D900D3E9D900D0A
:109E30001124E80FF91FE452F54F808181FD02C023
:109E400084E101C08FE70E94284E82B18F71FE012C
:109E5000E25CFD4F9081892B82B988E290E00E94FC
:109E6000136C14982196C830D10509F0B9CF88E257
:109E700090E00E94136C149ADF91CF911F910F9183
:109E8000FF90EF9008956F927F928F929F92AF9282
:109E9000BF92CF92DF92EF92FF920F931F93CF93D7
:109EA000DF9381E00E94D3059093280980932709CE
:109EB0008091C409882379F08091590990915A09B9
:109EC000089749F483E090E090935A0980935909E8
:109ED00081E0809346028091590990915A09059733
:109EE00011F01092F0088091590990915A0984302C
:109EF000910531F00C9721F01092C90910920333AB
:109F00008091AD33882379F00E94AC6B6093AF33BE
:109F10007093B0338093B1339093B23381E08093E8
:109F2000AE331092AD338091AE338823F1F080913F
:109F3000C4098823D1F00E94AC6B2091AF333091DB
:109F4000B0334091B1335091B233621B730B840B29
:109F5000950B615971408040904038F081E08093CA
:109F6000AC33109255021092AE338091840888234E
:109F700041F08091C208882321F480915502882302
:109F800029F48091AB33882309F446C081E08093A3
:109F9000C409109276011092B5331092AB3310922F
:109FA00063091092CE0A1092CD0A2C982C9A109226
:109FB0005F0980930D2F10928E0810926901109204
:109FC000680180E090E021E0FC01EB58F64F108240
:109FD000FC01EF50F64F1082FC01E253F64F208354
:109FE000FC01E956F64F1082FC01E257FC4C20833D
:109FF000FC01E855F64F208301968131910521F748
:10A0000080911633882311F0109212338091173308
:10A01000882311F0109213338091B533882341F0D7
:10A020008091C409882321F01092B53310928E08D4
:10A0300080918B08882341F08091C208882321F405
:10A0400080915502882341F480918933882321F43B
:10A050008091AC338823D9F15F981092020A109254
:10A060005F091092C9091092D00A1092CF0A80910C
:10A070008933882311F010928E088091AC338823A5
:10A0800011F010928E081092AC3310918E081F5F61
:10A0900010938E08113019F01230C9F40FC01093CC
:10A0A00076011092C40980915E09882381F080E0D6
:10A0B00090E80E94550A1093600909C01092760139
:10A0C00081E08093C40910928E08109263098091F8
:10A0D000C2088823E1F080910209882321F0809151
:10A0E000CA090E941B1A80910909882321F08091D6
:10A0F000CA090E94491C8091A708882309F4B3C0AB
:10A100008CE090E090935A0980935909A9C08091FE
:10A11000590990915A098230910569F48091020998
:10A12000882311F00E94C417809109098823D9F06F
:10A130000E940E1818C00397B1F480910209882379
:10A1400041F08091CA090E94CE148091CA0980937F
:10A15000512680910909882331F08091CA096091C4
:10A1600051260E94DA1580911709882391F0809179
:10A17000590990915A09039719F083E090E002C0C1
:10A1800082E090E090935A098093590981E080938E
:10A1900046028091A7088823E1F0809159099091A7
:10A1A0005A09049719F084E090E002C083E090E03F
:10A1B00090935A09809359098091CA09803121F4FA
:10A1C00081E08093033302C01092033381E08093D7
:10A1D00046028091ED08882331F18091F0088F5F6D
:10A1E0008093F008813019F08230D1F40FC0809153
:10A1F000590990915A099093C6098093C50985E041
:10A2000090E090935A09809359090AC08091C5093A
:10A210009091C60990935A09809359091092F008B9
:10A2200081E0809346028091590990915A090597DF
:10A2300011F01092F0088091590990915A090897ED
:10A2400011F0109245338091590990915A0907975E
:10A25000029710F0109245338091B608882319F0C8
:10A2600081E080934602809184088823E9F0809100
:10A27000C2088823C9F08091C4098823A9F488E022
:10A2800090E090935A0980935909809145338F5FEC
:10A2900080934533833018F081E0809345331092EA
:10A2A000433381E0809346028091BC08882321F0EB
:10A2B00081E08093493307C08091BD08882329F04D
:10A2C0001092493381E0809346028091AE08882342
:10A2D00021F081E08093483307C08091AF08882344
:10A2E00029F01092483381E0809346022091590969
:10A2F00030915A09C9010397029768F02730310558
:10A3000051F02930310539F02630310521F02C305B
:10A31000310509F02FC68091270990912809892BD2
:10A3200011F4109226098091C9088823F1F18091D7
:10A33000FB08882369F083E090E090935A098093AA
:10A3400059090E94B1088093CA0981E080934602AE
:10A350008091D108882361F087E090E090935A09BA
:10A360008093590980E18093CA0981E08093460275
:10A3700080911009882361F083E090E090935A095E
:10A380008093590980E18093CA0981E08093460255
:10A3900080919208882349F086E090E090935A09D2
:10A3A0008093590981E08093460280919208882326
:10A3B000E1F02091CA092031C1F48091C9088823B5
:10A3C000A1F487E090E090935A0980935909809115
:10A3D0003F338093D50A91E0909346028F5F80933C
:10A3E0003F33823010F010923F33809159099091A1
:10A3F0005A09079711F010923F3380911009882372
:10A4000089F08091590990915A09079759F410924F
:10A410003F3383E090E090935A098093590981E09B
:10A420008093460280911D09882309F4BEC0809163
:10A43000C409882309F4B9C0F090CA093091D22E1A
:10A4400040E1F41609F040C08091740990E0232F98
:10A4500030E0FC01EE0FFF1FE80FF91F87E299E0E3
:10A46000B901689F9001699F300D789F300D1124CC
:10A47000E20FF31FEF5BFC4E80818E7F8083809123
:10A48000740990E0FC01EE0FFF1FE80FF91FE20FC7
:10A49000F31FDF01AF5BBC4E8C918E7F8C93EE5B24
:10A4A000FC4E8081877080839C9111968C911197CE
:10A4B000887F846011968C931197917098619C931A
:10A4C00081E08093D30A71C06F2D70E08B010C592D
:10A4D000164FD8012C91DB01AA0FBB1FCB0146E020
:10A4E000880F991F4A95E1F7A80FB91FFD01E20FE8
:10A4F000F11D3D96232F30E0EE0FFF1F87E299E01C
:10A50000289FA001299F500D389F500D1124E40F62
:10A51000F51FE452F54F80818E7F8083F801208102
:10A5200030E0A20FB31F1D96AA0FBB1FA40FB51FCB
:10A53000A452B54F8C91837C8C938F2D90E0FC01BD
:10A54000B6E0EE0FFF1FBA95E1F7880F991FE80FED
:10A55000F91FE20FF31F3D96EE0FFF1FE40FF51FEB
:10A56000E452F54F80818F7380838181887F84607E
:10A5700081838F2D90E0FC0116E0EE0FFF1F1A95EE
:10A58000E1F7880F991FE80FF91FE20FF31FEE0F95
:10A59000FF1FE40FF51FE950F54F8081877080831E
:10A5A0006A52714D81E0DB018C938091C20888234F
:10A5B00069F080911E09882349F08091CA09803191
:10A5C00019F00E94131702C00E9470178091D708DB
:10A5D000882309F444C18091FB08882309F43FC112
:10A5E0008091C208882309F46EC08091D22E90E039
:10A5F00027E239E0829F8001839F100D929F100D0A
:10A6000011240452154FF801F0800E94B108E09126
:10A61000CA09F0E0E851F14D90819295907F980F32
:10A62000D8019C9320E030E064E870E047E259E014
:10A6300011E08091D22E90E0269FF001279FF00D2F
:10A64000369FF00D1124DC01A49FC001A59F900D41
:10A65000B49F900D1124E80FF91FEA58F44FDC0164
:10A66000A452B54F8C918083F901EA52F14D1083C9
:10A670002F5F3F4F20313105E1F6FD01EF59F74FD4
:10A680008C9180831093D30A80915D09813009F009
:10A69000E3C010E0C7E2D9E08091D22E90E08C9F19
:10A6A000F0018D9FF00D9C9FF00D1124E452F54FA9
:10A6B0004081F41620F4812F6F2D0E9465181F5FD2
:10A6C000113151F7C9C08091CA093091D22E803121
:10A6D000E9F4032F10E00E94B10827E239E0029F5D
:10A6E000D001039FB00D129FB00D1124A35CBC4E8E
:10A6F000E091CA09F0E0E851F14D90819295907F88
:10A70000980F9C9381E08093D30A52C0232F30E0AE
:10A7100090E044E8E42EF12C8E9DF0018F9DF00D29
:10A720009E9DF00D1124C7E2D9E02C9F80012D9F42
:10A73000100D3C9F100D1124E00FF11FEA58F44F4B
:10A74000D0800E94B1085091CA09A52FB0E0AE9DFB
:10A750009001AF9D300DBE9D300D1124020F131FCF
:10A760000A58144FFD01E851F14D90819295907F68
:10A77000980FF8019083AA52B14D81E08C9380919B
:10A780005D098130A9F48091D22E90E08C9FF00178
:10A790008D9FF00D9C9FF00D1124E20FF31FEA58DE
:10A7A000F44F4081D41620F4852F6D2D0E9465183A
:10A7B0008091D22E90E027E239E0829FF001839FC2
:10A7C000F00D929FF00D1124E452F54F108220E01D
:10A7D00030E064E870E047E259E08091D22E90E0EA
:10A7E000269FF001279FF00D369FF00D1124DC010C
:10A7F000A49FC001A59F900DB49F900D1124E80F58
:10A80000F91FEA58F44FE081DC01A452B54F8C9156
:10A810008E1718F4EC932093E72E2F5F3F4F2031D3
:10A820003105D9F68091D22E90E027E239E0829F5F
:10A83000F001839FF00D929FF00D1124E452F54F2B
:10A84000EF59F74F9081E156F8408081891720F445
:10A85000908380E18093E72E81E08093460280918F
:10A86000C208882309F45DC08091CA08882309F4CE
:10A8700058C04091CA094E3009F453C04F3009F412
:10A8800050C0403109F44DC08091D22E90E027E2B3
:10A8900039E0829FF001839FF00D929FF00D11240B
:10A8A000E452F54FE40FF11D8781882379F1178277
:10A8B00020E030E047E259E08091CA0990E0FC01D5
:10A8C00006E0EE0FFF1F0A95E1F7880F991FE80FCA
:10A8D000F91FE20FF31F3D968091D22E90E0EE0F0C
:10A8E000FF1FBC01649FC001659F900D749F900D78
:10A8F0001124E80FF91FE452F54F808182608083B4
:10A900002F5F3F4F20343105B9F602C081E08783C5
:10A9100081E080934602E091CA09F0E0EA52F14DED
:10A9200080838091590990915A098330910539F0BB
:10A930008730910521F08930910509F057C1809148
:10A94000FC08882321F0109226091092CE338091C2
:10A95000D708882309F00EC38091C908882309F01D
:10A9600009C38091C2088823A9F480915909909164
:10A970005A09039779F48091CA09209127093091E7
:10A980002809803121F4C9010E94470703C0C90189
:10A990000E944B068091FB08882309F49AC080919D
:10A9A000590990915A098930910519F0079709F0D2
:10A9B00090C00E94B108E091CA09F0E0E851F14D61
:10A9C00090819295907F980F909362098091C20830
:10A9D000882309F47BC08091590990915A090997FD
:10A9E00009F074C040E050E0C7E2D9E08091270947
:10A9F00090912809042E02C0969587950A94E2F753
:10AA000080FF5EC06091CA093091D22E6031E1F4BE
:10AA1000832F90E0FA01EE0FFF1FE40FF51FDC011A
:10AA2000AC9FC001AD9F900DBC9F900D1124E80F0D
:10AA3000F91FEF5BFC4E90E0808180FF91E0808108
:10AA40008E7F892B80833CC0232F30E0862F90E0BF
:10AA5000DC01E6E0AA0FBB1FEA95E1F7880F991F1A
:10AA6000A80FB91FA40FB51F1D96AA0FBB1FF90190
:10AA7000EC9F9001ED9F300DFC9F300D1124A20F33
:10AA8000B31FA452B54F70E0862F90E0FC0106E0A2
:10AA9000EE0FFF1F0A95E1F7880F991FE80FF91FC6
:10AAA000E40FF51F3D96EE0FFF1FE20FF31FE45278
:10AAB000F54F808180FF71E08C918E7F872B8C9386
:10AAC0004F5F5F4F4031510509F090CF81E0809397
:10AAD00046028091590990915A098930910541F0B7
:10AAE000079709F062C08091CA09803109F05DC002
:10AAF0000E94CD08082F0E94B10810E0081B110920
:10AB00000130110509F0A7C48091CE33882309F0E4
:10AB1000A2C42091D22E30E08091620990E0FC0125
:10AB2000EE0FFF1FE80FF91F87E299E0AC01249FA9
:10AB3000C001259F900D349F900D1124E80FF91F3F
:10AB400022C00E94CD08682F8091D22E90E027E28B
:10AB500039E0829FA001839F500D929F500D1124D8
:10AB6000FA01E35CFC4E80816817F9F48091CE33E2
:10AB70008823D9F4862F90E0FC01EE0FFF1FE80F29
:10AB8000F91FE40FF51FED5BFC4E90E0808187FF1D
:10AB900091E097959927979580818F77892B80836E
:10ABA00081E08093CE33809346028091C20888234F
:10ABB00009F4E0C18091FB08882309F4DBC189E036
:10ABC00090E090935A09809359090E94B108E0914E
:10ABD000CA09F0E0E851F14D90819295907F980F6D
:10ABE0009093620981E080934602C4C1843091054C
:10ABF00009F037C18091C409882361F08091D108A0
:10AC0000882341F090E08091C909882309F491E0FC
:10AC10009093C90980911D09882309F451C0A0911E
:10AC2000CA093091D22EA031F9F48091740990E0D4
:10AC3000232F30E0FC01EE0FFF1FE80FF91F87E222
:10AC400099E0BC01269FC001279F900D369F900D73
:10AC50001124E80FF91FEF5BFC4E80818E7F80830B
:10AC600081E08093D30A2CC0B0E0FD01EC59F64F8F
:10AC70002081FD01EE0FFF1FCD0176E0880F991FA7
:10AC80007A95E1F7E80FF91FE20FF11D3D96232FAA
:10AC900030E0EE0FFF1F87E299E0AC01249FC00176
:10ACA000259F900D349F900D1124E80FF91FE45259
:10ACB000F54F80818E7F8083AA52B14D81E08C93C5
:10ACC0008091D708882351F48091C908882331F4F2
:10ACD00080910333882369F00E94A30E20E030E0C6
:10ACE00054E8652E712C47E2842E49E0942E01E051
:10ACF0005EC091E3E92E97E0F92EC0E0D0E081E05C
:10AD0000C82ED12C80912709909128090C2E02C0C1
:10AD1000969587950A94E2F7982F9170D7019C93A6
:10AD200011968C9111979817A9F112968C918823FE
:10AD300089F5913079F586010C2E02C0000F111FA4
:10AD40000A94E2F7C8010E94914EC8010E94550A78
:10AD500080ED97E00E94136C80E090E00E94550A1D
:10AD60008091C4098823B1F08091C909813091F4A0
:10AD7000FE01EA57F64F8081FE0106E0EE0FFF1F4D
:10AD80000A95E1F7E80FF11DEE0FFF1FEE5AF94D9E
:10AD9000D182C082F70180818183219627E030E053
:10ADA000E20EF31EC031D10509F0ACCF97CFF90107
:10ADB000EB58F64F8081882309F04CC010E0269DA7
:10ADC0005001279DB00C369DB00C11247901B6E0DE
:10ADD000EE0CFF1CBA95E1F7B901660F771F6E0DF7
:10ADE0007F1DF6EDCF2EFEE2DF2EC20ED31E20C059
:10ADF000412F50E0D701A40FB51FAA0FBB1FAE5AB9
:10AE0000B94D8D919C911197892B89F0FB01E40F2D
:10AE1000F51F3D96EE0FFF1FEC0FFD1FE452F54F9F
:10AE2000808183608083F60100831D921C921F5FE6
:10AE30008091D22E90E0889DE001899DD00D989D53
:10AE4000D00D1124F501EC0FFD1FEA58F44F80815D
:10AE5000181770F22F5F3F4F2031310509F0A7CF4F
:10AE600089C00C9709F086C0809127099091280924
:10AE70009093B8338093B7338091C409882309F441
:10AE800079C08091D108882341F090E08091C90970
:10AE9000882309F491E09093C9098091C909882316
:10AEA00009F468C060E070E007E219E0FF24F39461
:10AEB00037E08091B7339091B833062E02C0969553
:10AEC00087950A94E2F780FF4FC0EB01CC59D64F2B
:10AED0002881AB01440F551FCB01B6E0880F991FA5
:10AEE000BA95E1F7480F591FFA01E20FF11D3D969F
:10AEF0008091D22E90E0EE0FFF1F809FD001819FA6
:10AF0000B00D909FB00D1124EA0FFB1FE452F54FD6
:10AF10008081816080839091B6339923A1F08881EC
:10AF2000FA01E80FF11DEE0FFF1FEA0FFB1FE950BA
:10AF3000F54F232F291B922F990F990F990F80817D
:10AF40008770892B0CC08881FA01E80FF11DEE0F84
:10AF5000FF1FEA0FFB1FE950F54F80818770808348
:10AF6000FB01EA52F14DF0826F5F7F4F6031710556
:10AF700009F09FCF8091590990915A09029709F0E1
:10AF80001FC18091C908882389F08091FB0888231C
:10AF900069F083E090E090935A09809359090E94E8
:10AFA000B1088093CA0981E0809346028091D70856
:10AFB000882309F455C08091FB08882309F450C008
:10AFC0000091D22E10E00E94B10827E239E0029FE2
:10AFD000D001039FB00D129FB00D1124A452B54FA4
:10AFE000E091CA09F0E0E851F14D90819295907F8F
:10AFF000980F9C9320E030E0C4E8D0E067E279E06D
:10B0000041E08091D22E90E02C9FF0012D9FF00D19
:10B010003C9FF00D1124DC01A69FC001A79F900D5D
:10B02000B69F900D1124E80FF91FEA58F44FDC0188
:10B03000A452B54F8C918083E091CA09F0E0EA52A6
:10B04000F14D40832F5F3F4F20313105D1F6FD0197
:10B05000EF59F74F8C9180834093D30A4093460277
:10B060008091D808882321F081E08093463307C07F
:10B070008091D908882329F01092463381E080938B
:10B08000460280911E09882361F08091FA08882386
:10B0900041F09091CC098091CD09981711F40E944C
:10B0A00059188091FC08882331F08091D7088823B3
:10B0B00011F4109226098091270990912809892B73
:10B0C00009F45AC08091D708882309F055C08091AF
:10B0D000F3088823C1F00E94B108873010F087E0A0
:10B0E00002C00E94B1088093CB098091CB09829560
:10B0F000807F2091CC09922F9F70890F8093CD097A
:10B100002817B9F539C08091C9088823A9F50E948C
:10B11000CD088823B9F00E94CD08182F0E94B108ED
:10B12000181B10930B2F0E94B1089091CB09929598
:10B13000907F980F90930C2F9093CD0981E080938E
:10B1400026090FC080912609882369F40E94B1085E
:10B150009091CB099295907F980F9093CD09109282
:10B160000B2F10920D2F9091CC098091CD0998173B
:10B1700019F081E08093D32E8091F009882301F1AA
:10B1800080910B2F8823E1F01092F00980910D2F10
:10B1900090910C2F890F8093CD099091CC0998172D
:10B1A00019F081E08093D32E80910D2F90910B2F79
:10B1B0008F5F80930D2F8150891710F010920D2F03
:10B1C0008091590990915A09019711F40E94292000
:10B1D0008091D32E8823B1F11092D32E81E08093F9
:10B1E0004602E6EDFEE21192BEE2E63EFB07D9F72B
:10B1F0001092D52E1092D30A8091C208882369F04C
:10B200008091CD096091D22E0E94BB4B8091CD09D7
:10B210008093CC090E94631F11C060E08091D22E00
:10B22000882309F461E08091CD090E94BB4B809195
:10B23000CD098093CC0981E08093D42E8091CC09F4
:10B240000E94AA308091D42E882381F08091C40975
:10B25000882361F41092D42E90E08091D22E88231E
:10B2600009F491E09093D22E0E94631F8091D1083F
:10B270008823B1F08091C908882391F4C6EDDEE2FD
:10B2800010E08881882341F018828091CC09612FD9
:10B290000E94F5460E941B331F5F2196103189F7EB
:10B2A0008091D30A8823B9F08091D108882399F03E
:10B2B0008091C908882379F48091590990915A099D
:10B2C000049749F01092D30A8091CC0960E10E9462
:10B2D000F5460E941B33809133338823A1F080917F
:10B2E000D108882381F08091C908882361F4809176
:10B2F000590990915A09049731F010923333809193
:10B30000CC090E9413308091D208882319F081E083
:10B31000809346028091590990915A09059709F046
:10B32000A0C08091C908882309F05FC080912709D7
:10B33000909128090E9413088091C2088823A9F1DE
:10B340008091ED08882321F480911E09882339F02B
:10B350001092102F10920F2F10921A3315C0809157
:10B360001009882311F18091112F882381F0809199
:10B370000C0A882349F41092102F10920F2F10926C
:10B380000C0A1092112F0EC010920C0A0BC01092D2
:10B390000C0A81E08093112F8FEF9FEF9093102F75
:10B3A00080930F2F81E0809346028091920888233A
:10B3B00059F090E080911A33882309F491E090933A
:10B3C0001A3381E080934602809110098823F1F0BE
:10B3D0008091C2088823D1F490E080910C0A8823E0
:10B3E00009F491E090930C0A0EC08091FB08882329
:10B3F00069F083E090E090935A09809359090E9484
:10B40000B1088093CA0981E0809346028091F009D7
:10B41000882339F180910B2F882319F11092F009BC
:10B4200080910D2F90910C2F890F8093CD099091D1
:10B43000CC09981719F081E08093D32E80910D2FBD
:10B4400090910B2F8F5F80930D2F8150891748F0BB
:10B4500010920D2F06C00E94B108882309F0A5CBD9
:10B4600070CBDF91CF911F910F91FF90EF90DF9004
:10B47000CF90BF90AF909F908F907F906F900895E6
:10B480008091C409882311F4109289330E94EE2E12
:10B490000E9499200E94CF100E940A450E94434FAB
:10B4A0000E943A3508952F923F924F925F926F9289
:10B4B0007F928F929F92AF92BF92CF92DF92EF9244
:10B4C000FF920F931F93DF93CF93CDB7DEB72897EB
:10B4D0000FB6F894DEBF0FBECDBF8091020A88235D
:10B4E000B1F08091D20A882391F42091CD0A309155
:10B4F000CE0A8091CF0A9091D00A8217930738F430
:10B500005F981092020A1092CE0A1092CD0A809192
:10B51000320990E0882309F491E0909332098091F8
:10B52000630960E30E940977943041F480914401FB
:10B5300090E0882309F491E090934401809163099D
:10B540006CE00E940977943071F4E091CA09F0E050
:10B55000EB5BFE4F10821092BC091092BB09109257
:10B56000BE091092BD098091C409882309F499C7C6
:10B57000E2E1F3E38481882319F18681833081F04D
:10B58000843028F4813081F08230D1F405C08430D9
:10B5900059F08530A9F40CC08091C309813081F441
:10B5A0008091630960E307C08091630960E603C08E
:10B5B0008091630968E10E940977992309F4108258
:10B5C000319623E3E431F207A9F680914E098230E7
:10B5D00028F580915209813059F0813028F082306D
:10B5E00059F08330D9F40CC08091630960E60BC038
:10B5F0008091630960E307C08091630968E103C03B
:10B60000809163096CE00E940977992339F4809155
:10B610005F09882309F491E090935F091092BA09B9
:10B620001092B9091092D40A4EE853E35A83498321
:10B6300069EF7EE27C836B83AEEC8A2EA9E09A2EC2
:10B64000FFEDAF2EF9E0BF2E5E834D8318861F827B
:10B65000E7E26E2EE9E07E2E71E0272E312C412CA0
:10B66000512CDF80A091D22E70E1D71681F48A2F61
:10B6700090E0869DF001879DF00D969DF00D1124C0
:10B68000E452F54FE05AF74FC190F0801DC08A2F69
:10B6900090E0AF81B88524E830E0A29FF001A39F3D
:10B6A000F00DB29FF00D1124AC01469DC001479DE5
:10B6B000900D569D900D1124E80FF91FE452F54F9F
:10B6C000E556FF4FC080F2903296E080809163098A
:10B6D0009C2D9695292F30E090E06C2D70E00E9413
:10B6E00015778217930731F4EF81F885E855F64F07
:10B6F00051E050838091630990E06C2D70E00E94CE
:10B7000015778217930709F068C0EF81F885E9562D
:10B71000F64F80818F5F80838081F81608F4108255
:10B7200061E0E61681F0E61640F072E0E716C9F037
:10B7300083E0E81609F051C03DC0EF81F885E95675
:10B74000F64F808108C0EF81F885E956F64F808179
:10B750009F2D981B892FEF81F885EA57F64F80833C
:10B760003CC0EF81F885EA57F64F80818F1509F0CC
:10B77000FDC6D5018C91813009F0F8C61C9206C037
:10B78000F5018081882311F421E02083D5018C917B
:10B79000EF81F885E956F64FAF81B885AA57B64FC5
:10B7A000882311F0808104C08081EF2DE81B8E2F4B
:10B7B0008C9313C02F2D30E02F5F3F4F442737FD70
:10B7C0004095542F60E070E080E090E00E94157298
:10B7D000EF81F885EA57F64F6083A091D22E4F2D66
:10B7E00050E0F0E1DF1689F52A2F30E080917409EE
:10B7F00090E0841795071CF080E090E004C08091F1
:10B80000740990E00196FC01EE0FFF1FE80FF91F8D
:10B81000269DD001279DB00D369DB00D1124EA0F55
:10B82000FB1FEF5BFC4E90819295969596959370D9
:10B8300081818770880F880F892B482F50E04051F5
:10B840005040A25CBC4EAC914DC0B0E0EF81F88599
:10B85000EC59F64F808190E0841795071CF020E0AA
:10B8600030E005C08081282F30E02F5F3F4FEF810F
:10B87000F885EE0FFF1F8F81988546E0880F991F8E
:10B880004A95E1F7E80FF91FE20FF31F3D96EE0F1F
:10B89000FF1FA69D9001A79D300DB69D300D112470
:10B8A000E20FF31FE452F54F90819295969596958D
:10B8B000937081818770880F880F892B482F50E003
:10B8C000405150406F81788584E890E0689FF00196
:10B8D000699FF00D789FF00D1124E20FF31FE758D8
:10B8E000F44FA081A150209163090F8118850F505A
:10B8F000164FF8018081EA2FF0E0EE0FFF1FE80FEE
:10B90000F11DEE0FFF1FE858FE4F80819181820FDD
:10B91000911D841B950B6C2D70E00E942977892B5B
:10B9200009F044C2EF81F885E855F64F80818823FD
:10B9300009F43CC21082D8018C9190E0882309F46C
:10B9400091E0EF81F885EF50F64F9083EF81F88515
:10B95000EB5BFE4FB1E0B083EB16A1F0EB1640F0CD
:10B96000E2E0EE16D1F0F3E0EF1609F051C03DC071
:10B97000EF81F885EB58F64F8081EF81F885EC591F
:10B98000F64F2DC0EF81F885EB58F64F8081F81AFD
:10B99000EF81F885EC59F64F26C0EF81F885EC5918
:10B9A000F64F80818F1508F4EAC5D4018C9181305F
:10B9B00009F0E5C51C9206C0F4018081882311F4CA
:10B9C00021E02083D4018C91EF81F885EC59F64F6A
:10B9D000AF81B885AB58B64F882319F08C9180831E
:10B9E00017C08C91F81AF08213C02F2D30E02F5F12
:10B9F0003F4F442737FD4095542F60E070E080E0D2
:10BA000090E00E941572EF81F885EC59F64F608343
:10BA1000A091D22EEF81F885EC59F64FB0E1DB16FC
:10BA2000C9F4808190E02A2F30E0FC01EE0FFF1F67
:10BA3000E80FF91F269DC001279D900D369D900DA2
:10BA40001124E80FF91FEE5BFC4E60816695669548
:10BA5000669525C02081EF81F885EE0FFF1F8F814D
:10BA6000988566E0880F991F6A95E1F7E80FF91F3E
:10BA7000E20FF11D3D968A2F90E0EE0FFF1F9C0113
:10BA8000269DC001279D900D369D900D1124E80F35
:10BA9000F91FE452F54F6081669566956F70EF81EE
:10BAA000F885EC59F64F808182958F70AB81BC810F
:10BAB0009C918917B1F0908192959F709C93809191
:10BAC0000A2F882329F0EF81F885E851F14D908302
:10BAD0008091590990915A09039719F4B1E0B093F4
:10BAE0004602A091D22EE0E1DE16D1F480917409D5
:10BAF00090E02A2F30E0FC01EE0FFF1FE80FF91F46
:10BB0000269DC001279D900D369D900D1124E80FB4
:10BB1000F91FEF5BFC4E808181708093D40A3AC09C
:10BB2000EF81F885EC59F64F2081EF81F885EE0F13
:10BB3000FF1F8F81988516E0880F991F1A95E1F7EE
:10BB4000E80FF91FE20FF11D3D968A2F90E0EE0FEE
:10BB5000FF1F9C01269DC001279D900D369D900DD5
:10BB60001124E80FF91FE452F54F808180FF12C0C5
:10BB70002091B9093091BA0981E090E00F8002C0AC
:10BB8000880F991F0A94E2F7822B932B9093BA099E
:10BB90008093B909EF81F885EB58F64F80818F5F6C
:10BBA00080836B3008F4AAC030E1D316B9F020913D
:10BBB000B9093091BA09D201C1010F8004C0880FC0
:10BBC000991FAA1FBB1F0A94D2F7809590958223D4
:10BBD00093239093BA098093B90902C01092D40AB2
:10BBE0006D3091F16E3030F46B3059F06C3009F0FB
:10BBF000D5C010C06E3009F440C06F3009F0CEC01F
:10BC000055C060E070E080E090E029E030E040E086
:10BC100050E054C060E070E080E090E027E030E069
:10BC200040E050E00E9415729B01AC01613071054B
:10BC30008105910509F0B2C080E1D81609F04BC02A
:10BC400091E09093D40AAAC060E070E080E090E0B8
:10BC500024E030E040E050E00E9415729B01AC010E
:10BC6000613071058105910509F098C0A0E1DA16EF
:10BC700091F5B1E0B093D40A91C060E070E080E04B
:10BC800090E023E030E040E050E00E9415729B011C
:10BC9000AC01613071058105910509F07FC0E0E1DB
:10BCA000DE16C9F4F1E0F093D40A78C060E070E0E9
:10BCB00080E090E022E030E040E050E00E94157229
:10BCC0009B01AC01613071058105910509F066C0E9
:10BCD00060E1D61679F08091B9099091BA090F8088
:10BCE00004C0220F331F441F551F0A94D2F7822B22
:10BCF000932B4DC071E07093D40A50C0862F8150B1
:10BD0000873068F470E06F5F7F4FAD81BE818C91AA
:10BD100090E00E942977892B09F440C015C0683053
:10BD200049F4ED81FE81808163E00E9409779923C7
:10BD3000A9F518C0693061F4AD81BE818C9190E0A5
:10BD400083709070892B51F5B0E1DB1671F424C03B
:10BD50006A3021F5ED81FE81808190E087709070DE
:10BD6000892BE1F4F0E1DF16B9F02091B9093091A7
:10BD7000BA09D201C1010F8004C0880F991FAA1F00
:10BD8000BB1F0A94D2F780959095822393239093BA
:10BD9000BA098093B90902C01092D40A8091B909F6
:10BDA0009091BA099093C0098093BF0920E1D216FF
:10BDB00009F479C04091D22E50E0A4E6EA2EA9E021
:10BDC000FA2E6F817885E60EF71ED7019C9180913F
:10BDD00063098B01000F111F9B01E6E0220F331F47
:10BDE000EA95E1F7020F131FF801E90FF11DEE0FBD
:10BDF000FF1F469D9001479D300D569D300D11242B
:10BE0000E20FF31FE950F54FE081E695E695E695E0
:10BE1000F0E0E659FE4FE08190E06E2F70E00E9466
:10BE20001577892B09F03FC0EE23E9F18091BF0916
:10BE30009091C0090F8002C0969587950A94E2F709
:10BE400080FF31C0F7018081F801E80FF11D3D96B8
:10BE5000EE0FFF1FE20FF31FE452F54F808180FFCA
:10BE600022C04091B9095091BA092091B909309185
:10BE7000BA09D201C1010F8004C0880F991FAA1FFF
:10BE8000BB1F0A94D2F7282B392B3093BA09209381
:10BE9000B9098091B9099091BA09842B952B909397
:10BEA000BA098093B9092F8138852F5F3F4F3887B2
:10BEB0002F834D815E814F5F5F4F5E834D836B812A
:10BEC0007C816F5F7F4F7C836B830894811C911C06
:10BED0000894A11CB11C2131310509F0C2CB80911D
:10BEE0004E09823038F480915F09882311F02C9A32
:10BEF00001C02C988091D40A882309F48FC18091C5
:10BF00000C0A882309F08AC18091D20A882309F09B
:10BF100085C18091D22EE82EFF2420917409409192
:10BF2000740987E299E0E89E8001E99E100DF89E71
:10BF3000100D1124B8016452754F615A774FDB011F
:10BF40008C91C82EDD2430E0F901EE0FFF1FE20FC7
:10BF5000F31FE00FF11FED5BFC4E80818F70F60147
:10BF6000EE0FFF1FEC0DFD1DEE0FFF1FEE0FFF1F6D
:10BF7000E80FF11DE854FE4FA081B0E0AA0FBB1FEF
:10BF8000AE56BE4F50E0FA01EE0FFF1FE40FF51F53
:10BF9000E00FF11FED5BFC4E8081869586958695BE
:10BFA000382F3E7020E08D919C91820F931F9093CB
:10BFB000D70A8093D60A809174096E5F7F4FFB0188
:10BFC0002081422F50E090E0841795071CF080E01C
:10BFD00090E004C08091740990E00196FC01EE0F9E
:10BFE000FF1FE80FF91F87E299E09C01E29EC00164
:10BFF000E39E900DF29E900D1124E80FF91FED5B6A
:10C00000FC4E30813F708091740990E08417950751
:10C010001CF080E090E004C08091740990E00196EB
:10C02000F601EE0FFF1FEC0DFD1DEE0FFF1FEE0FD3
:10C03000FF1FE30FF11DE854FE4FA081B0E0AA0FEF
:10C04000BB1FAE56BE4FFC01EE0FFF1FE80FF91FDE
:10C0500007E219E0E09EA001E19E500DF09E500D18
:10C060001124E40FF51FED5BFC4E808186958695CB
:10C070008695382F3E7020E08D919C91820F931F02
:10C080009093D90A8093D80A2091D60A3091D70A82
:10C09000445C5C4EDA016C91821B930B70E00E9451
:10C0A00029777093DB0A6093DA0AC9010E94BF0AFC
:10C0B0005F9A81E08093020A9091D10A8091D22EFA
:10C0C000682F70E0609FF001619FF00D709FF00D90
:10C0D0001124E35CFC4E8081981711F450E002C0FB
:10C0E000592F5F5F8091740990E0FC01EE0FFF1FF4
:10C0F000E80FF91F87E299E0689FD001699FB00DB2
:10C10000789FB00D1124EA0FFB1FEF5BFC4E4081BE
:10C1100046954F71A45CBC4EAC912091CF0A3091F2
:10C12000D00A8A2F90E02817390708F431C280918D
:10C130007409851709F02CC2A03671F42091CF0A3A
:10C140003091D00A842F90E00196880F991F880FB4
:10C15000991F820F931F22C0242F30E0A03359F47F
:10C160008091CF0A9091D00A2F5F3F4F220F331F4B
:10C17000280F391F20C08091CF0A9091D00A0196D4
:10C18000820F931F9093D00A8093CF0A1FC0842FF1
:10C1900090E00196880F991F880F991F9093D00AFD
:10C1A0008093CF0AF9C1242F30E0A03349F42F5FE8
:10C1B0003F4F220F331F3093D00A2093CF0AECC198
:10C1C0002F5F3F4F3093D00A2093CF0A842F90E007
:10C1D00001962A2F30E08217930721F48091740989
:10C1E0008093D10A8091740990E0FC01EE0FFF1F4B
:10C1F000E80FF91F87E299E09C01629FC001639FED
:10C20000900D729F900D1124E80FF91FEF5BFC4E0B
:10C210004F71440F8081817C842B808380917409CD
:10C2200090E02091D22E30E0FC01EE0FFF1FE80FCE
:10C23000F91F87E299E0AC01249FC001259F900D72
:10C24000349F900D1124E80FF91FED5BFC4E8081A7
:10C2500087FF10C08091DA0A9091DB0A2091D60AFC
:10C260003091D70A820F931F9093D70A8093D60AF2
:10C270000E94BF0A2091B7333091B83321153105A0
:10C28000C1F080916309E091B633F0E0E35AFD4FCD
:10C29000608190E070E00E941577892B51F48091C5
:10C2A000B9099091BA09822B932B9093BA09809384
:10C2B000B9098091B9099091BA09892BA1F18091AE
:10C2C000B9099091BA099093BC098093BB098091F8
:10C2D000BB099091BC099093BE098093BD098091E0
:10C2E000B9099091BA090E94914E80915E09882304
:10C2F00049F08091B9099091BA099F779093BA0952
:10C300008093B9092091B9093091BA0980910F2F12
:10C310009091102F80959095822393230E94550A27
:10C3200081E080936009E091E72EF0E0EB58F64F52
:10C33000808190E090936901809368017091D22E82
:10C34000472F50E087E299E0489FF001499FF00DA8
:10C35000589FF00D1124EA58F44F20E030E061E0DE
:10C36000D901AB58B64F9C918081891750F41C922B
:10C37000A981BA818C918F5F8C938150833D08F0A5
:10C380006C932F5F3F4FEC57FF4F89819A81019645
:10C390009A8389832031310519F72091850987E235
:10C3A00099E0489FF001499FF00D589FF00D11242E
:10C3B000E35CFC4E8081821768F4109285098091BD
:10C3C0009E338F5F80939E338150833D18F081E0D0
:10C3D00080939E33209168013091690187E299E052
:10C3E000489FF001499FF00D589FF00D1124E45231
:10C3F000F54F808190E08217930794F51092EE3309
:10C4000081E080930233109269011092680180915B
:10C41000D42E882329F18091590990915A098230AC
:10C42000910529F08530910511F00197C9F410921A
:10C43000D42E1092D22E772319F481E08093D22E3D
:10C440000E94631F80E090E0FC01EB58F64F1082E1
:10C45000FC01EF50F64F1082019681319105A1F752
:10C4600040916801509169018091D22E90E027E2BD
:10C4700039E0829FF001839FF00D929FF00D11240F
:10C48000E452F54F808190E001974817590749F42D
:10C490008091EE33882329F481E08093F009809322
:10C4A000EE338091C409882309F52091B733309188
:10C4B000B83321153105D1F080916309E091B6338D
:10C4C000F0E0E35AFD4F608190E070E00E94157744
:10C4D000892B61F4C9010E94914E8091B7339091EC
:10C4E000B8330E94550A81E0809360098091630906
:10C4F0008F5F809363098150803650F181E0809393
:10C5000063098091C309823010F01092C3098091B1
:10C510001633882351F08091C309813031F4809122
:10C520001833882311F41092123380911733882323
:10C5300051F08091C309813031F4809119338823FF
:10C5400011F4109213338091C3098F5F8093C30954
:10C550008091020A882321F18091CD0A9091CE0A20
:10C5600001969093CE0A8093CD0A1AC0EF81F88588
:10C57000EA57F64F8081882309F008C901C9EF8185
:10C58000F885EC59F64F8081882309F01BCA14CA3C
:10C59000A03609F008CEFBCD473109F017CE1ECEEC
:10C5A00028960FB6F894DEBF0FBECDBFCF91DF91B6
:10C5B0001F910F91FF90EF90DF90CF90BF90AF90C1
:10C5C0009F908F907F906F905F904F903F902F90B3
:10C5D000089580ED84B982EF8AB98CEF81B989E042
:10C5E00061E00E94876C12B85F980E94CF658FEF60
:10C5F0000E94AD6582E095E30E94DA6808951F927B
:10C600000F920FB60F920BB60F9211240F931F9338
:10C610002F933F934F935F936F937F938F939F934A
:10C62000AF93BF93EF93FF9300914E09013031F028
:10C630000130D8F0023009F0DBC068C08BED97E321
:10C640000E94D56E181619060CF0D2C08BED97E338
:10C650000E94066F883F08F4CBC0883F49F40E94CF
:10C66000535A0E94535A0E94535A0E94535AC0C0B0
:10C670008A3F09F045C00093C409109276011092D8
:10C68000B533109263091092CE0A1092CD0A00932E
:10C690000D2F2C982C9A10925F091092690110921C
:10C6A000680110928E0880E090E021E0FC01EB58D8
:10C6B000F64F1082FC01EF50F64F1082FC01E2535E
:10C6C000F64F2083FC01E956F64F1082FC01E85535
:10C6D000F64F2083FC01E257FC4C20830196813108
:10C6E000910521F780911633882311F010921233AF
:10C6F00080911733882309F47BC01092133378C0DC
:10C700008C3F09F075C00093893372C08091AA33C1
:10C71000882389F11092A4331092A3331092AA3384
:10C7200080916309843520F4809163098C3010F482
:10C7300010926309809163098C3038F0809163090D
:10C74000843218F488E1809363098091630984320C
:10C7500038F0809163098C3318F480E38093630987
:10C76000809163098C3338F080916309843518F423
:10C7700088E4809363090091A3331091A4336091FE
:10C780004C0270914D0280914E0290914F0228E12F
:10C7900030E040E050E00E943C770217130720F0A1
:10C7A0001092A4331092A3338091A3339091A433B9
:10C7B000892B11F40E94535A80919F339091A0339A
:10C7C000A091A133B091A2330196A11DB11D809318
:10C7D0009F339093A033A093A133B093A233809161
:10C7E000A3339091A43301969093A4338093A33301
:10C7F000FF91EF91BF91AF919F918F917F916F9139
:10C800005F914F913F912F911F910F910F900BBE10
:10C810000F900FBE0F901F901895FF920F931F93CC
:10C820008BED97E342E15AE760E070E00E944F6EC3
:10C830000E94E962E7E3F7E01082379687E0E73A83
:10C84000F807D1F710928E0810929C081092A30856
:10C85000109295081092F00882E095E367E570E089
:10C860000E94FC6782E095E36FEF0E947E6882E0A1
:10C8700095E36DEF0E947E6882E095E30E94C168B7
:10C8800082E095E367E570E043E050E00E94D26803
:10C8900082E095E30E940F68082F82E095E30E94F2
:10C8A0000F68F82E82E095E30E940F6810E00F0DEC
:10C8B000111D080F111D0430110531F00E9458336D
:10C8C0000E9459490E94E02F0E945E0B80918B3399
:10C8D000843051F40E9436338FE70E94284E80E066
:10C8E00094E00E94BF0AF8CF80918A33833041F4EC
:10C8F0000E9458330E9459490E94E02F0E949930AB
:10C900000E94473180918C33803F51F490E08091B8
:10C910008D33882309F491E090938D330E94A130E8
:10C920000E94384B80916800816080936800D89A9B
:10C9300080916B00836080936B0080E06091D22EC9
:10C940000E94BB4B0E94631F80E090E00E94550A4A
:10C950000E94C4171092B1008091B1008093B00082
:10C960008091B00082608093B0008091B1008260BD
:10C970008093B1008FE78093B30080917000826054
:10C98000809370000E943F31789489EB93E360E0DC
:10C9900044EA52E00E94A66689EB93E361E04CEA28
:10C9A00052E00E94A66689EB93E362E044EB52E01A
:10C9B0000E94A66689EB93E363E04CEB52E00E9491
:10C9C000A66689EB93E364E044EC52E00E94A6661D
:10C9D00089EB93E365E04CEC52E00E94A66689EB9C
:10C9E00093E360E142E020E00E94FC6689EB93E380
:10C9F00060E00E949C6689EB93E361E00E949C6684
:10CA000089EB93E362E00E949C6689EB93E364E028
:10CA100040E00E94CE6689EB93E364EC0E946F7065
:10CA200089EB93E36EED0E946F7089EB93E367ED02
:10CA30000E946F7089EB93E361ED0E946F7089EB48
:10CA400093E369E040E00E94CE6689EB93E36CEBF0
:10CA50000E946F7089EB93E360EB0E946F7089EB2B
:10CA600093E369EB0E946F7089EB93E36FEB0E9495
:10CA70006F7089EB93E36BEB0E946F7089EB93E32C
:10CA800060EB0E946F7089EB93E360E041E00E94ED
:10CA9000CE6689EB93E363E00E949C6689EB93E3A7
:10CAA00064E00E949C6689EB93E365E00E949C66CB
:10CAB00089EB93E366E041E00E94CE6689EB93E365
:10CAC00066E475E00E944C7060ED77E080E090E0F5
:10CAD0000E94BA6B89EB93E360E044E652E00E9467
:10CAE000A66689EB93E361E04CE652E00E94A666FD
:10CAF00089EB93E362E044E752E00E94A66689EB8B
:10CB000093E363E04CE752E00E94A66689EB93E36F
:10CB100064E044E852E00E94A66689EB93E365E096
:10CB20004CE852E00E94A66689EB93E366E044E994
:10CB300052E00E94A66689EB93E367E04CE952E07D
:10CB40000E94A66689EB93E360E142E020E00E9448
:10CB5000FC661F910F91FF900895982F8091F533F7
:10CB60008230E0F42FB7F894913029F0913060F0E2
:10CB7000923029F402C092E008C094E006C082E03E
:10CB80008093F5332FBF089591E081E08093F533D2
:10CB90008091F633892B8093F6332FBF089584E07C
:10CBA00061E00E94EB6C84E061E00E94876C8CB5D0
:10CBB00080618CBD8CB580648CBD87E061E00E9493
:10CBC000876C85E061E00E94876C08950F931F9346
:10CBD0008C01FC01868160E00E94EB6C81E090E0BA
:10CBE0000E94136CF801868161E00E94EB6C81E089
:10CBF00090E00E94136CF801868160E00E94EB6C6B
:10CC000084E690E00E94136C1F910F910895CF92DB
:10CC1000DF92EF92FF920F931F93CF93DF93D82E63
:10CC2000C92E282F392FC9018C01C0E0D0E0E62E93
:10CC3000FF24F801878161E00E94876CB7010C2E08
:10CC400002C0759567950A94E2F76170F8018781D3
:10CC50000E94EB6C21960F5F1F4FC830D10549F73A
:10CC60008D2D9C2D0E94E665DF91CF911F910F9134
:10CC7000FF90EF90DF90CF900895CF92DF92EF92E8
:10CC8000FF920F931F93CF93DF93D82EC92E282F97
:10CC9000392FC9018C01C0E0D0E0E62EFF24F80155
:10CCA000878161E00E94876CB7010C2E02C07595E8
:10CCB00067950A94E2F76170F80187810E94EB6C36
:10CCC00021960F5F1F4FC430D10549F78D2D9C2D44
:10CCD0000E94E665DF91CF911F910F91FF90EF9039
:10CCE000DF90CF9008951F93CF93DF93EC01162F21
:10CCF0008C81642F0E94EB6C8D818F3F19F060E076
:10CD00000E94EB6C8F8584FF05C0CE01612F0E94CD
:10CD100007660EC0612F70E084E0759567958A956F
:10CD2000E1F7CE010E943D66CE01612F0E943D6673
:10CD3000DF91CF911F91089541E00E94736681E0D9
:10CD400090E0089540E00E9473660895EF92FF928C
:10CD50000F931F93CF93DF938C017A016770660F57
:10CD6000660F660F60640E94A266C0E0D0E0D80142
:10CD7000ED91FC91D701AC0FBD1F0190F081E02D2A
:10CD8000C8016C9109952196C830D10581F7DF91D2
:10CD9000CF911F910F91FF90EF900895DF93CF9364
:10CDA000CDB7DEB728970FB6F894DEBF0FBECDBF64
:10CDB0009C01FE013196AFEEB6E088E00D90019245
:10CDC0008150E1F7F9018389481708F040E0E42F2A
:10CDD000F0E0EE0FFF1FEC0FFD1F8181680F606810
:10CDE000C9010E94A26628960FB6F894DEBF0FBE56
:10CDF000CDBFCF91DF910895CF93DF93EC01423007
:10CE000018F08F8588608F874B8B1C8A222329F02E
:10CE1000413019F48F8584608F8780E593EC0E9400
:10CE2000136C8C8160E00E94EB6C8E8160E00E944C
:10CE3000EB6C8D818F3F19F060E00E94EB6CCE01AE
:10CE400063E00E943D6688E893E10E94136CCE0186
:10CE500068E00E943D6688E893E10E94136CCE0171
:10CE600062E00E943D6688E893E10E94136CCE0167
:10CE700062E00E943D6688E893E10E94136CCE0157
:10CE800068E00E943D6688E893E10E94136CCE0141
:10CE900068E00E94A26688E893E10E94136CCE01CC
:10CEA00061E00E94A26688E893E10E94136CCE01C3
:10CEB00066E00E94A26688E893E10E94136CCE01AE
:10CEC00062E00E94A26688E893E10E94136CCE01A2
:10CED0006CE00E94A26688E893E10E94136CDF91E7
:10CEE000CF9108956F927F928F92AF92CF92EF92EF
:10CEF0000F931F93DF93CF93CDB7DEB73C01162F6F
:10CF0000842FF301448325830683E782C086A186AC
:10CF100082869D8593879E8594879F85958798892E
:10CF2000968761E00E94876CF30185818F3F19F03D
:10CF300061E00E94876CF301868161E00E94876C4A
:10CF4000112319F0F301178603C080E1F3018787ED
:10CF5000C30160E141E020E00E94FC66CF91DF91D7
:10CF60001F910F91EF90CF90AF908F907F906F9027
:10CF700008958F92AF92CF92EF920F931F93CF931A
:10CF8000DF93DC01362F542F722F102FAE2C8C2CF8
:10CF900013961C921E9212978BEE96E011969C931C
:10CFA0008E9300D000D0EDB7FEB73196CDB7DEB787
:10CFB0001982118212821382CD0161E0432F2FEF7B
:10CFC000052FE72EC12E0E9472670F900F900F90D1
:10CFD0000F90DF91CF911F910F91EF90CF90AF9075
:10CFE0008F90089581E08093013560937C34109296
:10CFF000FF3410920035089581E0809301356093ED
:10D000007C341092FF3410920035089520917B34C7
:10D0100030E080917A34281B3109C901089540918C
:10D020007A3480917B34481718F02FEF3FEF0AC015
:10D03000E42FF0E0E850FC4C8081282F30E04F5F77
:10D0400040937A34C9010895E0917A3480917B3419
:10D05000E81718F0EFEFFFEF06C0F0E0E850FC4CE7
:10D060008081E82FF0E0CF010895089510920535F2
:10D070001092043588EE93E0A0E0B0E0809306358E
:10D0800090930735A0930835B09309358BEF96E060
:10D0900090930335809302350895CF92DF92EF92FB
:10D0A000FF920F931F93CF93DF937C016B018A0153
:10D0B000809101358823A1F0C0E0D0E00DC0D701F8
:10D0C000ED91FC91D601AC0FBD1F0190F081E02DD8
:10D0D000C7016C9109952196C017D10780F304C050
:10D0E000CB01642F0E948369C801DF91CF911F910A
:10D0F0000F91FF90EF90DF90CF900895DF93CF9343
:10D100000F92CDB7DEB7FC0169838091013588238A
:10D11000C9F080910035823838F081E090E0938347
:10D12000828320E030E015C08091FF34E82FF0E0EA
:10D13000E358FB4C998190838F5F8093FF348093F9
:10D14000003505C0CE01019661E00E94836921E0AF
:10D1500030E0C9010F90CF91DF9108950F93062F12
:10D1600080917C346DE774E34091003521E00E94AA
:10D170002E691092FF3410920035109201350F91F4
:10D18000089561E00E94AE680895433808F042E8CF
:10D19000862F68EF73E30E94E56810927A348093DB
:10D1A0007B34089521E00E94C568089521E00E9423
:10D1B000C568089510927A3410927B341092FF342F
:10D1C000109200350E94336B0895382F433810F0C9
:10D1D00040E042C080910E358823E1F791E09093C2
:10D1E0000E35209310358FEF8093A136109298352D
:10D1F0004150409399354F5F90930F3580910F3593
:10D20000330F832B80930F3580911135813041F49A
:10D210001092113580910F358093BB0085EC01C0D1
:10D2200085EE8093BC0080910E358130E1F38091D2
:10D230009835841710F44091983520E030E00AC00A
:10D24000FB01E20FF31FD901AA5EBA4C8C918083D7
:10D250002F5F3F4F2417A0F3842F08950F931F9340
:10D26000582F122F433810F081E04AC080910E35BC
:10D270008823E1F782E080930E35009310358FEF1D
:10D280008093A1361092983540939935A6E1B5E385
:10D29000FB0102C081918D938E2F861B8417D0F3E2
:10D2A00010920F3580910F35550F852B80930F35D8
:10D2B00080911135813041F41092113580910F35F4
:10D2C0008093BB0085EC01C085EE8093BC001123E8
:10D2D00021F080910E358230E1F38091A1368F3FAD
:10D2E00011F480E00DC08091A136803211F482E00B
:10D2F00007C08091A136803311F084E001C083E043
:10D300001F910F910895482F633810F081E0089520
:10D3100080910E35843011F082E0089560931D36BF
:10D32000AAE9B5E3842F9C01F90102C081918D9394
:10D330008E2F841B8617D0F380E008951F920F92E2
:10D340000FB60F920BB60F9211242F933F934F936A
:10D350005F936F937F938F939F93AF93BF93EF935D
:10D36000FF938091B90090E0887F9070803691059E
:10D3700009F4F2C081369105CCF58832910509F4A3
:10D380007BC089329105B4F48031910509F46FC0F6
:10D39000813191053CF4009709F447C1089709F0E1
:10D3A0004FC165C08831910509F466C0809709F0C6
:10D3B00047C182C08034910509F4A4C0813491052D
:10D3C00044F48033910509F482C0C89709F038C14C
:10D3D00089C08035910509F489C08835910509F423
:10D3E00096C08834910509F02BC1AEC088399105EB
:10D3F00009F413C189399105ECF48837910509F4D2
:10D40000ABC0893791054CF48836910509F4A4C066
:10D410008037910509F014C19FC08838910509F43F
:10D42000FCC08039910509F49DC08038910509F050
:10D4300007C198C0803B910509F4C6C0813B9105A6
:10D440004CF4803A910509F49FC0883A910509F09F
:10D45000F7C0BAC0803C910509F4E3C0883C91054F
:10D4600009F4DFC0883B910509F0EAC0C2C0809191
:10D470000F358093BB00CFC090919835809199353E
:10D48000981768F490919835E92FF0E0EA5EFA4C2D
:10D4900080818093BB009F5F90939835BCC0809142
:10D4A0001035882309F44BC085ED8093BC00809132
:10D4B000BC0084FDFCCFC2C080E28093A13685ED24
:10D4C0008093BC008091BC0084FDFCCFB7C080E39A
:10D4D0008093A13685ED8093BC008091BC0084FDD3
:10D4E000FCCFACC088E38093A1369BC08091983577
:10D4F0009091BB00E82FF0E0EA5EFA4C90838F5FDA
:10D5000080939835909198358091993582C080911B
:10D5100098359091BB00E82FF0E0EA5EFA4C9083DA
:10D520008F5F8093983580911035882341F085ED89
:10D530008093BC008091BC0084FDFCCF7FC081E063
:10D540008093113584EA6EC085ED8093BC00809194
:10D55000BC0084FDFCCF72C083E080930E35109236
:10D56000A03659C08091A036823808F056C080910C
:10D57000A0369091BB00E82FF0E0E25EF94C90837A
:10D580008F5F8093A03647C08091A036823830F4F8
:10D59000E091A036F0E0E25EF94C108285ED8093D8
:10D5A000BC008091BC0084FDFCCF10920E356091D0
:10D5B000A036E0911435F09115358EE196E370E0D8
:10D5C00009951092A0362DC084E080930E351092FC
:10D5D0001C3610921D36E0911235F09113350995E5
:10D5E00080911D36882329F481E080931D361092A6
:10D5F0009A3590911C36E92FF0E0E656FA4C80817E
:10D600008093BB009F5F90931C3690911C36809155
:10D610001D36981710F485EC01C085E88093BC0096
:10D620000FC085EC8093BC0009C01092A13685ED37
:10D630008093BC008091BC0084FDFCCF10920E351D
:10D64000FF91EF91BF91AF919F918F917F916F91DA
:10D650005F914F913F912F910F900BBE0F900FBE96
:10D660000F901F90189510920E3581E08093103521
:10D670001092113581E161E00E94EB6C80E161E084
:10D680000E94EB6CE9EBF0E080818E7F80838081EB
:10D690008D7F808388E48093B80085E48093BC000C
:10D6A0000895F999FECF72BD61BDF89A80B50895CD
:10D6B000F999FECF1FBA72BD61BD40BD0FB6F89497
:10D6C000FA9AF99A0FBE08951F920F920FB60F9211
:10D6D00011242F933F938F939F93AF93BF93809188
:10D6E000A7369091A836A091A936B091AA3630916C
:10D6F000AB360196A11DB11D232F2D5F2D3720F0D4
:10D700002D570196A11DB11D2093AB368093A736EE
:10D710009093A836A093A936B093AA368091A336E9
:10D720009091A436A091A536B091A6360196A11D80
:10D73000B11D8093A3369093A436A093A536B093E1
:10D74000A636BF91AF919F918F913F912F910F90EE
:10D750000FBE0F901F9018958FB7F8942091A736A1
:10D760003091A8364091A9365091AA368FBFB901A1
:10D77000CA0108959B01AC017FB7F8948091A3364C
:10D780009091A436A091A536B091A63666B5A89B17
:10D7900005C06F3F19F00196A11DB11D7FBFBA2FC3
:10D7A000A92F982F8827860F911DA11DB11D62E01A
:10D7B000880F991FAA1FBB1F6A95D1F7BC012DC006
:10D7C000FFB7F8948091A3369091A436A091A53626
:10D7D000B091A636E6B5A89B05C0EF3F19F00196BB
:10D7E000A11DB11DFFBFBA2FA92F982F88278E0F1B
:10D7F000911DA11DB11DE2E0880F991FAA1FBB1F3B
:10D80000EA95D1F7861B970B885E9340C8F22150AA
:10D8100030404040504068517C4F21153105410552
:10D82000510571F60895019739F0880F991F880FF7
:10D83000991F02970197F1F70895789484B5826053
:10D8400084BD84B5816084BD85B5826085BD85B5A4
:10D85000816085BDEEE6F0E0808181608083E1E853
:10D86000F0E010828081826080838081816080838B
:10D87000E0E8F0E0808181608083E1EBF0E080818E
:10D8800084608083E0EBF0E0808181608083E1E967
:10D89000F0E0808182608083808181608083E0E924
:10D8A000F0E0808181608083EAE7F0E0808184603D
:10D8B0008083808182608083808181608083808199
:10D8C000806880831092C1000895982F883108F0F5
:10D8D000985197708091D4028295880F880F807C30
:10D8E000892B80937C0080917A00806480937A00F9
:10D8F00080917A0086FDFCCF2091780040917900DC
:10D90000942F80E030E0282B392BC9010895482F4F
:10D9100050E0CA0185579A4FFC01249145595A4F4E
:10D92000FA0184918823C1F0E82FF0E0EE0FFF1F89
:10D93000E35BFA4FA591B491662341F49FB7F89445
:10D940008C91209582238C939FBF08959FB7F89464
:10D950008C91822B8C939FBF08958430C9F08530C1
:10D9600038F48230F1F0833078F4813099F516C0C4
:10D970008730F9F0883018F4863061F516C08830A9
:10D98000F1F0893039F521C0809180008F7703C094
:10D99000809180008F7D80938000089584B58F777B
:10D9A00002C084B58F7D84BD08958091B0008F77CB
:10D9B00003C08091B0008F7D8093B0000895809166
:10D9C00090008F77809390000895809190008F7DD4
:10D9D000809390000895FF920F931F93F62E482F87
:10D9E00050E0CA0185559A4FFC012491CA01855720
:10D9F0009A4FFC01149145595A4FFA0104910023A2
:10DA0000C9F0222319F0822F0E94AD6CE02FF0E0C4
:10DA1000EE0FFF1FE95AFA4FA591B4919FB7F89402
:10DA2000FF2021F48C911095812302C08C91812BD1
:10DA30008C939FBF1F910F91FF90089508951F929F
:10DA40000F920FB60F920BB60F9211242F933F93A4
:10DA50004F938F939F93EF93FF934091C600209134
:10DA6000EC363091ED362F5F3F4F2F733070809141
:10DA7000EE369091EF362817390759F0E091EC36E1
:10DA8000F091ED36E455F94C40833093ED36209318
:10DA9000EC36FF91EF919F918F914F913F912F9194
:10DAA0000F900BBE0F900FBE0F901F90189508950A
:10DAB0001F920F920FB60F920BB60F9211242F9355
:10DAC0003F934F938F939F93EF93FF934091CE009B
:10DAD00020917437309175372F5F3F4F2F7330701F
:10DAE00080917637909177372817390759F0E09170
:10DAF0007437F0917537EC5CF84C40833093753790
:10DB000020937437FF91EF919F918F914F913F91A7
:10DB10002F910F900BBE0F900FBE0F901F90189576
:10DB2000E091C837F091C937E05CFF4F8191919146
:10DB300020813181821B930B8F739070892B11F0A0
:10DB40000E941E6DE091E737F091E837E05CFF4FEF
:10DB50008191919120813181821B930B8F73907001
:10DB6000892B11F00E94576D08951F920F920FB6E6
:10DB70000F920BB60F9211242F933F934F935F9305
:10DB80006F937F938F939F93AF93BF93EF93FF9385
:10DB9000209130373091313780913237909133373F
:10DBA0002817390731F48091C1008F7D8093C1001F
:10DBB00016C0E0913237F0913337E051F94C408193
:10DBC0008091323790913337019660E470E00E9483
:10DBD000297790933337809332374093C600FF9173
:10DBE000EF91BF91AF919F918F917F916F915F91D5
:10DBF0004F913F912F910F900BBE0F900FBE0F9042
:10DC00001F9018951F920F920FB60F920BB60F929E
:10DC100011242F933F934F935F936F937F938F9331
:10DC20009F93AF93BF93EF93FF932091B8373091B9
:10DC3000B9378091BA379091BB372817390731F43B
:10DC40008091C9008F7D8093C90016C0E091BA37DA
:10DC5000F091BB37E858F84C40818091BA379091E9
:10DC6000BB37019660E470E00E9429779093BB3740
:10DC70008093BA374093CE00FF91EF91BF91AF915F
:10DC80009F918F917F916F915F914F913F912F91D4
:10DC90000F900BBE0F900FBE0F901F901895AF9274
:10DCA000BF92DF92EF92FF920F931F93CF93DF9378
:10DCB000EC017A018B01DD24403081EE580780E0D1
:10DCC000680780E0780711F0DD24D39491E0A92E55
:10DCD000B12CEC89FD89DD2069F0C5010E8C02C0F4
:10DCE000880F991F0A94E2F7808360E079E08DE362
:10DCF00090E005C0108260E874E88EE190E0A80131
:10DD000097010E943C77215030404040504056954A
:10DD100047953795279580E12030380720F0DD20A2
:10DD200011F0DD24D6CFE889F9893083EA89FB89AF
:10DD30002083EE89FF89408121E030E0C9010A8C0F
:10DD400002C0880F991F0A94E2F7482B4083EE899E
:10DD5000FF894081C9010B8C02C0880F991F0A946A
:10DD6000E2F7482B4083EE89FF894081C9010C8C82
:10DD700002C0880F991F0A94E2F7482B4083EE896E
:10DD8000FF8980810D8C02C0220F331F0A94E2F7B5
:10DD9000209528232083DF91CF911F910F91FF9031
:10DDA000EF90DF90BF90AF900895DC011C96ED914D
:10DDB000FC911D97E05CFF4F219131918081918111
:10DDC000281B390B2F733070C9010895DC011C9694
:10DDD000ED91FC911D97E05CFF4F20813181E05473
:10DDE000F040DF01AE5BBF4F8D919C9111972817DA
:10DDF000390719F42FEF3FEF07C08D919C91E80F81
:10DE0000F91F8081282F30E0C9010895DC011C969C
:10DE1000ED91FC911D97E05CFF4F20813181E05432
:10DE2000F040DF01AE5BBF4F8D919C911197281799
:10DE3000390719F42FEF3FEF10C08D919C91119786
:10DE4000E80FF91F20818D919C91119701968F7396
:10DE5000907011969C938E9330E0C9010895FC0157
:10DE600086859785DC01A05CBF4FFC01EE5BFF4F10
:10DE70002D913C9111978081918128173907C1F725
:10DE80000895CF93DF93EC01462FEE85FF85E05C8C
:10DE9000FF4F80819181E054F040019660E470E092
:10DEA0000E9429779C01DF01AE5BBF4F8D919C9151
:10DEB000119728173907D1F3E05CFF4F80819181DA
:10DEC000E054F040E80FF91F4083EE85FF85E05CE9
:10DED000FF4F31832083EE89FF89208181E090E02C
:10DEE0000D8C02C0880F991F0A94E2F7282B20831B
:10DEF00081E090E0DF91CF9108951F931092BF379A
:10DF00001092BE3728EE33E040E050E02093C03757
:10DF10003093C1374093C2375093C3376BE077E0FB
:10DF20007093BD376093BC378CEA96E39093C93702
:10DF30008093C83780EF96E39093CB378093CA37AE
:10DF400085EC90E09093CD378093CC3784EC90E0D3
:10DF50009093CF378093CE3780EC90E09093D13779
:10DF60008093D03781EC90E09093D3378093D23771
:10DF700086EC90E09093D5378093D43714E01093DB
:10DF8000D637B3E0B093D737A7E0A093D837F5E002
:10DF9000F093D937E1E0E093DA371092DE37109250
:10DFA000DD372093DF373093E0374093E1375093EC
:10DFB000E2377093DC376093DB3784E397E3909329
:10DFC000E8378093E73788E797E39093EA378093C1
:10DFD000E9378DEC90E09093EC378093EB378CEC45
:10DFE00090E09093EE378093ED3788EC90E090933B
:10DFF000F0378093EF3789EC90E09093F23780937D
:10E00000F1378EEC90E09093F4378093F3371093D0
:10E01000F537B093F637A093F737F093F837E093DE
:10E02000F9371F910895CF93DF930E941D6C0E94D2
:10E030000D64C0E9DDE60E94405A2097E1F30E949A
:10E04000906DF9CFCF92DF92EF92FF920F931F93D3
:10E05000CF93DF937C016B018A01C0E0D0E00FC059
:10E06000D6016D916D01D701ED91FC910190F08188
:10E07000E02DC7010995C80FD91F015010400115A7
:10E08000110571F7CE01DF91CF911F910F91FF9094
:10E09000EF90DF90CF900895EF92FF920F931F9330
:10E0A000CF93DF937C018B01C0E0D0E0F8010F5FDC
:10E0B0001F4F6491662359F0D701ED91FC910190B7
:10E0C000F081E02DC7010995C80FD91FEFCFCE0110
:10E0D000DF91CF911F910F91FF90EF900895DC0198
:10E0E000ED91FC910190F081E02D09950895CF9379
:10E0F000DF93DB010D900020E9F71197A61BB70B0A
:10E10000EC01E881F9810280F381E02DAD010995F0
:10E11000DF91CF9108954F925F927F928F929F925D
:10E12000AF92BF92CF92DF92EF92FF920F931F9325
:10E13000DF93CF93CDB7DEB7A1970FB6F894DEBFCC
:10E140000FBECDBF2C01742ECB01223008F42AE083
:10E1500019A231E2C32ED12CCC0EDD1E822E9924C1
:10E16000AA24BB24672D752FA50194010E943C773A
:10E1700079018A01C801B701A50194010E94EA76DC
:10E18000472D461B0894C108D1084A3014F4405D5D
:10E1900001C0495CF6014083E114F1040105110559
:10E1A00021F07E2C5F2DC801DDCFC201B6010E9497
:10E1B0007770A1960FB6F894DEBF0FBECDBFCF919A
:10E1C000DF911F910F91FF90EF90DF90CF90BF9064
:10E1D000AF909F908F907F905F904F900895DC015B
:10E1E0002115310541F4ED91FC910190F081E02D74
:10E1F000642F099508950E948B700895EF92FF9205
:10E200000F931F939A017B0100E010E0B801A70172
:10E210000E94EF701F910F91FF90EF900895EF9281
:10E22000FF920F931F939A01E62EFF2400E010E067
:10E23000B801A7010E94EF701F910F91FF90EF901E
:10E240000895CF92DF92EF92FF920F931F93CF9397
:10E25000DF93EC016A017B012115310541F4E8816E
:10E26000F9810190F081E02D642F09951FC02A30BB
:10E270003105D1F477FF17C0E881F9810190F08171
:10E28000E02D6DE209958C0144275527BA014C1900
:10E290005D096E097F09CE012AE00E948B7098010A
:10E2A000280F391F04C02AE00E948B709C01C9010D
:10E2B000DF91CF911F910F91FF90EF90DF90CF9062
:10E2C0000895EF92FF920F931F937B019A0100270D
:10E2D000F7FC0095102FB801A7010E9421711F9132
:10E2E0000F91FF90EF9008950E9477700895AF927C
:10E2F000BF92CF92DF92EF92FF920F931F93CF9333
:10E30000DF935C016B01EE24FF24C0E0D0E010C07D
:10E31000D501ED91FC9100811181C601BE010E94E1
:10E320003B72682FC501F8010995E80EF91E219688
:10E33000F60184819581C817D90750F3C701DF9191
:10E34000CF911F910F91FF90EF90DF90CF90BF90F2
:10E35000AF9008952F923F924F925F926F927F926B
:10E360008F929F92AF92BF92CF92DF92EF92FF92E5
:10E370000F931F93DF93CF93CDB7DEB73B014C01D3
:10E3800019012A016D897E898F89988D6A197B0907
:10E390008C099D09621A730A840A950AA4019301E3
:10E3A0000E94EA76E218F30804091509A80197010A
:10E3B0000E945E772A0D3B1D4C1D5D1DB901CA01EF
:10E3C000CF91DF911F910F91FF90EF90DF90CF9051
:10E3D000BF90AF909F908F907F906F905F904F9085
:10E3E0003F902F900895EF92FF920F931F937B0120
:10E3F0008C01611571058105910529F420E030E05B
:10E4000040E050E00BC00E946C04A80197010E94FC
:10E410005E77AC01CB01DA019C01AD01B901CA0103
:10E420001F910F91FF90EF900895EF92FF920F933D
:10E430001F937B018C01621773078407950764F4AF
:10E44000261B370B480B590BCA01B9010E94F37107
:10E45000E60EF71E081F191FB701C8011F910F9183
:10E46000FF90EF900895009729F0BC0180E090E0C4
:10E470000E9471040895FC018481958168177907D1
:10E4800048F40190F081E02D309721F0E60FF71F5E
:10E490008081089580E00895DC01FB0114968D9140
:10E4A0009C911597892B31F461157105A9F090E0C5
:10E4B000808108C00D90BC91A02D6115710529F4D3
:10E4C00090E08C91882349F407C0CD010E945F053C
:10E4D0009C0190E0232B09F491E0892F0895CF93BC
:10E4E000DF939C01FB01EC01A881B981109729F011
:10E4F0006081718161157105D1F4C081D18120974E
:10E5000059F084819581892B39F0888190E0222708
:10E510003327281B390B12C0109771F0F901848141
:10E520009581892B49F08C91282F30E007C0CD01CF
:10E530000E945F059C0102C020E030E0C901DF912C
:10E54000CF910895FC01DB012481358114968D91D2
:10E550009C9115972817390711F020E007C0CF01CB
:10E560000E946F7220E0892B09F421E0822F089528
:10E570000F931F93CF93DF93EC018B016F5F7F4F5E
:10E58000888199810E947A04009711F480E005C087
:10E59000998388831B830A8381E0DF91CF911F9148
:10E5A0000F910895CF93DF93EC0188819981892B96
:10E5B00029F08A819B818617970760F4CE010E941B
:10E5C000B872882341F08C819D81892B19F4E881F0
:10E5D000F981108281E0DF91CF910895EF92FF924F
:10E5E0000F931F93CF93DF93EC017B016C817D81AF
:10E5F000E114F104C1F04115510599F08A01060FAB
:10E60000171FB8010E94D272882369F0888199810E
:10E610002C813D81820F931FB7010E9468051D83E5
:10E620000C8381E001C080E0DF91CF911F910F91B9
:10E63000FF90EF900895DF93CF9300D0CDB7DEB772
:10E6400069831A82BE016F5F7F4F41E050E00E94F4
:10E65000EE720F900F90CF91DF910895CF93DF93DB
:10E66000EC0188819981009711F00E94C103198201
:10E6700018821D821C821B821A82DF91CF9108951D
:10E680000F931F93182F092F0E941B73882321F4C7
:10E69000812F902F0E942E73812F902F1F910F9109
:10E6A00008950F931F93182F092FFB01608171812B
:10E6B000448155810E94EE72882321F4812F902F8E
:10E6C0000E942E73812F902F1F910F910895EF922A
:10E6D000FF920F931F93CF93DF93EC017B018A018D
:10E6E000BA010E94D272882321F4CE010E942E73B7
:10E6F00007C01D830C8388819981B7010E9468053A
:10E70000CE01DF91CF911F910F91FF90EF9008956F
:10E71000CF93DF93EC01198218821B821A821D822B
:10E720001C821E826115710551F0DB010D900020E5
:10E73000E9F71197A61BB70BAD010E946773DF9134
:10E74000CF910895CF93DF93EC01198218821B8239
:10E750001A821D821C821E826115710551F0DB0137
:10E760000D900020E9F71197A61BB70BAD010E9491
:10E770006773DF91CF9108950F931F93182F092F7F
:10E780006115710559F0DB010D900020E9F7119733
:10E79000A61BB70BAD010E94677302C00E942E73C7
:10E7A000812F902F1F910F910895EF92FF920F9359
:10E7B0001F93DF93CF93CDB7DEB761970FB6F89471
:10E7C000DEBF0FBECDBF8C01CB01F80111821082DC
:10E7D000138212821582148216827E010894E11C33
:10E7E000F11CB70150E00E949005C801B7010E94DA
:10E7F000BC7361960FB6F894DEBF0FBECDBFCF914C
:10E80000DF911F910F91FF90EF900895EF92FF928B
:10E810000F931F93DF93CF93CDB7DEB762970FB6F9
:10E82000F894DEBF0FBECDBF8C01CB01F801118281
:10E830001082138212821582148216827E0108943D
:10E84000E11CF11CB70150E00E946F05C801B7013F
:10E850000E94BC7362960FB6F894DEBF0FBECDBFA8
:10E86000CF91DF911F910F91FF90EF900895EF925C
:10E87000FF920F931F93DF93CF93CDB7DEB7299706
:10E880000FB6F894DEBF0FBECDBF8C01862FF80106
:10E89000118210821382128215821482168290E0F5
:10E8A0007E010894E11CF11CB70150E00E94900524
:10E8B000C801B7010E94BC7329960FB6F894DEBF59
:10E8C0000FBECDBFCF91DF911F910F91FF90EF90C1
:10E8D0000895DF93CF9300D0CDB7DEB7FC0111824E
:10E8E00010821382128215821482168269831A8220
:10E8F000BE016F5F7F4F0E94BC730F900F90CF914E
:10E90000DF910895DF93CF9300D0CDB7DEB7FC0140
:10E9100011821082138212821582148216826983F8
:10E920001A82BE016F5F7F4F0E94BC730F900F90E1
:10E93000CF91DF910895CF93DF93EC01FB01861710
:10E94000970761F0608171816115710529F044813B
:10E9500055810E94677302C00E942E73CE01DF9121
:10E96000CF910895FC0111821082138212821582C8
:10E97000148216820E949B740895FC0111821082F9
:10E98000138212821582148216820E949B7408954B
:10E99000FC01808191810E94C1030895FC01808166
:10E9A00091810E94C10308955058BB27AA270ED019
:10E9B00070C161D130F066D120F031F49F3F11F485
:10E9C0001EF456C10EF4E095E7FB4CC1E92F72D15D
:10E9D00080F3BA17620773078407950718F071F47C
:10E9E0009EF58AC10EF4E0950B2EBA2FA02D0B01D7
:10E9F000B90190010C01CA01A0011124FF27591B84
:10EA000099F0593F50F4503E68F11A16F040A22F89
:10EA1000232F342F4427585FF3CF469537952795FA
:10EA2000A795F0405395C9F77EF41F16BA0B620BF9
:10EA3000730B840BBAF09150A1F0FF0FBB1F661F40
:10EA4000771F881FC2F70EC0BA0F621F731F841F83
:10EA500048F4879577956795B795F7959E3F08F0A9
:10EA6000B3CF9395880F08F09927EE0F9795879568
:10EA70000895D4D008F481E008950CD00AC102D1E1
:10EA800040F0F9D030F021F45F3F19F0EBC05111A4
:10EA900034C1EEC00FD198F39923C9F35523B1F3D4
:10EAA000951B550BBB27AA2762177307840738F0FD
:10EAB0009F5F5F4F220F331F441FAA1FA9F333D05C
:10EAC0000E2E3AF0E0E830D091505040E695001C10
:10EAD000CAF729D0FE2F27D0660F771F881FBB1FCC
:10EAE000261737074807AB07B0E809F0BB0B802DA6
:10EAF000BF01FF2793585F4F2AF09E3F510568F0F2
:10EB0000B1C0FBC05F3FECF3983EDCF38695779590
:10EB10006795B795F7959F5FC9F7880F911D9695F3
:10EB2000879597F90895E1E0660F771F881FBB1F4F
:10EB3000621773078407BA0720F0621B730B840BFC
:10EB4000BA0BEE1F88F7E0950895BCD088F09F5768
:10EB500090F0B92F9927B751A0F0D1F0660F771F29
:10EB6000881F991F1AF0BA95C9F712C0B13081F009
:10EB7000C3D0B1E00895C0C0672F782F8827B85F51
:10EB800039F0B93FCCF3869577956795B395D9F76A
:10EB90003EF490958095709561957F4F8F4F9F4F74
:10EBA0000895E89409C097FB3EF490958095709580
:10EBB00061957F4F8F4F9F4F9923A9F0F92F96E9C9
:10EBC000BB279395F695879577956795B795F1113E
:10EBD000F8CFFAF4BB0F11F460FF1BC06F5F7F4FDB
:10EBE0008F4F9F4F16C0882311F096E911C07723ED
:10EBF00021F09EE8872F762F05C0662371F096E8F6
:10EC0000862F70E060E02AF09A95660F771F881FC4
:10EC1000DAF7880F9695879597F90895990F000868
:10EC2000550FAA0BE0E8FEEF16161706E807F907DE
:10EC3000C0F012161306E407F50798F0621B730B79
:10EC4000840B950B39F40A2661F0232B242B252BFA
:10EC500021F408950A2609F4A140A6958FEF811D9D
:10EC6000811D089597F99F6780E870E060E008953E
:10EC70009FEF80EC089500240A94161617061806D4
:10EC80000906089500240A941216130614060506B0
:10EC90000895092E0394000C11F4882352F0BB0F41
:10ECA00040F4BF2B11F460FF04C06F5F7F4F8F4FA4
:10ECB0009F4F089557FD9058440F551F59F05F3FDF
:10ECC00071F04795880F97FB991F61F09F3F79F08E
:10ECD00087950895121613061406551FF2CF469510
:10ECE000F1DF08C0161617061806991FF1CF869592
:10ECF0007105610508940895E894BB276627772776
:10ED0000CB0197F908958ADF08F48FEF08950BD0AF
:10ED1000C0CFB1DF28F0B6DF18F0952309F0A2CFFD
:10ED2000A7CF1124EACFC6DFA0F3959FD1F3950FAB
:10ED300050E0551F629FF001729FBB27F00DB11D7F
:10ED4000639FAA27F00DB11DAA1F649F6627B00D0F
:10ED5000A11D661F829F2227B00DA11D621F739FF8
:10ED6000B00DA11D621F839FA00D611D221F749F06
:10ED70003327A00D611D231F849F600D211D822F4D
:10ED8000762F6A2F11249F5750408AF0E1F0882394
:10ED90004AF0EE0FFF1FBB1F661F771F881F9150A1
:10EDA0005040A9F79E3F510570F05CCFA6CF5F3F62
:10EDB000ECF3983EDCF3869577956795B795F795D4
:10EDC000E7959F5FC1F7FE2B880F911D969587955C
:10EDD00097F90895629FD001739FF001829FE00D23
:10EDE000F11D649FE00DF11D929FF00D839FF00DCA
:10EDF000749FF00D659FF00D9927729FB00DE11D76
:10EE0000F91F639FB00DE11DF91FBD01CF01112452
:10EE10000895991B79E004C0991F961708F0961B76
:10EE2000881F7A95C9F780950895AA1BBB1B51E1ED
:10EE300007C0AA1FBB1FA617B70710F0A61BB70B6A
:10EE4000881F991F5A95A9F780959095BC01CD010F
:10EE5000089597FB092E07260AD077FD04D0E5DF39
:10EE600006D000201AF4709561957F4F0895F6F74B
:10EE7000909581959F4F0895A1E21A2EAA1BBB1B66
:10EE8000FD010DC0AA1FBB1FEE1FFF1FA217B30776
:10EE9000E407F50720F0A21BB30BE40BF50B661F8C
:10EEA000771F881F991F1A9469F760957095809550
:10EEB00090959B01AC01BD01CF01089597FB092EF0
:10EEC00005260ED057FD04D0D7DF0AD0001C38F439
:10EED00050954095309521953F4F4F4F5F4F089586
:10EEE000F6F790958095709561957F4F8F4F9F4F66
:10EEF0000895EE0FFF1F0590F491E02D09942F92D5
:10EF00003F924F925F926F927F928F929F92AF92B9
:10EF1000BF92CF92DF92EF92FF920F931F93CF9306
:10EF2000DF93CDB7DEB7CA1BDB0B0FB6F894DEBF9D
:10EF30000FBECDBF09942A88398848885F846E84C3
:10EF40007D848C849B84AA84B984C884DF80EE800D
:10EF5000FD800C811B81AA81B981CE0FD11D0FB616
:10EF6000F894DEBF0FBECDBFED01089515E0C2EDF0
:10EF7000D5E004C0FE010E947B772296C43DD107F4
:06EF8000C9F7F894FFCF71
:10EF8600002D00202020200078002000435600524B
:10EF960073657400544945004F666600323A330083
:10EFA600333A3400373A3800313A002B002F0070DC
:10EFB6006F733A007074726E3A002000FE370000DC
:10EFC6000100000001010000000000000000000038
:10EFD6000000000000002000280037004600550011
:10EFE6006400730082009100FFFF00030406080C12
:10EFF6001018203040600104000000000000FFFFF0
:10F006000000FEFF0000FDFF0000FCFF0000FBFF0C
:10F016000000FAFF00002B0055008000AB00D50071
:10F0260000012B0155018001AB01D5010002040549
:10F0360007090B0002050709010203040506070874
:10F04600090A0B0C0101030305060608080A0A0C47
:10F0560001010303040606080809090B010103035D
:10F0660003050508080A0A0A01010303040606083F
:10F07600080A0A0B01010202040606080809090B20
:10F086000101030305070708080A0A0C0101030327
:10F0960005060608080A0A0B01010202040606070D
:10F0A6000709090B03030000003F0000803F713D84
:10F0B600AA3F00000040713D2A4000008040E0C0A9
:10F0C600A0806040200001010004080C90010000AF
:10F0D6005802000001011018203040608018100C02
:10F0E600080604031010111204081000000017147B
:10F0F600171517000000101810100C0000000E0A5B
:10F106000E0A0E0000001B091B0A1B00010101016B
:10F11600010F1F0E00000A0A0E02020000000E0276
:10F126000E080E0000030408121313111F0000003E
:10F136000000000000180402091919111008060140
:10F14600000000000004001F0000000001020C1077
:10F156000000000001808386898C8F9295989C9F81
:10F16600A2A5A8ABAEB0B3B6B9BCBFC1C4C7C9CC23
:10F17600CED1D3D5D8DADCDEE0E2E4E6E8EAECED9F
:10F18600EFF0F2F3F5F6F7F8F9FAFBFCFCFDFEFEFC
:10F19600FFFFFFFFFFFFFFFFFFFFFFFEFEFDFCFC83
:10F1A600FBFAF9F8F7F6F5F3F2F0EFEDECEAE8E63C
:10F1B600E4E2E0DEDCDAD8D5D3D1CECCC9C7C4C10F
:10F1C600BFBCB9B6B3B0AEABA8A5A29F9C989592AA
:10F1D6008F8C898683807C797673706D6A676360AD
:10F1E6005D5A5754514F4C494643403E3B3836339F
:10F1F600312E2C2A272523211F1D1B191715131203
:10F20600100F0D0C0A090807060504030302010185
:10F2160000000000000000000000000101020303DE
:10F226000405060708090A0C0D0F10121315171905
:10F236001B1D1F212325272A2C2E313336383B3E12
:10F24600404346494C4F5154575A5D6063676A6D57
:10F25600707376797C828486888A8C8E9092949656
:10F26600989A9C9EA0A2A4A6A8AAACAEB0B2B4B628
:10F27600B8BABCBEC0C2C4C6C8CACCCED0D2D4D618
:10F28600D8DADCDEE0E2E4E6E8EAECEEF0F2F4F608
:10F29600F8FAFCFEFEFCFAF8F6F4F2F0EEECEAE818
:10F2A600E6E4E2E0DEDCDAD8D6D4D2D0CECCCAC8E8
:10F2B600C6C4C2C0BEBCBAB8B6B4B2B0AEACAAA8D8
:10F2C600A6A4A2A09E9C9A98969492908E8C8A88C8
:10F2D600868482807E7C7A78767472706E6C6A68B8
:10F2E600666462605E5C5A58565452504E4C4A48A8
:10F2F600464442403E3C3A38363432302E2C2A2898
:10F30600262422201E1C1A18161412100E0C0A0887
:10F31600060402010000020406080A0C0E1012146C
:10F3260016181A1C1E20222426282A2C2E30323487
:10F3360036383A3C3E40424446484A4C4E50525477
:10F3460056585A5C5E60626466686A6C6E70727467
:10F3560076787A7C7E800102030405060708090A8E
:10F366000B0C0D0E0F101112131415161718191A6F
:10F376001B1C1D1E1F202122232425262728292A5F
:10F386002B2C2D2E2F303132333435363738393A4F
:10F396003B3C3D3E3F404142434445464748494A3F
:10F3A6004B4C4D4E4F505152535455565758595A2F
:10F3B6005B5C5D5E5F606162636465666768696A1F
:10F3C6006B6C6D6E6F707172737475767778797A0F
:10F3D6007B7C7D7E7F808182838485868788898AFF
:10F3E6008B8C8D8E8F909192939495969798999AEF
:10F3F6009B9C9D9E9FA0A1A2A3A4A5A6A7A8A9AADF
:10F40600ABACADAEAFB0B1B2B3B4B5B6B7B8B9BACE
:10F41600BBBCBDBEBFC0C1C2C3C4C5C6C7C8C9CABE
:10F42600CBCCCDCECFD0D1D2D3D4D5D6D7D8D9DAAE
:10F43600DBDCDDDEDFE0E1E2E3E4E5E6E7E8E9EA9E
:10F44600EBECEDEEEFF0F1F2F3F4F5F6F7F8F9FA8E
:10F45600FBFCFDFEFF00FFFFFFFFFFFFFFFFFFFFBF
:10F46600FFFFFFFFFFFFFFFFFFFFFFFFFFFFFFFFA6
:10F47600FFFFFFFFFFFFFFFFFFFFFFFFFFFFFFFF96
:10F48600FFFFFFFFFFFFFFFFFFFFFFFFFFFFFFFF86
:10F49600FFFFFFFFFFFFFFFFFFFFFFFFFFFFFFFF76
:10F4A600FFFFFFFFFFFFFFFFFFFFFFFFFFFFFFFF66
:10F4B600FFFFFFFFFFFFFFFFFFFFFFFFFFFFFFFF56
:10F4C600FFFFFFFFFFFFFFFFFFFFFFFFFFFFFFFF46
:10F4D600FFFFFFFFFFFF000000000000000000002C
:10F4E6000000000000000000000000000000000016
:10F4F6000000000000000000000000000000000006
:10F5060000000000000000000000000000000000F5
:10F5160000000000000000000000000000000000E5
:10F5260000000000000000000000000000000000D5
:10F5360000000000000000000000000000000000C5
:10F5460000000000000000000000000000000000B5
:10F55600000000000000000C0D0E0F08090A0B0445
:10F5660005060700010203000000009C66227000E9
:10F5760000400014005400000000007E684D68063C
:10F58600680F682468356800000000416F2270D556
:08F596006E066FE66E2F6F0098
:00000001FF
